:020000040000FA
:040000006FD00400B9
:101000006F00907E00000000000000009020002093
:10101000AA220020A9BDF9F56C23002000000000E1
:10102000000000006C230020902000200000000041
:101030000000000090200020000000009020002010
:101040000000000090200020902000209020002030
:101050009020002090200020582F00209424002071
:101060000000000090200020902000201E2400207E
:1010700090200020D22300209020002090200020EB
:101080009020002090200020902000209020002020
:101090009020002001A04111B7170040985F3AC688
:1010A000945F3247E39CE6FE3245410182800111A4
:1010B00013078008F337078093F787083EC20100C3
:1010C0000100B7170040930570052380B70413068D
:1010D00080FA2380C7040100010083C6B70493F699
:1010E000F60DA385D704238007049246F3A6068055
:1010F0000100010093760502D5CEF336078093F602
:10110000860836C4010001002380B7042380C70489
:1011100001000100B70614007D89558D88C70100C4
:1011200001000100010023800704A246F3A6068007
:101130000100010073370780137787083AC6010062
:1011400001002380B7042380C704010001000100CF
:1011500001003727004093061005A303D7802380A2
:101160000704B247F3A70780010001009307800836
:10117000F3B7078093F787083ECE01000100B71749
:101180000040130770052380E704130780FA2380CB
:10119000E7040100010003C7B70413670708A3852C
:1011A000E70423800704F247F3A70780010001004A
:1011B0000561828093760504BDC6F336078093F6F9
:1011C000860836C8010001002380B7042380C704C5
:1011D00001000100B7061400938606047D89558D31
:1011E00088C7010001000100010023800704C246F6
:1011F000F3A6068001000100733707801377870884
:101200003ACA010001002380B7042380C70401000B
:1012100001003727004093062005A303D7802380D1
:101220000704D24781B773370780137787083ACC12
:10123000010001002380B7042380C70401000100DE
:1012400098471367070C98C723800704E24719BF24
:101250000111814601468145114506CE97000000E7
:10126000E780605893078008F3B7078093F78708F3
:101270003EC601000100B717004013077005238028
:10128000E704130780FA2380E7040100010003C785
:101290006704136717002383E70423800704B2471A
:1012A000F3A7078001000100F2400561828041112F
:1012B000814601468145114597000000E780A05214
:1012C00013078008F337078093F787083EC40100AF
:1012D0000100B7170040130670052380C70493066A
:1012E00080FA2380D70401000100FD552396B70240
:1012F00023800704A245F3A5058001000100733790
:101300000780137787083AC6010001002380C704CD
:101310002380D7040100010003C767041367170087
:101320002383E70423800704B247F3A70780010063
:10133000010001A0B1473305F50201007D1575FDDF
:101340008280411122C426C206C6AA8401446317C2
:101350009400B24022449244410182800504130566
:10136000803E420497000000E78000FD4180C5B741
:101370009305000273A04580824573901534924016
:101380002242B2424243D2436244F2440255925551
:101390002256B2564257D2576258F25806499649D9
:1013A000264AB64A464BD64B664CF64C065D965DD1
:1013B000265EB65E465FD65F09617300203041113C
:1013C000B7170040985F3AC6945F3247E39CE6FE49
:1013D000324541018280B71700401307000323887C
:1013E000E702854717170000232EF74673002030C9
:1013F000411122C42D6426C24AC006C637190040D6
:101400001304A4AAB704002023208900976000E0F9
:10141000E78000219C408297976000E0E7804020B1
:10142000E5B737370040834747009146BD8B639E41
:10143000D702B73600401306F00F973500009385AA
:10144000651F9737000083D7E72E03C7A6001377E1
:10145000F70F1DE3B7E70400BC4F09468945171590
:1014600000000345A5F7829731A099466394D70001
:10147000834757007300203003C786001377F70FA8
:10148000E365F6FC13851700AE97173800002313A9
:10149000A82A2380E70075B7B787004003C7670015
:1014A000098B6309071003C77700930600031377BE
:1014B0000703630DD708173800000348787A1736FA
:1014C00000001306E6760547B30606012380E60012
:1014D00083C577001737000013078777429793F586
:1014E000F50F2300B70003C58700973500009385EB
:1014F0002575C2951375F50F2380A50003470700D6
:1015000089451377F703630CB70C63E7E50A6306B5
:10151000071A8545630CB7129737000083C75774C5
:101520003307F600034707001377F70F19CB85073A
:1015300093F7F70F3D476363F71A17370000A301CE
:10154000F772B787004009472383E700B787004059
:1015500083C77700E207E18763DE0704973700005F
:1015600083C71770173700001307876C3E978546AF
:101570002300D700173700001307876D3E979306A7
:1015800000032300D700173700001307676B3E974F
:10159000A14685072300D70093F7F70F3D47636403
:1015A000F71417370000A30DF76AB7870040094703
:1015B0002383E70073002030930610026300D70EE8
:1015C000930620026305D70693060002E316D7F4BC
:1015D00003C727021377C70F13672700D5A803C7D0
:1015E00067001377070465CB03C7A702173800000D
:1015F00013088845173500001305C53C1347070835
:101600002385E70203C7A7021377370F1367870005
:101610002385E702814713070004B305F5008C41D9
:10162000B306F80091078CC2E399E7FEF5B503C74E
:10163000A702134707042385E70203C7A70213770E
:10164000C70F136727002385E702F9B503C76700B3
:101650001377070449C303C767021738000013084C
:101660006832173500001305A5291347070823839F
:10167000E70203C767021377370F136787002383D7
:10168000E702814713070004B305F5008C41B30658
:10169000F80091078CC2E399E7FEBDBD03C767025E
:1016A000134707042383E70203C767021377C70FB3
:1016B000136727002383E70285B503C76700137705
:1016C000070411CB03C727021377370F136787006F
:1016D0002381E70291B5238006003DBD97370000C6
:1016E000A3800758B9BD97370000A38B075675BD77
:1016F0002303048015472303E48001002302A48010
:10170000828083076480E3CE07FE23030480828007
:1017100083076480E3CE07FE03454480828083070D
:101720006480E3CE07FE2302A4808280411126C498
:101730004AC24EC006C61377F50BAD47AA892E895B
:101740009544630CF700194597000000E78080FA84
:1017500097000000E78020FB8D444E859700000035
:10176000E78040F9FD59FD1463983401B240A2446A
:101770001249824941018280135509011375F50F01
:1017800097000000E780E0F92209F1BF011126CCA3
:1017900006CEB704080097000000E780C0F61545A4
:1017A00097000000E78000F597000000E78080F6D2
:1017B00097000000E78000F62AC697000000E78047
:1017C00080F432459377150089EB13651500137586
:1017D000F50FF240E24405618280FD14E9F0014515
:1017E000CDBF397126DC4ADA4ED852D656D45AD2F9
:1017F0005ED006DE62CE66CCB7E700E07D5783AAF6
:10180000070022C603AA470023A0E71823A2E7186F
:10181000B7170040130770052380E704130780FA09
:101820002380E70483C74704930B75FFB684E20760
:1018300093FBFB0F8546AA892E8B32893724004003
:10184000E187015763FA76016308D50089461307DB
:1018500000026313D5000157D98F93F7F70FB71C18
:1018600000402382FC0411472303E4801305F00F9A
:1018700097000000E78000E8094C97000000E7802F
:1018800080E863657C15B7050700DA9537870700A0
:10189000795563FEE504B3879500636AF704370B57
:1018A0000800A94733EB65016395F90881E8814495
:1018B00097000000E78020E5268515A8DA85094510
:1018C00097000000E780C0E605090345F9FFFD1415
:1018D000050B97000000E780C0E481C49377FB0FFD
:1018E000E5F797000000E780A0EA69F17D55B7179A
:1018F0000040130770052380E704130780FA238054
:10190000E70403C74704418B2382E704F250B7E79B
:1019100000E023A0571123A24711E2543244525948
:10192000C259325AA25A125B825B724CE24C21615C
:101930008280A547639BF90685691309F00FB306FA
:101940009900B3742B01B6941349F9FFB37499004D
:10195000856B33796901416B9387F9FFB3F72701F1
:1019600099E363FC340193D94900C147E3E637FFAB
:101970003DBF0569C1697D19D9B71305800D63881D
:101980006901130500026384790113051008CA85F3
:1019900097000000E780C0D997000000E78040DF93
:1019A00031D54E99B38434416DBFDA852D4597000A
:1019B0000000E780E0D7CA94E30B99EE0509970091
:1019C0000000E78020D5A30FA9FEFDB79387F9FF9C
:1019D00093F7F70F636DFC0C83C71C0413073008E3
:1019E0006315F706370708006361EB06B3079B0032
:1019F000B706100063FBD704334BEB0089476399AC
:101A0000F9068980D549E38404EADA850945970017
:101A10000000E780E0D111090327C9FF9147232087
:101A2000E48003076480E34E07FE23033481FD173F
:101A3000EDFBFD14110B81C49377FB0FE9FF9700B9
:101A40000000E780E0D461F155B5B717004003C747
:101A50005704B70708001377070219E3B787070091
:101A60007955E376FBE833079B00E3F9E7F841B5E6
:101A70008547E380F9F0DA852D4597000000E7807F
:101A800020CB9389F4FFE38404E297000000E78011
:101A900060C893F7390091EB83260480032709007F
:101AA00093074900E396E6E03E89CE84D9BFB54767
:101AB0006399F9001305900B97000000E78080C33D
:101AC000FDB3B1471305B00AE388F9FE9947639760
:101AD000F904B7050800B365BB002D459700000069
:101AE000E78000C581448D4BA14997000000E78045
:101AF00060C263967401832704802320F900850463
:101B0000E39534FF8327048013172B0163550700E7
:101B10002312F90069BB2322F90051BB9D47639F43
:101B2000F90281451305B00497000000E78040C02A
:101B3000BD442320090023220900FD59970000001D
:101B4000E78040BD93F77400CA9703C70700FD14F0
:101B5000398D2380A700E39334FF91BBA14763979E
:101B6000F90697000000E780A0C28144630D0B00D6
:101B70008D479304C0036308FB00930400056304CE
:101B80008B01930440041375C507E30295D21945F0
:101B900097000000E78000B697000000E780A0B63D
:101BA000054597000000E780E0B426859700000017
:101BB000E78020B7094597000000E78080B69700CE
:101BC0000000E780E0BCE31405CE0DB39147639FAE
:101BD000F9001305600697000000E780A0B19700A8
:101BE0000000E78040B213059009F9B5E38109CC04
:101BF000F1547DB9BD660147173600001306C623B0
:101C0000938606A685458347060093F7F70F91C391
:101C100082800507E3F9E6FE97370000238EB720A0
:101C2000DDB77D166206618693178601E18763D46E
:101C3000070001458280931726003307F500AE9711
:101C400018439C4363E7E7007D16E37FF7FC7D556F
:101C5000828005458280FD15E205E18513978501A7
:101C6000618793F7F50F63480700FD15139725006B
:101C70002A97584365D713851700620561858280CE
:101C80003308B5021C4283A80600B335B502C297DB
:101C900033B50701AE98469585486367B5006394F0
:101CA000A50063E3070181480C43C6950CC388C2B5
:101CB0001CC2828081471397870161876343B70005
:101CC0008280139727002A97232007008507E5B70E
:101CD0008147014793968701E18663C5B6001335B6
:101CE0001700828093962700AA9694428507558F05
:101CF000D5B793D755408A07AA979C430545331516
:101D0000B5007D8D828017F3FFDFE702833D2A84D3
:101D100097000000E78060F405C5931725003E9406
:101D20000327C4FF814711EB7D1516053E9542053B
:101D3000418517F3FFDF6700033D05838507E5B79E
:101D40000145C5BF81471397870161876343C7007A
:101D5000828013972700B386E50094422A9785076F
:101D600014C3D5B77D1662066186014793178601B5
:101D7000E18763D50700133517008280931726008B
:101D8000B306F500AE9794429C437D16B58F5D8FE8
:101D9000F1BF8A05AA9501476363B500828083A6D7
:101DA000C5FFF11593D71600D98F9CC11397F60183
:101DB000E5B72A830148014701456343D700828084
:101DC000B387050183A80700B30706019C43C697A4
:101DD000AA976384F80033B517010507B308030118
:101DE000620723A0F80061871108C1BF2A83014759
:101DF0008147014563C3D70082803388E50083288B
:101E00000800330EE600032E0E003388A840330886
:101E1000C8416384080133B508018507B308E300AE
:101E2000E20723A00801E1871107E9B717F3FFDFF5
:101E3000E702232B0111B286B2842E86AA850A8579
:101E400097000000E780C0FA2A84A6850A859700DB
:101E50000000E78020E833348000060413351500C5
:101E6000018D056117F3FFDF6700E32917F3FFDF3B
:101E7000E702A3244111AA89AE8A328BB68402C23A
:101E800002C402C60144131C8401135C8C416349E3
:101E90009C02939B1400FD1B0549138CF4FFF15C1D
:101EA00033048901620461846340740792478E049D
:101EB000CE9423AEF4FE410117F3FFDF67006323E6
:101EC00013192400B30B2B01014A93172A00D6974C
:101ED00083A50B0088437800340050009700000071
:101EE000E78040DA050A93178A01E187F11BE35E78
:101EF000FCFC92474E9905042320F900A2473EC2FC
:101F0000B24702C63EC441B7131A8901135A8A4127
:101F1000131D240093178A01E18763CF970092472E
:101F20000A044E941CC0A24705091379F90F3EC25A
:101F3000B24702C63EC4ADB7B3079A0313152A00D1
:101F400056950841780034005000050AEA97DA9760
:101F50008C4397000000E780E0D26DBF197106C284
:101F600012C416C61AC81ECA22CC26CE2AD02ED219
:101F700032D436D63AD83EDA42DC46DECAC0CEC2C9
:101F8000D2C4D6C6DAC8DECAE2CCE6CEEAD0EED2F9
:101F9000F2D4F6D6FAD8FEDA971500009385058CB0
:101FA0008841E700050092402242B2424243D243B8
:101FB0006244F244025592552256B2564257D257C5
:101FC0006258F25806499649264AB64A464BD64BBD
:101FD000664CF64C065D965D265EB65E465FD65F45
:101FE0000961730020300000972100209381810156
:101FF000175100201301018117F5FFFF1305C500DC
:102000009705002093850500171600201306C6FDCE
:1020100063FAC5008322050023A055001105910530
:10202000E3EAC5FE17050200130505E59715002034
:102030009385C5FB171600201306C66563FAC50015
:102040008322050023A0550011059105E3EAC5FE92
:1020500017150020130505649745002093858529F1
:102060006377B500232005001105E36DB5FEFD4241
:10207000739002BC8D4273904280B722000093821D
:10208000828873900230970200209382A2F793E235
:1020900032007390523097420000938262767390C0
:1020A00012346FB0F47573002030397101436EC67D
:1020B00019A0397141536AC866CA62CC5ECE19A0B4
:1020C000397101535AD056D252D44ED64AD826DA54
:1020D00022DC06DE33016140828241114AC026C201
:1020E00022C406C68282B24D4101024D924C224C5E
:1020F000B24B4101024B924A224AB2494101024984
:1021000092442244B240410182803D432A87637356
:10211000C3029377F700BDEFADE5937606FF3D8AE6
:10212000BA960CC34CC30CC74CC74107E36BD7FE30
:1021300011E28280B306C3408A0697020000969699
:102140006780A6002307B700A306B7002306B700E1
:10215000A305B7002305B700A304B7002304B70005
:10216000A303B7002303B700A302B7002302B700FD
:10217000A301B7002301B700A300B7002300B700F5
:10218000828093F5F50F93968500D58D9396050182
:10219000D58D61B7939627009702000096968682A8
:1021A000E78086FA9680C1171D8F3E96E374C3F8C8
:1021B000A5B73367B500FD530D8B79E7B7877F7FF0
:1021C0009387F7F710419441B372F6003363F6003A
:1021D000BE92B3E262006397720C6318D606504158
:1021E000D441B372F6003363F600BE92B3E26200EC
:1021F0006398720A631BD60410459445B372F600C7
:102200003363F600BE92B3E262006391720A631E0A
:10221000D6025045D445B372F6003363F600BE9241
:10222000B3E26200639A72086311D60210499449BE
:10223000B372F6003363F600BE92B3E262006393BA
:1022400072085105D105E30FD6F6131706019397CF
:102250000601631CF7001357060193D706013305E7
:10226000F7409375F50F91E982804183C18333056F
:10227000F7409375F50F91E182801377F70F93F78D
:10228000F70F3305F74082800346050083C605003B
:10229000050585056313D60065FA3305D6408280AF
:1022A00011059105E312D6FE014582802105A105A5
:1022B000E31CD6FC014582803105B105E316D6FC4E
:1022C000014582804105C105E310D6FC01458280AD
:1022D000B717004003C777051377E70FA38BE70411
:1022E000130700F8A38DE7043D47238CE704130789
:1022F0005003A38CE70403C7A7051377D70F238DDB
:10230000E7048280B717004003C7E7020D89411137
:102310001377C70F498F93068008F3B6068093F6AC
:10232000860836C601000100930670052380D70495
:10233000930680FA2380D704010001002387E70277
:1023400023800704B247F3A7078001000100410181
:10235000828041112A83014E930E407E130F001993
:10236000930F400663E56E129308001913034006AD
:10237000B3781503854E0D4FA14F337365020D8958
:102380001335150063EFBE121308F6FF79467298F5
:102390004208135808013307C70213D61700BE07B7
:1023A00032976146B3F6C60213068070B386C60242
:1023B0003697A166F58F42075D8FB716004083C739
:1023C000F60293F70708A303F1000346710083C7E1
:1023D000F60293F70708E394C7FE83477100B71628
:1023E000004093F7F70F6388071293078008F3B74D
:1023F000078093F787083EC401000100B71700402B
:10240000930670052380D704930680FA2380D704AF
:102410000100010023AA070383C6170393E60608F9
:10242000A388D70223800704A247F3A707800100EF
:1024300001001166B71700407D16D45BC85F938515
:102440004703A98EF18EF5FA93068008F3B606804D
:1024500093F6860836C601000100930670052380B6
:10246000D704930680FA2380D7040100010098C1A5
:1024700003C7170313670704A388E7022380070431
:10248000B247F3A7078001000100410182807D135C
:102490003368E3039308E016630E08003368F30320
:1024A0009308D016630808009378330093B8180097
:1024B0009388D81633081E01131E0801135E0E01FF
:1024C00055B56393E5030548638608000148630337
:1024D00003002A8871087298FD15131E0801C205B1
:1024E000135E0E01C18179BD13F8150063F4BF00BE
:1024F0007908D5B713381800E5BF83C7F60293F7FC
:102500000708A303F1000346710083C7F60293F79F
:102510000708E394C7FE8347710093F7F70FF1DFD5
:10252000E9B531714AD966CB06DF22DD26DB4ED70D
:1025300052D556D35AD15ECF62CD6AC96EC7AA8C26
:1025400002D897100000E78020B12A8993078008FD
:10255000F3B7078093F787083EDA01000100B71749
:102560000040130770052380E704130780FA2380D7
:10257000E7040100010003C7F7021377770FA38771
:10258000E70203C7F70213678700A387E7022380E8
:102590000704D257F3A70780010001000545970003
:1025A0000000E78060D6130780C13347E902116A53
:1025B00093070AE893065002BD69930BA004814A71
:1025C000014B13048008930470057D1AB347F90288
:1025D0003307D7023EC0FD873ECC938709A69309F7
:1025E000803E3347F7023AC27D873AC43347390306
:1025F0008549B399990193D93940B306D702B30BF2
:102600007703B3C6F602B3CBFB0236C6FD8636C8E7
:1026100093D6FB4136CEB7460F0093860624334946
:10262000D9028566938606FAB3969601B389E902C4
:10263000130760553309D90293060010B389E902E4
:102640003349D902B3C9F9029316390036CA37198A
:102650000040FD8636D0930D090493D7F9413ED250
:10266000F336048093F6860836DC010001009307F8
:1026700070052380FD00930680FA2380DD000100B1
:1026800001008346390593F6860FA309D9048346D2
:10269000390593E61600A309D90423800D00E256FC
:1026A000F3A6068001000100130C80FA116DF336C9
:1026B000048093F6860836DE01000100930770055A
:1026C0002380FD0023808D01010001008346390530
:1026D000216693E60602A309D90483560905B3E6E9
:1026E000A6012318D90483560905D18E2318D904CD
:1026F00023800D00F256F3A60680010001008346F8
:10270000390593F606026381061A03463905218AC4
:102710006DDE081897100000E7800098733604807B
:1027200013768608B2C20100010023809D00238039
:102730008D0101000100B717004003C6370513766D
:10274000F60DA389C70403C6370513660602A389DD
:10275000C704835609052166B3E6A6012318D904E8
:1027600083560905D18E2318D90423800D0096467F
:10277000F3A60680010001008346390593F60602A0
:10278000638B061483463905A18AEDFE970000206D
:10279000E7806090AA8636D497000020E780A08F5B
:1027A000A256E30AD5FE835609054255B3E6A601B3
:1027B0002318D90497100000E780C08F834639059D
:1027C000A18AEDDE03560905834629058247337643
:1027D000CA00B306DA0293D5F641B296B388F64042
:1027E000E24733B8C6002E983308F840A247B3B684
:1027F00016013308D84063C70701631DF8009247EC
:1028000063FA1701C247634FF80E63950701B24799
:1028100063EAF80E894663E9660FF24693151800DD
:1028200013D3F8015E8613951800B365B30042D642
:1028300046D497C00100E78000CB3258050B137BCC
:10284000FB0F63470001631A0838A25863870838F2
:1028500013081500B336A800B69513D6F5013298C3
:10286000B336C800AE9613581800FE06B3E606014C
:102870007336048013768608B2C6010001002380F7
:102880009D0023808D01010001000356C902B2960C
:10289000C206C1822316D90223800D00B646F3A6D4
:1028A00006800100010021B5F336048093F6860806
:1028B000B6C00100010023809D0023808D0101002E
:1028C00001008346390593E60602A309D904238053
:1028D0000D0086460DB5F336048093F68608B6C41F
:1028E0000100010023809D0023808D010100010073
:1028F0008346390593E60602A309D90423800D0017
:10290000A646BDB5E30B0BF0F336048093F68608BC
:10291000B6C801000100930680FA23809D00238041
:10292000DD00010001008346390593F5FC0F93F6A5
:10293000860FA309D90483463905CD8EA309D9048E
:1029400023800D00C646F3A6068001000100130592
:1029500080FA03463905930639051D8A631C9629BA
:102960007336048013768608B2CC0100010013068A
:1029700080FA23809D002380CD000100010003C662
:1029800006001376F60D2380C60003C60600136604
:1029900006022380C600835609051166D18E2318CE
:1029A000D904835609052166D18E2318D9042380C2
:1029B0000D00E646F3A6068001000100130680FA2A
:1029C0008346390593F60602638006268346390559
:1029D000130C3905A18AFDDA081897000000E7807A
:1029E000A06BF336048093F68608B6D00100010090
:1029F000930680FA23809D002380DD000100010002
:102A000083460C00116693F6F60D2300DC00834626
:102A10000C0093E606022300DC0083560905D18EE4
:102A20002318D904835609052166D18E2318D904A9
:102A300023800D008656F3A60680010001001306D0
:102A400080FA8346390593F60602638A0620834698
:102A50003905A18AEDFE97F0FF1FE780C0632A8C3D
:102A600097F0FF1FE7802063E30C85FF835609057D
:102A700011664255D18E2318D90497000000E780D3
:102A800060638346390513063905A18AFDDAF336FA
:102A9000048093F68608B6D401000100930680FAFC
:102AA00023809D002380DD00010001008346060095
:102AB00093F6F60D2300D60023800D00A656F3A64C
:102AC0000680010001008356090503462905D24707
:102AD000B376DA003306CA021305800C9355F6412B
:102AE0003696330DF6408257333CD6002E9C333653
:102AF000A601330CFC40330CCC40330885039256BE
:102B00004E86B335A5033305A503C29597C00100D2
:102B1000E780609D63468001631E0C16630C0D16F2
:102B2000130615003335A6002E959356F5013696FB
:102B3000B335D600AA959396F50105828585D18E89
:102B40006346B000639D051A638B061A0356C902DB
:102B500015823305D6003336C500B2956348B00000
:102B6000639105241306F00F637DA622894663F363
:102B7000561593078008F3B7078093F78708BED6EA
:102B80000100010037170040930770052300F70488
:102B9000930780FA2300F704010001008356C7025F
:102BA00089678117D58FC207C1832316F7022300D7
:102BB0000704B657F3A7078001000100FA506A54D2
:102BC000DA544A59BA592A5A9A5A0A5BFA4B6A4C49
:102BD000DA4C4A4DBA4D296182801308F5FF33352E
:102BE000A800FD152E951356F5013298B336C8008E
:102BF000AA9695B9F336048093F68608B6CA010002
:102C0000010023809D002380AD0001000100834668
:102C10003905CD8EA309D90423800D00D646F3A62D
:102C200006800100010035B3F336048093F6860870
:102C3000B6CE0100010023809D002380CD0001005D
:102C400001008346390593E60602A309D9042380CF
:102C50000D00F646F3A606800100010095B3F33699
:102C6000048093F68608B6D20100010023809D00FF
:102C70002380CD00010001008346390593E606025A
:102C8000A309D90423800D009656F3A606800100FF
:102C9000010045BB9306F5FF33B5A600FD152E9543
:102CA0009355F501AE96B3B5B600AA951396F50106
:102CB000858269B5F336048093F68608B6D801009C
:102CC0000100930680FA23809D002380DD0001002F
:102CD00001008356C9020566011693F6F60FD18EE0
:102CE000C206C1822316D90223800D00C656F3A660
:102CF000068001000100850A93FAFA0F95B233E6C7
:102D0000B60045C20356C9023305D0403338A0008F
:102D1000B305B040B385054115826345B000D1E1EC
:102D20006371A608894663F0560593078008F3B7D8
:102D3000078093F78708BEDA01000100B71700404B
:102D4000130770052380E704130780FA2380E70444
:102D50000100010003D7C7027D8B2396E702238081
:102D60000704D65781BDF336048093F68608B6DC97
:102D700001000100930680FA23809D002380DD007E
:102D8000010001008356C9020566011693F6F60F8D
:102D9000D18EC206C1822316D90223800D00E656C9
:102DA000B9B793078008F3B7078093F78708BEDEAB
:102DB0000100010037170040930770052300F70456
:102DC000930780FA2300F704010001000356C702AD
:102DD00093975600B297C207C1832316F7022300C8
:102DE0000704F657C1BB914763EEB70217D701003E
:102DF0001307C70C8A05BA959C41BA978287B71703
:102E0000004003A7470B1345F5FF698F23AAE70A84
:102E100003A7070B698F23A8E70A03A7070A798D81
:102E200023A0A70A8280B717004083A6470B134749
:102E3000F5FFF98E23AAD70A83A6070B558D23A881
:102E4000A70A83A6070A758F23A0E70A8280B7170F
:102E5000004003A7470B498F23AAE70A03A7070BE4
:102E60001345F5FF45BFB717004083A6470B13472F
:102E7000F5FF758F23AAE70A03A7070A598D4DB7F7
:102E8000B717004003A7470B498FEDB7914763EE93
:102E9000B70217D701001307A7038A05BA959C410B
:102EA000BA978287B717004003A7470D1345F5FF70
:102EB000698F23AAE70C03A7070D698F23A8E70CE6
:102EC00003A7070C798D23A0A70C8280B7170040B9
:102ED00083A6470D1347F5FFF98E23AAD70C83A6C7
:102EE000070D558D23A8A70C83A6070C758F23A06B
:102EF000E70C8280B717004003A7470D498F23AA2C
:102F0000E70C03A7070D1345F5FF45BFB7170040B2
:102F100083A6470D1347F5FF758F23AAE70C03A778
:102F2000070C598D4DB7B717004003A7470D498FC0
:102F3000EDB7797122D43714004026D24AD0035914
:102F400024028354040206D64209C2044ECE52CC57
:102F500056CA13590901C1802DE11379F9F793F489
:102F6000F49F4209C20413590901C18093078008E4
:102F7000F3B7078093F787083EC401000100930769
:102F800070052300F404930780FA2300F404010081
:102F90000100231124032310940223000404A247F8
:102FA000F3A7078001000100B25022549254025945
:102FB000F249624AD24A45618280B7F507008146EC
:102FC0003000B105194597000020E7808081A247B5
:102FD00013972701E34A07FC1369090893E40440A7
:102FE00093098008F3B7098093F787083EC0010072
:102FF0000100930A700523005405130A80FA230088
:10300000440501000100231124032310940223002E
:1030100004048247F3A7078001000100294597F0C7
:10302000FF1FE7802031F3B9098093F989084EC268
:1030300001000100230054052300440501000100A4
:103040008357040293E707202310F40223000404AB
:103050009247B9B7B7170040884742054181937737
:10306000050491EB9377F5013755E80113050580C9
:103070003345F50282809377050C130700046397AC
:10308000E7009377F50137459C1CCDB72165130503
:1030900005D0828037E700E01C435443A183E20659
:1030A000D58F1CC1FD572320F7182322F7188280E3
:1030B00013178500B7E700E023A0E710618123A282
:1030C000A7108280B7F700E08847CC47828081470D
:1030D00037370040A14663C4C7003285828003456C
:1030E000B740E38EA6FE3385F5000345050085074E
:1030F0002304A740CDB797070020938727EF9C4371
:10310000173700201307071F3E95636EE50017373A
:1031100000201307274F6368A70017070020232705
:10312000A7EC3E858280FD57EDBF8280411122C40D
:1031300006C62A8497000000E78000F22947B307FB
:10314000E502B2408D83B3D7870222449507B3D7F7
:10315000E70237370040C207C1832316F700410159
:103160008280411137150E0006C697000000E780E7
:1031700020FCB7370040130770F82381E7000D47A4
:10318000A381E70013070004A380E7000547238716
:10319000E700B24041018280B737004003C7170003
:1031A00019C9D98DA380B70003C70700136787002B
:1031B0002380E700828093C5F5FFF98DA380B700D7
:1031C0008280AE872A87B7360040214637380040D4
:1031D00089E717030000670083F583C8B600E30999
:1031E00016FF05078348F7FFFD17C20723041801E0
:1031F000C183F9BF411122C406C62A84970000008A
:10320000E78080E52947B307E502B2408D83B3D755
:10321000870222449507B3D7E70237370040C20739
:10322000C1832316F7404101828071654111130566
:10323000052006C697000000E78000FCB737004075
:10324000130770F82381E7400D47A381E740130778
:103250000004A380E74005472387E740B2404101CF
:103260008280CC41411106C6328503C6150083C554
:10327000050022064D8E42068D654186138875A293
:10328000630C0611634BC804138845A26300060D46
:10329000634AC800938535A26301B60823900600EF
:1032A00029464DA0138855A26305060D938565A296
:1032B000E316B6FE8D451D4663E6E5081146198EF8
:1032C00063F3C7003E86B7E704002390C600FC47BF
:1032D00097D50100938505C29DA0138895A263032D
:1032E0000611634E060D1388A5A26300061393858D
:1032F00005A5E315B6FA99451D4663E5E504198E63
:1033000063F3C7003E86B7E704002390C600FC477E
:10331000970500209385C5D71DA09D451D4663E3F5
:10332000E5022146198E63F3C7003E86B7E7040025
:10333000FC472390C6009705002093852536BA9553
:1033400082970146B240328541018280AD451D46DB
:10335000E3EAE5FE3146198E63F3C7003E86B7E720
:1033600004002390C600FC4797D50100938505BB58
:10337000F9B7B1451D46E3E7E5FC3546198E63F321
:10338000C7003E86B7E704002390C600FC4797D5E8
:1033900001009385A5B965B78D451D46E3E4E5FABF
:1033A0001146198E63F3C7003E86B7E704002390E9
:1033B000C600FC4797D50100938585B449B78D4574
:1033C0001D46E3E1E5F81146198E63F3C7003E861A
:1033D000B7E704002390C600FC4797D5010093850A
:1033E000A5B6B1BFA5451D46E3EEE5F42946198E05
:1033F00063F3C7003E86B7E704002390C600FC478E
:1034000097D50100938585B01DBFB5451D46E3EBFB
:10341000E5F23946198E63F3C7003E86B7E704002C
:103420002390C600FC4797D501009385A5AB01BF4B
:10343000B7E7040003A3071397060020938646C44A
:103440004146A54517050020130585BA02832D4581
:103450005DE703C505000947631FE50803A84500AC
:10346000411106C6034718003285034608002207AB
:103470004168518F930828FE6307170563E9E80048
:1034800005186303070323900600294591A8130636
:1034900048FE630AC7041518E31707FF15463E8761
:1034A000637BF600154701A8130600023E8763748C
:1034B000F60013070002B7E704002390E600FC477C
:1034C0001316070111A83E8691C30546B7E704000D
:1034D000FC472390C6004206CC45418282970145B5
:1034E000B24041018280130600083E87E375F6FC76
:1034F00013070008C9B72390060005458280828023
:10350000416779176304E504411122C406C6854763
:103510002A84639FF500B7E7040022852244B24065
:1035200003A387139705002093858531410102830A
:1035300089476399F500B7E7040083A7070B854522
:10354000829771D9B2402244410182808280797190
:1035500026D252CCAE842A8A97D501009385C5A085
:1035600017D501001305C5A206D63AC622D44AD003
:10357000368432894ECE97B00100E7800042A285A2
:1035800017D501001305C5A197B00100E780E04001
:10359000294597B00100E780204583C7840093F751
:1035A0000702F9E383C9040089470545324763965A
:1035B000F908D44083C7160083C60600A207D58F3A
:1035C000C166138616FE638CC7028D16638FD706FD
:1035D0008D669386269029456391D706B7E7040048
:1035E000A286225403A34714B250F2494A86A68504
:1035F000025992545285624A8547456102832D459E
:103600000DEF93070002354563E98702B7E7040031
:10361000FC47C84413060002CA8582978149970770
:1036200000209387A7229C43014581CB9C4391C7EF
:103630004E852286CA8582970145B2502254925403
:103640000259F249624A456182802D457DF7930710
:10365000700F3545E3E387FEB7E70400FC47C84435
:103660002286CA85829765BF2145C1BF411122C408
:1036700037E404008327841326C2AA84416506C662
:10368000970500209385C51B7D1582978327C40A63
:1036900017050000130505E78588829795C0032369
:1036A00004132244B2409244970600209386C6AF8A
:1036B0004146C545170500201305059E41010283BB
:1036C000B2402244924401454101828019C59707C6
:1036D000002023ADA7160145828045458280114711
:1036E000636AA70A97D601009386C6860A053695AF
:1036F0001841411106C63697AE87B2850287130777
:1037000000026145639DE700B7E70400FC4713062C
:103710000002170500201305E5F882970145B24025
:103720004101828005476145E39BE7FEB7E704005E
:10373000FC470546170500201305C5F8F9BF130718
:10374000700F6145E39DE7FCB7E70400FC471306F3
:10375000700F17050020130525F7C1B713070008E0
:103760006145E39EE7FAB7E70400FC47130600084B
:10377000170500201305C5044DB715476145E390B3
:10378000E7FAB7E70400FC471546170500201305C4
:10379000650B61B709458280411126C2B7E4040078
:1037A00083A7C41322C44AC006C62E8497050020EE
:1037B000938505092A898297058905C59707002001
:1037C0009387878D83D7A70BA28503A3440D23106E
:1037D000F4002244B24092444A8502490146410124
:1037E0000283B24022449244024949454101828009
:1037F00097070020238E07049707002023AC0704B7
:10380000B717004003A7070CB706C0FFFD16758F5A
:1038100023A0E70C03A7070DB7064000558F23A888
:10382000E70C03A7070C3D9B23A0E70C03A7070D9C
:103830001367070123A8E70C8280B717004003A590
:10384000470C83A7470C598113451500C18B058987
:1038500099E3136525009707002083C767FF6380FE
:10386000A702970700202385A7FE11C9970700200C
:10387000938747FE03A3070063030300028382804C
:10388000114517F3FFFF670003CA011122CC06CED2
:103890003714004026CA4AC84EC652C48344740531
:1038A000034AB405834984050349940597F0FFFF53
:1038B000E78040A28347A40593F4F40F137AFA0F2C
:1038C00093E71700230DF40493F9F90F1379F90F17
:1038D000B717004003C7A705058B6DFF03D5C705C4
:1038E000A38D4705238C3705A38C2705A38B97044D
:1038F000F2406244D2444249B249224A0561828080
:1039000041119397050122C406C626C2C1872E84A1
:1039100063DC0700B7E40400FC54829719C1BC546F
:1039200082972165218D15A893F7150013C5150001
:103930008DE793F725009DC797000000E78020F0F2
:10394000B7E70400BC4F1306000A8945170500209D
:103950000345C5F0829713452400B24022449244A7
:10396000410182809397250163D80702B7E40400E0
:1039700083A7C41E829797000000E780A0F0BC4C8C
:1039800037560700130606308965170500200345E2
:10399000E5EC8297096579B7939715010145E3DE58
:1039A00007FA17C501001305A56797B00100E78066
:1039B000A016B7E70400BC4F130600649165170515
:1039C00000200345A5E982971165A9BF1D71A2CC0E
:1039D00037E404005C5C485886CE494697C5010030
:1039E0009385855F829711E917C50100130505606E
:1039F00097B00100E780401201A0B7F600E07957C8
:103A000098CAFD57DCCA0567B7E700E023A0E710B6
:103A10001306F00290C223A0E71801000100370747
:103A2000002018471306000481459706002023A5AF
:103A3000E6E24157A38AE7403C440808829797078B
:103A400000209387A77E3EC885671387074093872A
:103A500057D1231AE1002312F1021307B00F97F791
:103A6000FFFF938767662310E1023ED8154797074B
:103A700000009387C7E1B7F50700A30FE1003EDC24
:103A80000547970700009387E7DF81463000E1058F
:103A900019452301E1023EDE97F0FF1FE78060D465
:103AA00018088147994630003E9603460600850770
:103AB0000507A30BC700E398D7FEC24791C703577A
:103AC000410185676373F70001A0B7E7040083A78E
:103AD000470A08088297AA8511C917C5010013056E
:103AE000255297B00100E78040EB01A0F640664404
:103AF00025618280411126C2B7E4040083A704082F
:103B000006C622C4170500001305C5DF82971704F7
:103B100000201304A4D42300A40097000000E78031
:103B2000800297000000E780E0CC034504002244B7
:103B300003A38405B2409244130600328965410113
:103B40000283797106D622D413078008F3370780E1
:103B500093F787083EC201000100B71700409305A4
:103B600070052380B704130680FA2380C704010080
:103B7000010083C6F70293F6A60FA387D70223801E
:103B800007049246F3A60680010001007337078000
:103B9000137787083AC4010001002380B70423800B
:103BA000C7040100010003C7F70213672700A387BA
:103BB000E70223800704A247F3A707800100010062
:103BC000054597E0FFFFE780207497000000E7803D
:103BD00060CB014781468147054685451305407EF8
:103BE00097E0FFFFE780207737E404003C4468005B
:103BF000514681458297B707C0A83EC8B787E803FA
:103C0000938707D03ECA97E7FF1F9387477B3EC63F
:103C10007C5868008297B2502254456182804111DD
:103C200097D50100938505A217C5010013054536F8
:103C300006C697B00100E78040D617D501001305EE
:103C400025B997B00100E78040D5B2402945410130
:103C500017B30100670043D9411197D5010093853F
:103C6000A59F17C501001305A53206C697B0010030
:103C7000E780A0D217D50100130545B497B0010025
:103C8000E780A0D1B2402945410117B30100670088
:103C9000A3D5411122C406C6834705002A849DC7C7
:103CA00097D50100938505A117C501001305452E81
:103CB00097B00100E78060CE4C4017D50100130596
:103CC00065C397B00100E78040CD3DA058410DEF9E
:103CD00097D501009385059E17C501001305452B57
:103CE00097B00100E78060CB17D50100130505C22E
:103CF00097B00100E78060CA2244B24029454101E3
:103D000017B30100670043CEA1679386D7036313FF
:103D1000D70297D501009385E59917C501001305D2
:103D2000252797B00100E78040C717D5010013058C
:103D3000E5BE7DBFED0797D501009385A59717C513
:103D400001001305E524631BF70097B00100E7802D
:103D5000C0C417D501001305A5BD59BF97B0010018
:103D6000E780A0C34C4017D50100130565BE91BF85
:103D7000411197D501009385658F17C50100130583
:103D8000252106C697B00100E78020C1B240294531
:103D9000410117B30100670023C5797122D426D2EF
:103DA0004AD02E842A898145B2844800714606D6BD
:103DB00097E0FFFFE780A03597F7FF1F9387C75F66
:103DC000DC4783D70700231421012313F100975008
:103DD0000000E78060D79547A305F1009307401FD7
:103DE0003EC6FD572305A100230AF10097500000AD
:103DF000E780C0E92686A285480097500000E7804A
:103E000080D7B2502254925402594561828097273C
:103E10000020239907949727002023890780B7E77C
:103E20000400BC47411106C64146814517050020E4
:103E30001305452E8297170700200347A72F9307E6
:103E4000F00A6315F7029307F0F88945170500207B
:103E50001305452E17070020230EF72C9707002087
:103E6000A38A072C97600000E780609097600000AD
:103E7000E780C0BB8145370504009707002023A9D0
:103E800007289707002023930728970700202380FF
:103E9000072897070020239F071E97070020239DD0
:103EA000071C970700202392072697070020239BD3
:103EB000072697300000E780A017014597600000B3
:103EC000E780E09397C501009385C57C17C5010085
:103ED0001305050C97B00100E78020AC17D5010051
:103EE000130545AD97B00100E78020ABB2402945EE
:103EF000410117B30100670023AF4111814617F656
:103F0000FF1F1306A6488545170500200355851693
:103F100006C697C00000E780001A15C997C50100C2
:103F20009385057817C501001305850697B0010034
:103F3000E780A0A617D501001305C59797B001002B
:103F4000E780A0A5294597B00100E780E0A997C5C3
:103F500001009385E57417C501001305650397B04B
:103F60000100E78080A317D501001305E59597B000
:103F70000100E78080A2294597B00100E780C0A634
:103F800097F7FF1F93874743DC47054797C5010015
:103F9000938505712390E70017C50100130545FFC0
:103FA00097B00100E780609F17D5010013050593C6
:103FB00097B00100E780609EB2402945410117B3E8
:103FC0000100670063A2011122CC06CE26CA4AC8AE
:103FD0004EC693F715002E84B1CF97000000E780FE
:103FE00000F2930710F8170700202305F71497072E
:103FF000002083D7E70717070020A30DF712170546
:10400000002013052513A1839145170700202304E1
:10401000F71297070020A380071297500000E7804F
:10402000007513451400F2406244D2444249B2493B
:104030000561828093F72500E9CF17070020035719
:10404000E70C69C7AD64B71900409384A4AA23A004
:104050009900970600209386A60B944297D70100FB
:1040600093874797170600200346660A8145170580
:1040700000201305250A97700000E780801F23A009
:10408000990097F7FF1F239DA7222A8941C197C551
:1040900001009385A56717C50100130565EF97B06B
:1040A0000100E780808FCA8517C50100130505064A
:1040B00097B00100E780608E294597B00100E78046
:1040C000A0929707002023930704930710F817077F
:1040D00000202301F7069707002083D767F9170709
:1040E0000020A309F704A183170700202305F70484
:1040F00091458D47170500201305C50317070020BC
:10410000A30BF70297500000E78060661345240078
:1041100019BF93F74500D1C397C501009385055F8B
:1041200017C501001305C5E697B00100E780E086DA
:1041300017C50100130545FF97B00100E780E08532
:10414000294597B00100E780208A930720F81707D8
:1041500000202301F7FE9707002083D7A7F3170756
:104160000020A309F7FCA183170700202305F7FC13
:10417000854717070020A300F7FC97500000E78051
:10418000E0B0170500201305E5FA914597500000AF
:10419000E780E05D1345440079B593F78500A9C732
:1041A00097C501009385855617C50100130545DEA7
:1041B00097A00100E780607E17C50100130505F890
:1041C00097A00100E780607D294597B00100E78056
:1041D000A08197070020239B07F297700000E780DB
:1041E00020191345840081B593F70501D1C3854596
:1041F00017050020035505EA97600100E780E0CE2F
:1042000097C501009385855017C50100130545D852
:1042100097A00100E780607817C50100130545F3FA
:1042200097A00100E7806077294597A00100E7800B
:10423000A07B930730F817070020230DF7EE9707B0
:10424000002083D727E517070020A305F7EE170501
:104250000020130525EEA1838D4517070020230CB0
:10426000F7EC97500000E78080501345040165BBD0
:1042700093F70502D1C797C501009385254917C556
:1042800001001305E5D097A00100E780007117C574
:104290000100130525EE97A00100E7800070294575
:1042A00097A00100E7804074930740F817070020AB
:1042B0002302F7E89707002083D707DC17070020C1
:1042C000A30AF7E6A183170700202306F7E6854730
:1042D00017070020A301F7E697070020239E07D8C1
:1042E00097500000E780809A17050020130585E4A9
:1042F000914597500000E78080471345040225B39D
:1043000093F70504FDC397C501009385254017C5A4
:1043100001001305E5C797A00100E780006817C5F5
:1043200001001305A5E697A00100E7800067294575
:1043300097A00100E780406B9707002083C787DFC5
:104340001307700A6386E7061307800A638CE70881
:104350001307600A6393E704930760F817070020C8
:10436000230AF7DC9707002083D727DA17070020F6
:10437000A302F7DCA18317070020230EF7DA854795
:1043800017070020A30DF7DAB14517050020130524
:1043900065DA97500000E780803D97500000E78085
:1043A000E08E1345040497070020239007D6A5B993
:1043B000930770F817070020230EF7D69707002001
:1043C00083D7A7D417070020A306F7D6A183170722
:1043D00000202302F7D6854717070020A30EF7D445
:1043E000994565B7930780F8F1B793F7050801453C
:1043F000E38B07C297C501009385453117C50100BE
:10440000130505B997A00100E780205917C50100E1
:10441000130545D997A00100E7802058294597A0AA
:104420000100E780605C9307A0F8170700202303D2
:10443000F7D09707002083D7E7CE17070020A30BFC
:10444000F7CEA183170700202307F7CE854717076C
:104450000020A302F7CE97070020239507CC9750A2
:104460000000E780A082170500201305A5CC914528
:1044700097500000E780A02F134504086DB6411146
:1044800022C497C50100938525242A8417C50100FD
:10449000130505B006C697A00100E78000504C4008
:1044A00017C501001305853E97A00100E780E04E87
:1044B000294597A00100E780205303470400930794
:1044C000F00F631FF70297C501009385E51F17C51D
:1044D00001001305E5AB97A00100E780004C4C40BC
:1044E00017C501001305853B97A00100E780E04A4E
:1044F0002244B2402945410117A301006700C34E81
:10450000B240224441018280970700202394A7B63D
:1045100097070020239EB7B4854741111717002045
:104520002312B72417C50100130585A697C50100FE
:104530009385451517070020231DF7B21717002094
:104540002306F70E06C697A00100E78000459715E1
:10455000002083D5252117C501001305254497A008
:104560000100E7808043294597A00100E780C0470C
:1045700097F7FF1F938747E4DC4703D70700C1671E
:10458000FD176310F702B7E70400B24003A38705E5
:1045900017F5FF1F0345052D1306000A8545410148
:1045A0000283B24041018280B1C1411122C417C5CA
:1045B00001001305E59D2E8497C501009385C50B69
:1045C00006C697A00100E780403DA28517C50100FF
:1045D0001305053C97A00100E780203C2244B2402F
:1045E0002945410117A301006700034082800111A2
:1045F00022CC37E404005C5C06CE354697C501004A
:104600009385451E17D501001305C5EC829711E966
:1046100017C501001305859D97A00100E780C04FD5
:1046200001A097F7FF1F9387A7243EC4B7F50700A3
:10463000856793870780814617F6FF1F1306C622FA
:10464000E10519453EC697E0FF1FE78080197C44CD
:10465000194697F5FF1F938525211705002013059F
:10466000A5A38297340017F6FF1F1306E61F97C510
:1046700001009385A56817C501001305A56997700A
:104680000000E78000942A841DCD97C50100938522
:10469000E50617C501001305A58F97A00100E78067
:1046A000C02FA28517C501001305C51497A00100EE
:1046B000E780A02E294597A00100E780E032F24074
:1046C00062440561828097E00000E78000FA17C528
:1046D00001001305250997600000E780408897A036
:1046E0000000E780404E97600100E780C0B217F5F8
:1046F000FF1F1305E5C897600100E780609B17C5A1
:1047000001001305250797600100E78040B32A8464
:1047100097600000E78080EE97100100E780A08A94
:1047200097800100E780C02397700000E780604A0F
:1047300097600000E780806497300100E780004CBC
:1047400097C50100938585FB17C5010013054584B6
:1047500019C897A00100E7804024A28517C5010071
:104760001305850BA1B797A00100E780002317C5AB
:1047700001001305A50C97A00100E7800022294540
:1047800097A00100E780402697300100E780E027EE
:1047900097F00000E780A0467DC1854537050400FD
:1047A00097300000E780C08897C50100938505F524
:1047B00017B501001305C57D97A00100E780E01D36
:1047C00017C501001305050997A00100E780E01C4B
:1047D000294597A00100E780202197F7FF1F9387C5
:1047E00027AD83D7070017170020231DF7F685474D
:1047F00017170020230CF7E297F7FF1F9387C7BB1B
:10480000DC4703D70700C167FD176316F70097F071
:10481000FFFFE780C06E97700000E780A0C513051A
:10482000C51497700000E780A0C597200000E780BE
:10483000A0B597200000E78040A117150020035580
:1048400065F297500000E780E0C7054597500000EB
:10485000E780E0FA97C50100938545EA17B50100A6
:104860001305057397A00100E780201317C5010009
:104870001305850097A00100E780201225BD97C58C
:1048800001009385A5E717B501001305657097A092
:104890000100E780801017C501001305A51197A03E
:1048A0000100E780800F294597A00100E780C01331
:1048B000014569BF411122C437E404008327041A6B
:1048C00006C6829797500000E78080C383270408BC
:1048D00017F5FFFF1305656F829797F7FF1F238377
:1048E000A7F817F5FF1F130525AD97400000E780D7
:1048F000806C2244B240410117030000670063CF7F
:10490000B7E70400FC471171A2DDCAD986DFA6DB38
:10491000CED72E8432892E86AA851705002013054E
:1049200065818297170700201307C7808347070018
:10493000930680029387E70793F7F70FE3ECF610EF
:10494000BA898A0717B701001307C76DBA979C4346
:10495000BA9782878D4797C50100938565DC17B5A7
:1049600001001305E562630FF40097A00100E780E2
:10497000C00217C501001305659997A00100E780E3
:10498000C001BDA497A00100E780200117C5010068
:104990001305459997A00100E7802000294597A0BD
:1049A0000100E7806004930720F8114697F5FF1F88
:1049B000938545784A8517F7FF1F230DF77697F7FC
:1049C000FF1FA38A077697F0FFFFE780403D2A8408
:1049D0001DC997C501009385A5D417B5010013051E
:1049E000255B97A00100E78040FBA28517C5010069
:1049F0001305059797A00100E78020FA294597A0A5
:104A00000100E78060FE97C50100938565D117B569
:104A100001001305E55797A00100E78000F817C5CE
:104A200001001305259597A00100E78000F72945AF
:104A300097A00100E78040FB4165930730FA0546E7
:104A400097F5FF1F9385056F7D1517F7FF1F23034C
:104A5000F76E97F0FFFFE78080342A841DC997C561
:104A600001009385E5CB17B501001305655297A0AA
:104A70000100E78080F2A28517C501001305458E6D
:104A800097A00100E78060F1294597A00100E78029
:104A9000A0F5B7E70400BC4F0566130606C8A1459C
:104AA00017F5FF1F034505DC8297FE506E54DE5458
:104AB0004E59BE591161828091476303F40297C534
:104AC00001009385E5C517B501001305654C97A056
:104AD0000100E78080EC17C501001305E58C71BD6E
:104AE000B7E70400FC4F914517F5FF1F034585D735
:104AF000829797C501009385A5C217B501001305DC
:104B0000254997A00100E78040E917C5010013057A
:104B1000658B97A00100E78040E8294597A0010038
:104B2000E78080EC97400000E7804016914535A46F
:104B300085476303F40297C50100938565BE17B5E9
:104B400001001305E54497A00100E78000E517C5C3
:104B500001001305A58815B597F7FF1F239C275360
:104B6000B7E704000566BC4F130606C8C1450DBF74
:104B70008D476303F40297C50100938565BA17B5A5
:104B800001001305E54097A00100E78000E117C58B
:104B9000010013056586D5B3930740F8114697F5D4
:104BA000FF1F938525594A8517F7FF1F2304F758E0
:104BB00097F7FF1FA381075897F0FFFFE780201E9C
:104BC0002A84E30405EE97C50100938565B517B502
:104BD00001001305E53B97A00100E78000DCA285FA
:104BE00017B501001305C57797A00100E780E0DA4B
:104BF000294597A00100E78020DF45BD9147E31CD0
:104C0000F4F6B7E70400FC4F9305000217F5FF1F09
:104C1000034545C5829797C50100938565B017B5D3
:104C200001001305E53697A00100E78000D717B50E
:104C300001001305E57DF1BD894763E3870297C550
:104C400001009385E5AD17B501001305653497A004
:104C50000100E78080D417B501001305A57C31BBA6
:104C600097F4FF1F83C4244D97F7FF1F83C7974C0A
:104C700097C501009385C5AAA20417B501001305C5
:104C80002531DD8C97A00100E78020D1A28517B5E2
:104C900001001305657A97A00100E78000D0C204E7
:104CA000294597A00100E78020D4C1849305D4FF53
:104CB00093960401C1824A8693F5F50F17F5FF1FFD
:104CC0001305754797200000E780403AE35F90DCCA
:104CD000930750F817F7FF1F230EF74483C73900D7
:104CE000228697F5FF1F9385E54485074A8517F7C8
:104CF000FF1FA302F74497F0FFFFE780400A2A84D2
:104D0000E30505DA97C50100938585A117B5010074
:104D10001305052897A00100E78020C8A28517C5C4
:104D200001001305E5C5C9B5894763E3870297C547
:104D300001009385E59E17B501001305652597A031
:104D40000100E78080C517B501001305A57035B1D6
:104D500097400000E78080F3A28517F5FF1F130539
:104D6000653D97500000E78080A081B38D476303C5
:104D7000F40297C501009385A59A17B501001305A4
:104D8000252197A00100E78040C117B50100130558
:104D9000256EE5B6B76602000146B7750200054507
:104DA00097E0FF1FE780E0A3930760F817F7FF1F66
:104DB0002302F73897F7FF1FA38F073693070006E4
:104DC00017F7FF1F230AF736894717F7FF1FA305B9
:104DD000F73697F7FF1F2382073697F7FF1FA38E3B
:104DE0000734C14717F7FF1F230AF734930720F949
:104DF00017F7FF1FA304F734314697F7FF1FA3806F
:104E0000A73497F5FF1F9385E5324A8597F7FF1F73
:104E10002387073297F0FFFFE78060F82A84E306D4
:104E200005C897C501009385A58F17B50100130527
:104E3000251697A00100E78040B6A28517B50100AE
:104E40001305856455B3B1476303F40297C50100A8
:104E50009385058D17B501001305851397A00100F3
:104E6000E780A0B317B501001305C56339B6B7E7EE
:104E70000400FC4F9305000417F5FF1F0345859EB2
:104E8000829797400000E78060E0B145F9B591470F
:104E900063E3870297C501009385858817B50100F4
:104EA0001305050F97A00100E78020AF17B501009B
:104EB00013050561D9B497F4FF1F83C4E42797F75E
:104EC000FF1F83C75727A204DD8C8E04B77702002B
:104ED0006D14BE942286A68517B501001305855F63
:104EE00097A00100E78060ABB7E70400FC4722868B
:104EF00097F5FF1F93855524280082979316040188
:104F0000C1823000A685094597E0FF1FE780608DCC
:104F10002A8409C917B501001305855D97A0010012
:104F2000E78080BF930770F8194697F5FF1F9385B8
:104F300065204A8517F7FF1F230EF71E97F7FF1FFF
:104F4000A38C871E97F0FFFFE78060E52A84E30EBD
:104F500005B497B501009385A57C17B5010013052D
:104F6000250397A00100E78040A3A28517B50100A3
:104F70001305055995B99947630BF41297B50100CC
:104F80009385057A17B501001305850097A00100E8
:104F9000E780A0A017B5010013050558F9BA91479D
:104FA00063E3870297B501009385857717B5010004
:104FB000130505FE97A00100E780209E17B50100AC
:104FC000130505575DBA97F4FF1F83C4E41697F7DE
:104FD000FF1F83C75716A204DD8C8E04B77702002B
:104FE0006D14BE942286A68517B50100130585555C
:104FF00097A00100E780609AB7E70400FC4722868B
:1050000097F5FF1F93855513280082979316040187
:10501000C1823000A6850D4597D0FF1FE780607CD8
:105020002A8409C917B501001305855397A001000B
:10503000E78080AE930780F8194697F5FF1F9385A8
:10504000650F4A8517F7FF1F2306F70E97F7FF1F17
:10505000A384870E97F0FFFFE78060D42A84E306DD
:1050600005A497B501009385A56B17B5010013053D
:1050700025F297A00100E7804092A28517B50100B4
:105080001305454F95B699476303F40297B50100A0
:105090009385056917B50100130585EF97A00100F9
:1050A000E780A08F17B501001305454EF9B0B7E7AB
:1050B0000400FC4F9305000417E5FF1F0345857AA4
:1050C000829797400000E78060BC994579B18D4791
:1050D0006303F40297B501009385856417B5010059
:1050E000130505EB97A00100E780208B17B50100A1
:1050F0001305454B59B017B501001305A54B97A0F3
:105100000100E78060A11305C01297D0FF1FE78060
:105110004023014597E0FFFFE78000F80D45971019
:105120000000E78080A0294597D0FF1FE78060211D
:1051300097D0FF1FE780C0118DBA99476303F4022F
:1051400097B501009385C55D17B50100130545E4CA
:1051500097A00100E780608417B50100130545465C
:1051600029B817F7FF1F034737FD97F7FF1F83C7BE
:10517000A7FC22075D8F9166BA96C2061166C182AE
:105180001306F6EF8D476365D60297E7FF1F9387F7
:10519000A7229C4B17F6FF1F0346F6F99386C7001C
:1051A0002DC203D6070069CA8907E39CD7FE894749
:1051B0001307A0F8114697F5FF1F9385A5F74A85B9
:1051C00097F6FF1F2388E6F617F7FF1FA305F7F6EC
:1051D00097F0FFFFE780A0BC2A84E308058C97B511
:1051E00001009385E55317B50100130565DA979023
:1051F0000100E780807AA28517B501001305853D7F
:10520000E5B203D60700630EE60A8907E39BF6FEC4
:105210008D4779BF91476304F40297B501009385E8
:10522000255017B501001305A5D697900100E7801A
:10523000C07617B501001305653B6FF00FF4B7E7B3
:105240000400FC4F9305000817E5FF1F0345856127
:105250008297C9B897B501009385854C17B50100B1
:10526000130505D397900100E780207317B501005F
:10527000130545396FF06FF02390E70017E5FF1F26
:105280001305851397300100E780A09D97B50100B5
:105290009385054917B50100130585CF9790010047
:1052A000E780A06F17B501001305C5369790010080
:1052B000E780A06E294597900100E780E072814762
:1052C000C5BD2390070017E5FF1F1305E50E9730B6
:1052D0000100E780009997B501009385654417B5F3
:1052E00001001305E5CA97900100E780006B17B530
:1052F00001001305A5335DBF411122C406C68347D3
:1053000005002A849DC797B501009385253D17B5F3
:1053100001001305E5C797900100E78000684C4045
:1053200017B501001305056C97900100E780E06652
:10533000C9A85841B707CF009387777D6312F70854
:1053400097B501009385853917B50100130545C44C
:1053500097900100E78060641C448356E400835505
:10536000C40003C6070017B501001305256997900F
:105370000100E7808062294597900100E780C066C0
:105380000357E4009707002083D7C73D630EF7005B
:105390008355C4000844854717070020230BF738BE
:1053A00097300000E780202E0356E4008355C400A8
:1053B00008442244B240410117F3FFFF67008354C1
:1053C000B707CC009387777D6315F70497B5010085
:1053D0009385C53017B50100130585BB9790010073
:1053E000E780A05B1C448356E4008355C40003C6D9
:1053F000070017B501001305656097900100E7806D
:10540000C0592244B2402945410117930100670069
:10541000A35DB707CE009387777D6304F70297B546
:1054200001009385A52B17B50100130565B697906C
:105430000100E78080564C4017B501001305455127
:10544000E5B5B240224441018280B7E70400FC4741
:1054500041112E8606C622C426C24AC02E842A893D
:10546000AA8517F5FF1F1305E5CC829797B50100B4
:105470009385C52C17B50100130585B197900100E0
:10548000E780A05197F5FF1F83C5C5CA17B5010076
:105490001305C5D297900100E780205029459790C9
:1054A0000100E780605497F4FF1F9384A4C883C76A
:1054B000040041479387070693F7F70F636EF75A87
:1054C00017B70100130747C08A07BA979C43BA97DA
:1054D00082879D476307F40297B5010093850526EF
:1054E00017B501001305C5AA97900100E780E04AAF
:1054F00017B50100130505CD97900100E780E0493D
:105500008DA497F7FF1F83C7F7C2DDCB17F7FF1FE7
:10551000034777C297F7FF1F83C7E7C122075D8F55
:1055200097F7FF1F83C747C1C2075D8F97F7FF1F1C
:1055300083C797C0E207D98F17F7FF1F232AF7BC4D
:1055400083C7640097B501009385451F17B5010017
:10555000130505A417F7FF1F230BF7BA9790010057
:10556000E780A04397F7FF1F938787BA8C4317F60E
:10557000FF1F0346C6B917B50100130565C697900E
:105580000100E7808041294597900100E780C045F0
:1055900097F7FF1FA38007BA2244B2409244024902
:1055A000930700F817F7FF1F2306F7B89D4517F577
:1055B000FF1F130525B84101174300006700231B97
:1055C00097600000E78040EA97F7FF1F2385A7B6A2
:1055D0009357850017F7FF1FA30FF7B493570501E3
:1055E0002A8417F7FF1F2309F7B493578501014554
:1055F00017F7FF1FA302F7B497600000E78020EBC6
:1056000097F7FF1F238BA7B297B50100938505136A
:1056100017B501001305C59797900100E780E037A3
:1056200017F6FF1F034666B1A28517B501001305E3
:10563000A5BCB1B7CD476303F40297B501009385CC
:10564000E50F17B501001305A59497900100E780B9
:10565000C03417B501001305A5BB79BD37E40400BC
:105660007C44414697F5FF1F9385D5AC17F5FF1F86
:10567000130545AA829797F7FF1F83C7C7AC17F793
:10568000FF1F034737ACA20703238405D98F17F701
:10569000FF1F231DF7A61306000A89452244B240C6
:1056A0009244024917E5FF1F0345C51B41010283D0
:1056B0008D476303F40297B501009385250817B55C
:1056C00001001305E58C97900100E780002D17B5C8
:1056D00001001305A5C30DB517F4FF1F0344A4A5CE
:1056E00097F7FF1F83C717A597B501009385050599
:1056F000220417B501001305A5895D8C9790010060
:10570000E780A029A28517B501001305E5B19790A0
:105710000100E7808028294597900100E780C02C90
:105720000D4697F5FF1F9385E5A0228597E0FFFFC3
:10573000E780E066AA8421C197B501009385050042
:1057400017B501001305C58497900100E780E02498
:10575000A68517B50100130565AE97900100E78097
:10576000C0232244B2409244024929454101179383
:1057700001006700632797F7FF1F239D8790B7E716
:105780000400116603A38705130606E8914539B79F
:105790008D476303F40297B50100938525FA17A599
:1057A00001001305E57E97900100E780001F17B503
:1057B0000100130565C489B317F4FF1F0344A497C0
:1057C00097F7FF1F83C7179797B50100938505F7D4
:1057D000220417A501001305A57B5D8C979001009D
:1057E000E780A01BA28517B50100130565A6979059
:1057F0000100E780801A294597900100E780C01ECC
:105800000D4697F5FF1F9385E592228597E0FFFFF0
:10581000E780E058AA841DC197B50100938505F281
:1058200017A501001305C57697900100E780E016E3
:10583000A68517B501001305E5A205B797F7FF1F69
:10584000239C8782B7E70400116603A3870513062C
:1058500006E89305000299B5894763E3870297B587
:1058600001009385A5ED17A50100130565729790BA
:105870000100E780801217B501001305A5BAADB984
:1058800097F4FF1F83C4248B97F7FF1F83C7978A62
:1058900097B50100938585EAA20417A501001305B9
:1058A000256FDD8C97900100E780200FA68517B546
:1058B00001001305A59C97900100E780000E294583
:1058C00097900100E7804012228697F5FF1F93858D
:1058D0006586268597E0FFFFE780604C2A84630E8B
:1058E000051A97B50100938565E517A50100130515
:1058F000256A97900100E780400AA28517B501004C
:105900001305059999BD854763F9871883451900E3
:105910002244B24092440249B335B00097E7FF1FDA
:105920002384B77817B501001305C5974101179374
:10593000010067008306A2852244B24092444A8552
:10594000024941011703000067006324994763037C
:10595000F40297B50100938565DE17A501001305D4
:10596000256397900100E780400317B501001305F8
:1059700025C559B617E4FF1F0344E47B97E7FF1FD3
:1059800083C7577B97B50100938545DB220417A594
:1059900001001305E55F5D8C97900100E780E0FF53
:1059A000A28517B501001305659197900100E78066
:1059B000C0FE294597900100E7800003194697E54E
:1059C000FF1F93852577228597E0FFFFE780203D25
:1059D000AA841DC197B50100938545D617A501007E
:1059E0001305055B97900100E78020FBA68517B59E
:1059F00001001305A58D95B397E7FF1F23948772C8
:105A0000B7E70400116603A38705130606E89305AC
:105A1000000869B1854797B50100938525D217A580
:105A200001001305E556630BF40097900100E78031
:105A3000C0F617B501001305A58A7DBC979001003B
:105A4000E780A0F517B501001305058B97900100BD
:105A5000E780A0F4294597900100E780E0F8224410
:105A6000B2409244024997E7FF1F2391076A410120
:105A7000176300006700C38F97B50100938505CCBD
:105A800017A501001305C55097900100E780E0F0CD
:105A900017B50100130505B785B4B24022449244FE
:105AA000024941018280411106C622C497E0FFFFEE
:105AB000E780E02E21CD97E7FF1F83D7075F85079B
:105AC0002A8417E7FF1F2312F75E97B5010093851D
:105AD00065C897E7FF1F239BA75C17A50100130567
:105AE000254B97900100E78040EBA28517B5010098
:105AF000130505E997900100E78020EA2244B240AF
:105B00002945410117930100670003EE97E7FF1F46
:105B100083D7E759B2402244850717E7FF1F2318B0
:105B2000F75841018280411122C491462A8417E628
:105B3000FF1F1306266E9D652D4506C697D0FF1FD5
:105B4000E78020CAB7F7070003C70701A54763131B
:105B5000F70001A09306001001469D65254597D0EA
:105B6000FF1FE78000C897E7FF1F2385876A22444D
:105B7000B240914617E6FF1F1306C6699D65294589
:105B8000410117D3FF1F6700C3C51171CED7B7E915
:105B9000040083A7C904CAD917E9FF1F130989594B
:105BA000A2DD2E8686DFA6DB2E84AA854A85829713
:105BB00097E7FF1F83C707581307700A6385E7102D
:105BC000636DF7001307600A6385E704FE506E54A7
:105BD000DE544E59BE59116182801307800A6385D5
:105BE000E7161307900AE393E7FE8D476306F41C5C
:105BF00097B50100938505EC17A5010013054539FC
:105C000097900100E78060D917B501001305C5E73B
:105C100025A08D47630CF40297B50100938585E9B3
:105C200017A501001305C53697900100E780E0D65F
:105C300017B50100130585DE97900100E780E0D5D8
:105C4000294597900100E78020DA49B7854717B5C5
:105C50000100130565DE17E7FF1F2307F744979040
:105C60000100E78060EBB7750200B76602000146ED
:105C7000054597D0FF1FE780C0B6930760F817E788
:105C8000FF1F2309F74A97E7FF1FA386074A9307D9
:105C9000002617E7FF1F2321F74AE577938707219F
:105CA00017E7FF1F231CF748B14597E7FF1F23881D
:105CB000074897E7FF1FA384A7484A85970000007D
:105CC000E780E01621B7914763E3870297B50100AB
:105CD000938545DE17A501001305852B97900100DC
:105CE000E780A0CB17B50100130505D7B1B797E43E
:105CF000FF1F83C4644497E7FF1F83C7D743A204F1
:105D0000DD8C83A7C9046D14228697E5FF1F938558
:105D1000B542280082978E0493160401B7750200DD
:105D2000C1823000A695094597D0FF1FE78060AB80
:105D3000930770F817E7FF1F230EF73E994597E783
:105D4000FF1FA38BA73E95BF914763E3870297B5DB
:105D50000100938525D617A50100130565239790AB
:105D60000100E78080C317B50100130565D0E9B5D0
:105D700097E4FF1F83C4443C97E7FF1F83C7B73BEB
:105D8000A204DD8C83A7C9046D14228697E5FF1F4A
:105D90009385953A280082978E0493160401B7756F
:105DA0000200C1823000A6950D4597D0FF1FE78005
:105DB00040A3930780F8BDBF17B50100130505CEBA
:105DC00097900100E78040D5930790F82304F100F5
:105DD000834719008D452800A304F100834729005B
:105DE0002305F10097000000E78060041305C0124E
:105DF00097C0FF1FE780E054014597D0FFFFE78081
:105E0000A0290D4597000000E78020D2294597C0C2
:105E1000FF1FE780005397C0FF1FE78060437DB3FB
:105E200097E7FF1F23A0A740828097E7FF1F938774
:105E3000673F03A3070063030300028317430000C7
:105E40006700E39241114AC09706002083D68691ED
:105E5000328917D6FF1F0356465822C426C206C6EB
:105E60002A84AE8497000000E780405D35C12DC0D4
:105E7000994763FF97048347140003470400A20770
:105E8000D98F13978700A183D98FC2073167C18348
:105E90001307C755639EE70297D7FF1F83D7E753C2
:105EA000A301F400A1832302F4009707002083D705
:105EB000678B91C7A302F400A1832303F400A68596
:105EC00017B50100130505C397900100E780E0AC0A
:105ED00097F7FF1F83C78775B9CF97D5FF1F83D566
:105EE000C54F17B501001305A5C297900100E780C3
:105EF000C0AA2686A28517D5FF1F0355054E970019
:105F00000000E78080BA6301090497E7FF1F83C799
:105F1000A7319DCB95C897E7FF1F83C7E7188DE78B
:105F200022852244B2400249A6859244410117438A
:105F300000006700C38317B50100130565BE979085
:105F40000100E78060BDC1B7B240224492440249DB
:105F500041018280834755008345450017B5010004
:105F6000130505B8A207DD8D179301006700E3A2B2
:105F700017B501001305C5B5179301006700C3B934
:105F80008D4763FBB70A011126CA06CE22CC034413
:105F9000350097E4FF1F83C4342997B5010093852A
:105FA000E5B8B337800017E7FF1FA30FF72609C432
:105FB00097B50100938545B817B50100130545B89D
:105FC00097900100E780609D97E7FF1F83C7D72563
:105FD0006386970097000000E780E02E97E7FF1F99
:105FE00083C797248DC785472306F100B7E70400D0
:105FF00083A747177000854513055030829717B562
:1060000001001305E5B497900100E780E0B09967BF
:10601000938757EE2316F100680085479145A30743
:1060200081002307F10097000000E78040E0F24084
:106030006244D244056182808280894763F7B70851
:10604000011122CC06CE26CA8344250085472A8426
:10605000639DF404914763F5B70403454500834706
:10606000340022055D8D97D7FF1F2398A736970030
:106070000000E78080459967938767EE2314F1005D
:106080008347340023059100A305F10083474400B2
:10609000954528002306F10097000000E78020D9ED
:1060A000F2406244D24405618280FDF8996793878B
:1060B00067EE2314F10097D7FF1F83D70732A3059C
:1060C000F10023050100A183E1B7828001119967E6
:1060D00022CCD51717F4FF1F130444552314F100E5
:1060E0008347040026CA97F4FF1F9384A4672305FF
:1060F000F10083D7040028009545A305F100A18392
:1061000006CE2306F10097000000E78040D203D6B8
:1061100004008345040017B501001305E5A497901A
:106120000100E7808087F2406244D24405618280AA
:106130009D677971D9172316F10097F7FF1F83C761
:10614000E74E06D62307F100A9C3B7E70400FC47D2
:10615000414697E5FF1F9385E5FB1305F100829704
:106160006800CD4597000000E78060CC97F5FF1FE1
:1061700083C5C54B17B50100130505A29790010013
:10618000E780A081B25045618280B7E70400BC4738
:10619000414681451305F1008297D9B745C54111A4
:1061A00006C622C4930750FA2300F5009307A00502
:1061B000A300F50089472301F5009147A301F500ED
:1061C0009307E002A302F50097F7FF1F93870746A6
:1061D00083C70700230205002A842303F50097E7FD
:1061E000FF1F9387770483C70700414697E5FF1F8A
:1061F000938545F2A303F50097F7FF1F83D78756D2
:106200002304F500A183A304F50097D7FF1F83D7CC
:10621000C71C2305F500A183A305F500B7E704001B
:10622000FC47310582972285F14597000000E78001
:10623000E01C230EA4002181A30EA400B24022443E
:106240004101828082805D710A8586C6A2C4970062
:106250000000E780E0F437E404007C448A850810FD
:10626000794682973C441305E103094681458297AC
:10627000101093050002014597D0FFFFE7806046AC
:10628000B640264461618280411122C426C24AC0C0
:106290002A84AE843289AA8585660146254506C6CC
:1062A00097C0FF1FE780E053A2852244B240CA8610
:1062B0002686024992442945410117C3FF1F670002
:1062C00043520111B7C7A55A22CC9387C73317E4AD
:1062D000FF1F130474F53EC4834704002C002146BD
:1062E000196506CE3EC697000000E78020FA834578
:1062F000040017B501001305259997800100E78078
:10630000C069F2406244056182800111A1463000FB
:1063100099652D4522CC06CE97C0FF1FE780604CC3
:10632000A24737C4A55A1304C43363958702B24504
:1063300017B5010013058588B335B00097E7FF1F37
:10634000A384B7EE97800100E7802065F2406244A5
:10635000056182809165A1463000938505F02D4549
:1063600097C0FF1FE780E047A247E38287FC85478D
:1063700017E7FF1FA30AF7EA854517B501001305C4
:106380002586C9B77971D146700091652D4522D413
:1063900006D697C0FF1FE780C044B24737C4A55A4E
:1063A0001304F43563988702B7E70400FC4717E548
:1063B000FF1F130525D641460C08829717B501002B
:1063C0001305058897800100E7800075B2502254BC
:1063D000456182809165D1467000938505E82D4521
:1063E00097C0FF1FE780E03FB247E38F87FA17B5FA
:1063F00001001305E586F9B7C16769768146FD1787
:1064000005061397060141836364B7003E858280C9
:106410003307D50003470700B98F214713F817004A
:10642000858363050800B18FC207C1837D17137789
:10643000F70F6DF78506F1B741C5A547054763F22C
:10644000B70883471500034705003168A207D98FB5
:1064500013978700A183D98FC207C1831308C8553A
:10646000054763900707411106C622C426C20344AC
:106470002500914763F087049307540063ECF5020D
:10648000A301C50021822302C5009304340091C6F4
:10649000A302D500A1822303D5002A84A6859700F4
:1064A0000000E780A0F526942300A4002181A3002A
:1064B000A4000147B240224492443A8541018280BF
:1064C00005473A8582800111B7C7A55A22CC938728
:1064D000E7342A842AC621462C00156506CE3EC420
:1064E00097000000E78080DAA28517A50100130558
:1064F000A57B97800100E780404A97000000E78075
:10650000C0D4F2406244056182800111A14630008E
:1065100095652D4522CC06CE97C0FF1FE780602CE5
:10652000A24737C4A55A1304E43463958702B245E1
:1065300017A501001305C56C97D7FF1F239FB7E868
:10654000C205C18197800100E7802045F240624486
:10655000056182809165A1463000938505EE2D4549
:1065600097C0FF1FE780E027A247E38287FCD1475F
:1065700017D7FF1F2313F7E6D14517A50100130511
:10658000256AC9B797A701009387077613D7C50077
:106590003E97034707001105230EE5FE13D785003C
:1065A0003D8B3E9703470700A30EE5FE13D745003A
:1065B0003D8BBD893E97AE970347070083C7070011
:1065C000230FE5FEA30FF5FE8280011122CC06CE3B
:1065D00026CA4AC84EC693F715002E84638E071646
:1065E000AD679387A7AA371700401CC397F7FF1F13
:1065F00083C7271499EF97F7FF1F83C7C71685072F
:1066000093F7F70F1D47636AF70217F7FF1F230C75
:10661000F714B7E70400BC4F13060019854517D5DA
:10662000FF1F034565DB829713451400F240624467
:10663000D2444249B2490561828097F7FF1F238403
:106640000712B75720419304D0039387777497F5C7
:10665000FF1F83D5251117F5FF1F1305F50D13092E
:10666000000217F7FF1F2327F70C97F7FF1F23855B
:10667000970C97000000E78020F12300250197F791
:10668000FF1F83C7A7FAB337F00093870703A3015F
:10669000F5009309000593072004A30035012301A9
:1066A000950023022501A302F5002303950097D549
:1066B000FF1F83D525D01D0597000000E780C0ECA3
:1066C00023002501A3003501930750042301F500A1
:1066D000A301950097D5FF1F83D585BE11059700AF
:1066E0000000E78060EA9307B0042300250123013E
:1066F0009500A300F50097E7FF1F83C7A7A1A20796
:1067000097E5FF1F83C515A1DD8D0D0597000000DE
:10671000E78080E797E7FF1F83C7E79FA20797E51A
:10672000FF1F83C5559FDD8D97000000E780C0E502
:10673000B5472300F500A947A300F5009305250000
:1067400017F5FF1F130505FF898DC205C18197202D
:106750000000E78060FC75BD93F7250081CB97F7BB
:10676000FF1F239707FC13C52500C9B593F7450004
:106770000145E38D07EA17A501001305A55497808D
:106780000100E780603997300000E780E02B134577
:10679000440069BD411122C437E404005C5C06C6B4
:1067A000354697A501009385E50317B5010013054C
:1067B00065D2829711E917A50100130565519780ED
:1067C0000100E780603501A08327041C82972A849A
:1067D000054597C00000E780A0E897600100E780CA
:1067E000C06D97600100E780C04297B00000E7806D
:1067F00020FA2285B24022444101828041110545A0
:1068000006C622C426C297C0FFFFE780C0721305E8
:10681000A00497C0FF1FE7808089757585457D15A9
:1068200097C0FFFFE780605C7D7585451305F536F1
:1068300097C0FFFFE780C065371400408327840AB4
:106840008D451305002093E707202324F40A97C001
:10685000FFFFE7808059B7E4040097D0FFFFE7808F
:10686000009DC85897800100E780002B17B50100F4
:10687000130545C697800100E780002A8327840C12
:106880008545414593E707082324F40C97C0FFFF93
:10689000E78000608D451305000897C0FFFFE78083
:1068A000205F97D0FFFFE780008C37A50700130516
:1068B000051297D0FFFFE780A0879D45014597D03F
:1068C000FFFFE780A08DB7E700E03707000423A0B3
:1068D000E7180100010097D0FFFFE780600F97D015
:1068E000FFFFE780602197000000E780E0EA970063
:1068F0000000E780C0A197000000E78040C197E05A
:10690000FFFFE78060FB97000000E780A02597006D
:106910000000E780801083A7040817050000130516
:1069200005CB829797D7FF1F2388A7AABC4C1306D5
:1069300000648545829797C0FF1FE78060AB0145E3
:106940008280AD67371700409387A7AA1CC3B7E7BB
:1069500000E03707400023A0E71801000100B7F767
:10696000070003C70701A5476316F7009397450182
:1069700091C301A04111AE860146AA85254506C6F0
:1069800097C0FF1FE780E0E5B240B7E700E03707B8
:10699000400023A0E710410182804111B2862E867B
:1069A000AA852D4506C697C0FF1FE78080E3B24049
:1069B0000145410182809307000463ECC7041D7107
:1069C000A2CC2A840808A6CACAC886CE32C6978036
:1069D0000100E78020F1AD67371700409387A7AA31
:1069E0001CC3B7E400E03709400023A024190100CC
:1069F0000100B2461008A285294597C0FF1FE78015
:106A000040DEF640664423A02411D6444649256161
:106A100082803955828041110D658D4506C697C02B
:106A2000FFFFE780803CB71700408D6623A6D70A9A
:106A300017F5FF1F130545D31387C70A9387870AE6
:106A40001CC15CC5856689675CC958C114C518C975
:106A5000B7E70400B24003A3871E410102838145CA
:106A6000B307B5008387070089E717230000670095
:106A700083C18505C205C181E5B797A7010093874A
:106A800067401357C5003E9703470700011106CE24
:106A90002304E100135785003D8B3E970347070011
:106AA00023060100A304E100135745003D8B3D89F7
:106AB0003E97AA970347070083C7070028002305CE
:106AC000E100A305F10097000000E78080F9F240A3
:106AD00005618280411126C2E97797F4FF1F9384F4
:106AE00024D922C49387A7552E842381B4002E86EF
:106AF000AA8517F5FF1F1305E5D706C62390F400F6
:106B0000A381040097800100E780C0DD9305240085
:106B1000C205C18117F5FF1F1305A5D59700000019
:106B2000E780C08DB38784002382A7002181A382E0
:106B3000A700930564002244B24026859244C20512
:106B4000C1814101172300006700E3B309C993071E
:106B5000800263E6B700170300006700E3F7828056
:106B600097F7FF1F83C7A7D399EF411106C6972058
:106B70000000E78020A9B240854717F7FF1F2300D8
:106B8000F7D24101828082806301054A638F054804
:106B90005D71CAC04EDE86C6A2C4A6C252DC56DAF9
:106BA0005AD85ED662D466D26AD0B9472A89AE89ED
:106BB00063F9B706394697A501009385651A978052
:106BC0000100E780C0CF31ED8347E90013071003D0
:106BD0006394E702854717F7FF1F2309F7C817A536
:106BE00001001305E51897F7FF1F239007C89700CA
:106BF0000000E78000E771A01307000317A501005C
:106C00001305051AE395E7FE97F7FF1F238007C6D4
:106C100097F7FF1F239B07C417A501001305C5168F
:106C2000F9B797F7FF1F83C767C463870722BD6A59
:106C3000B96B938CFA55014A17FBFF1F130B8BB4EA
:106C4000138CEB65938AFA6605A8B307490183C6DE
:106C5000070097F7FF1F83D747C1B1E39307A0054C
:106C6000639BF600854717F7FF1F2310F7C097F7C0
:106C7000FF1F2389D7B0050A93170A01C183E3E6F2
:106C800037FDB640264496440649F259625AD25A14
:106C9000425BB25B225C925C025D61618280054D69
:106CA000639BA7039307500A639EF600894717F773
:106CB000FF1F231CF7BA930750FA17F7FF1FA30310
:106CC000F7AC55BF9307A005E387F6FA97F7FF1FC8
:106CD000239D07B84DB7138717004207DA97418302
:106CE0002380D70017F6FF1F2311E6B88D47E3F482
:106CF000E7F817F4FF1F034414A997F7FF1F83C792
:106D000087A822045D8C9307F4FFC207C183930612
:106D1000F00DE3EDF6FA93076400C207C183E31CAC
:106D2000F7F493052400C205C18117F5FF1F130571
:106D300085A597F0FFFFE780606C33078B008347E2
:106D4000570003474700A207D98F17F7FF1F231EDD
:106D500007B06318F50E8144630CA40197F4FF1F7C
:106D600083C484A2A20497F7FF1F83C7F7A1DD8C19
:106D7000170500001305C5DD97F0FFFFE780800AC7
:106D800063878407636D9C029387EB556382F404E9
:106D900097F7FF1F83C7479F05476389E70681CBA6
:106DA0001387A7051377F70F8D4663F2E6081307DD
:106DB000F0072300E100A300F10089459DA0638254
:106DC0009405E39754FD97F0FFFFE780A03611A8E4
:106DD000A28517F5FF1F1305259B97F0FFFFE7809E
:106DE000601A014597F0FFFFE780C00369B5A285EF
:106DF00017F5FF1F1305459997F0FFFFE780202443
:106E0000CDB797F0FFFFE780A02CE1BF930710F804
:106E1000130511002300F10097F0FFFFE7804038D1
:106E2000FD450A8597000000E78000CB5DBFA28585
:106E300017F5FF1F1305459597F0FFFFE78020D555
:106E40004DB79307F00789450A852310F100970095
:106E50000000E78060C805B5BD4763F837174146B5
:106E600097A50100938505F64A8597800100E78084
:106E700000A5631C051417A501001305E5F597008F
:106E80000000E78000BE17F5FF1F0355A58D970092
:106E90000000E780C0BE97E7FF1F83C7277917A5CB
:106EA00001001305E5EA89E717A501001305C5EA06
:106EB00097000000E780E0BA17A50100130545F32D
:106EC00097000000E780E0B917C5FF1F0355854E06
:106ED00097000000E780A0BA17A50100130585F10F
:106EE00097000000E780E0B717C5FF1F0355E54E88
:106EF00097000000E780A0B817A50100130505F072
:106F000097000000E780E0B517D5FF1F0355251A4D
:106F100097000000E780A0B617A50100130585EED5
:106F200097000000E780E0B317D5FF1F0355E51772
:106F300097000000E780A0B417A50100130505ED38
:106F400097000000E780E0B117D5FF1F0355051635
:106F500097000000E780A0B217A50100130545EBDC
:106F600097000000E780E0AF17C5FF1F03554535C8
:106F700097000000E780A0B017A501001305C5E940
:106F800097000000E780E0AD97D7FF1F83C7871801
:106F9000A20717D5FF1F0345F5175D8D9700000069
:106FA000E780E0AD97D7FF1F83C7E716A20717D585
:106FB000FF1F034555165D8D97000000E78020AC4C
:106FC00017950100130585591DB1C147E3FB37CB68
:106FD000414697A50100938565E44A8597800100A5
:106FE000E780E08DE31F05C88347090113071003FD
:106FF000639CE700854717E7FF1F2303F77817A572
:1070000001001305E5E2E5B61307000317A501002B
:10701000130505E5E39DE7BC97E7FF1F238207768D
:1070200017A50100130545E2D9B68280411126C299
:10703000AE848D4522C406C62A8497C0FFFFE78030
:1070400020E5B717004099C803A5C70C418D23A6BA
:10705000A70CB240224492444101828003A5870CD0
:10706000418D23A4A70CF5B78347050003471500FE
:10707000A207D98FC2076177C18713072720639AB8
:10708000E70083452500370504001703000067006B
:1070900023FA828017F6FF1F1306C6808147B28647
:1070A0001303F00FA9483308F6000348080013F74C
:1070B000F70F6307A80C630668008507E39517FFC1
:1070C0002947B387E6002380A70097E7FF1F938730
:1070D000277E5DA8411113D765001347170006C628
:1070E00093F63500058B954791CA05469947638706
:1070F000C60009469D476383C600A14713F64500B5
:107100003336C00093F68503050685C2A145638B1F
:10711000B604E145638AB604930580026388B60429
:10712000930580036393B600914697F5FF1F23866E
:10713000F59E97F5FF1F2381C59E97F5FF1FA38D31
:10714000D59CBE8517A501001305C5D79780010002
:10715000E780A084B240854717F7FF1FA30FF79A77
:10716000410182808546D1B78946C1B78D4675BF3A
:1071700017A50100130585D7178301006700E38178
:1071800017E7FF1F1307C772BA972380B700E147BD
:10719000E302F5F493077002E30CF5FC82802A8782
:1071A00023800500814717E5FF1F1305A56F13080E
:1071B000F00F2946B306F50083C606006396E60283
:1071C00097E6FF1F9386C66EB69783C707000545EF
:1071D0002380F5009947636EF7029D4763FDE70042
:1071E000E147630DF7008280638506018507E3931D
:1071F000C7FC0145C5B7238005008280B737004032
:1072000003C7370083C7050093F70704D98F23808E
:10721000F50082805D7152DC56DA5ED6716A97FBAA
:10722000FF1F938BABA08D6AA6C24EDE62D486C6CA
:10723000A2C4CAC05AD866D26AD06ECEC1495E8C8A
:1072400097E4FF1F93848467130A0A20938A7ADCE9
:1072500017F9FF1F034989A0B3872B0183C70700D4
:1072600093F7F70FC9EFB787004003C76700058B97
:10727000E310077C03C76700118BE30D077E83C70C
:107280005700918B99E36F10200317F7FF1F0347F7
:10729000079D85476304F7006F10400197F7FF1FB4
:1072A000A38DE78697E7FF1F238A076C97E7FF1FE9
:1072B0002388077897F7FF1F2386078497F7FF1F18
:1072C0002383078497E7FF1FA38A076A97E7FF1FB7
:1072D000A388077697F7FF1FA386078297F7FF1FFC
:1072E000A383078297F7FF1FA38A078297F7FF1FE1
:1072F000A3870796B787004011476F007077930701
:10730000190093F7F70F3D476364F70617F7FF1F60
:107310002306F79497F7FF1F93874793CA9783C76E
:1073200007001307100293F7F703638EE71E6366E7
:10733000F70405446385871CE38C07620947638E65
:10734000E71013070002E384E74EB7E700E03707D2
:10735000400023A0E7180100010062992300090002
:10736000FD1923A0E71093F9F90FE39309EEE5BDAA
:1073700097F7FF1F2384078E71BF130730026388BE
:10738000E70C63E8E71613074002638CE70A13076C
:107390000003E39CE7FA97F7FF1F9387278ACA97B2
:1073A00003C70700A1471377F70FE31BF71483C741
:1073B000640097E6FF1F2389F67497E7FF1F83C7D2
:1073C000575091C7FD5797E6FF1F238FF67297E539
:1073D000FF1F83C5B54E97E7FF1FA387B77297E7D7
:1073E000FF1F83C7A74D13FB07089306000493F7FD
:1073F0000706639FD74C9307A009638DF51663EAD0
:10740000B7129307F0056386F54A93075009638422
:10741000F52A014497E7FF1F83C7176F1547E392CB
:10742000E736B7E700E03707400023A0E718010080
:107430000100B786004023808602130680FC6F009F
:10744000500EFD5717E7FF1F230FF76AFDBDFD57CD
:1074500017E7FF1F2308F76ACDBD17A50100130525
:1074600065BA97700100E780206B97E7FF1F93874D
:10747000E77CCA9703C40700014B97ECFF1F938C6E
:107480006C5C1374F40F17AD0100130D2DB8634736
:107490008B04294597700100E7800055854717E761
:1074A000FF1FA30FF75817E7FF1F230C875817E795
:1074B000FF1F2305F76637E700E0B70640002320EB
:1074C000D71801000100378600408347A60293F7D2
:1074D000370F2305F6022320D71085BDB3876C0133
:1074E00083C507006A85050B97700100E780E04AB5
:1074F00079BF854717E7FF1F2304F754B9B517E78E
:10750000FF1F1307A7734A970347070097E6FF1F5C
:10751000A386F64697E6FF1F2383E64617E7FF1F7D
:10752000230EF75E1DB5854717E7FF1F2308F744B5
:1075300029BD9307400A6389F5349307200B6384C0
:10754000F5369307100AE396F5EC8387240001448F
:10755000E3D207EC97E7FF1F83C7773693F6370030
:10756000638A061A0546638AC62209466395C61AC7
:107570001D4755A217E5FF1F03456534C94797EC22
:10758000FF1F83CCDC3397E5FF1F83C5653317E40A
:10759000FF1F0344F4326315F510CD476392FC10CE
:1075A00093077008639CF5021307300FB7170E009E
:1075B0006308E4001307900DB7B704006314E408F0
:1075C00017E7FF1F2328F754BE8517A501001305F1
:1075D00065A497700100E780403C25BD93078008B3
:1075E000639DF500B307804013F4F70FB7774600AB
:1075F000938787CDB3D78702E1B793079008639A43
:10760000F500B307804013F4F70F91679387C766BF
:10761000D5B79307A008639BF500B307804013F428
:10762000F70FB7173D0093870790E9B79307B008A6
:10763000639AF500B307804013F4F70F91679387BF
:1076400097D04DBF93F5F5078D47639BF500B307C2
:10765000804013F4F70FB7975B00938707D859BFA3
:107660008947639BF500B307804013F4F70FB777A2
:107670000B009387071BBDBF8547639AF500B307CF
:10768000804013F4F70FDD67938767E3A5B7D287D0
:1076900085F9B307804093F7F70FB3D7FA020DB718
:1076A00097000000E780409FA28566859700000054
:1076B000E780809EB9BB9305610017E5FF1F034576
:1076C000052017E4FF1F0344941F97000000E78084
:1076D00040AD93057100228597000000E78060AC03
:1076E0003C0017E7FF1F2321F75483476100230461
:1076F000F10083477100A304F100894717E7FF1FDA
:107700002304F7408357810017E7FF1F2318F71A58
:10771000094409B3154793F64700B336D00093F7F1
:107720008703850685C32146638BC7066146638A46
:10773000C706130680026388C70613068003639397
:10774000C700914717E6FF1F2308D63C97E6FF1FA7
:10775000A384F63C97E7FF1F2381E73C17E7FF1F51
:10776000034707169376070497E7FF1F83C757154C
:107770008DEE1377770C93067008630CD70213779E
:10778000F7078D466312D70CB307F040B7955B003F
:1077900093F7F70F938505D849A81947ADBF8547DB
:1077A00055B7894745B78D4771BF93067008631178
:1077B000D7021307300FB7150E006389E7021307CE
:1077C000900DB7B504006383E7021307700845BF47
:1077D0009306800C6311D702B307F040B7754600DB
:1077E00013F7F70F938785CDB3D5E70297E7FF1F10
:1077F00023A2B732D9BB9306900C631CD700B30702
:10780000F04093F5F70F91679387C766B3D5B7023A
:10781000F1BF9306A00C631DD700B307F040B71566
:107820003D0093F7F70F93850590B3D5F5027DBF23
:107830009306B00CE315D7F4B307F04093F5F70FB8
:107840009167938797D0D9B78946631BD700B30751
:10785000F040B7750B0093F7F70F9385051BF1B751
:107860008546631AD700B307F040DD6593F7F70F3D
:10787000938565E35DBFD28535FBB305F04093F595
:10788000F50FB3D5BA029DB783C72400C18B99C742
:10789000854717E7FF1F230CF726A5BE97E7FF1FB5
:1078A00023870726BDB6854717E7FF1FA307F726DF
:1078B0008DB63C0017E7FF1F2328F73609479307CB
:1078C00000032314F10097E6FF1F238FE6222DBD4E
:1078D00063940756A94763E5B7421797010013075A
:1078E000A75B8A05BA959C41BA97828717E4FF1F68
:1078F0000344F4FC894C6306940D63E68C068547CB
:107900006303F4089307F00F17E7FF1F0347C71F30
:1079100063F6E70017E7FF1F2308F71E97ECFF1F2A
:1079200083CC8C1E9307000413F4FC0F63F49701BF
:107930001304000497E7FF1F9387072F03AD070089
:1079400022862685EA85B38C8C40229D97700100A3
:10795000E78040F997E7FF1F2388971B97E7FF1FF2
:1079600023A4A72D45BC8D47630CF40A9947E31B5C
:10797000F4F8979701009387A75817E7FF1F23256F
:10798000F72AA94751B717E7FF1F0347472D97E786
:10799000FF1F938767194946979501009385455FB7
:1079A00063068700979501009385855A3E859770F9
:1079B0000100E78020F317E7FF1F2327A726C94709
:1079C000A1B797E6FF1F83C68629054797E7FF1FE4
:1079D000938787156394E6023E8513067002979598
:1079E00001009385655897700100E780A0EF17E7C5
:1079F000FF1F232BA7229307700239B73E8513067A
:107A00003004979501009385655097700100E780D9
:107A100060ED17E7FF1F2329A72093073004EDB57A
:107A200097E5FF1F83C5A5E9179501001305C55FFD
:107A300097700100E78060F6054D97EDFF1F83CD3D
:107A40000D2297E5FF1F83C585E7179501001305F4
:107A5000A55D6398AD0B97700100E78000F497E790
:107A6000FF1F83C7C7E5B5CBE36EF4E817940100A9
:107A700013044456638CB701179401001304045691
:107A800063869701179401001304C45622859770EA
:107A90000100E780A0091375F50F9307150086070D
:107AA00017E7FF1F2302F7088D4717E7FF1FA30DF6
:107AB000F70697E7FF1F938727070147BE861376D0
:107AC000F70F89076365A60297E7FF1F23AED71458
:107AD00097E7FF1F83C7470505BD97970100938769
:107AE000674817E7FF1F2321F714914731BD33067D
:107AF000E40003460600A380070005072380C700B3
:107B00007DBF97700100E78040E997E7FF1F83C7BB
:107B100007DBE1D7E368F4DE17940100130484481F
:107B2000638CA701179401001304444863869701EE
:107B30001794010013040449228597700100E7801F
:107B4000E0FE1375F50F93071500860717E7FF1F73
:107B5000230CF7FC8D4717E7FF1FA307F7FC97E7F8
:107B6000FF1F938767FC0147BE861376F70F8907CF
:107B7000E37CA6F43306E40003460600A380070076
:107B800005072380C700D5B797E5FF1F83C525D319
:107B9000179501001305054A97700100E780E0DFA3
:107BA00097E7FF1F83C717F893E7470017E7FF1F03
:107BB000A30AF7F683C7240017E7FF1FA302F7F60F
:107BC00089B8179501001305254897700100E780D3
:107BD000A0F497E7FF1F9387A7F483C7070017E771
:107BE000FF1F230DF7CC17E4FF1F0344E4F13334E8
:107BF00080000DB0179501001305454697700100F0
:107C0000E78080F197E7FF1F83C7D7F193E707016C
:107C100017E7FF1FA308F7F083C7240017E7FF1F2C
:107C20002300F7F06FF0EFFE1795010013054544B0
:107C300097700100E78040EE03C704007D8B51EF91
:107C4000B787004003C767021377C70B1367270086
:107C50002383E70203C7A7021377C70B1367270025
:107C60002385E70203C7E7021377C70B13672700D3
:107C70002387E70203C727031377C70B1367270080
:107C80002389E702854717E7FF1F2309F7CE17E788
:107C9000FF1F2307F7DA17E7FF1F2305F7E617E7AC
:107CA000FF1F2302F7E697E7FF1FA38907CC97E79B
:107CB000FF1FA38707D897E7FF1FA38507E497E770
:107CC000FF1FA38207E497E7FF1FA38907E497E755
:107CD000FF1FA38607F86FF0CFF389476312F702FF
:107CE00097E7FF1F83C7C7BD9146638CD70863E042
:107CF000F604638EE70C6369F70A05476380E70EB5
:107D0000FD5717E7FF1FA301F7E037074000B7E76C
:107D100000E023A0E71801000100B7860040130629
:107D2000F0FC2381C60223A0E7106FF00FE21307D7
:107D300020086382E7086362F70213071008E391E3
:107D4000E7FC378700408347670293F7C70B93E749
:107D500027002303F7026FF0CFEB13073008638986
:107D6000E70213074008E39DE7F8378700408347A1
:107D7000270393F7C70B93E727002309F7026FF058
:107D80004FE9378700408347270393F73707F5B755
:107D9000378700408347E70293F7C70B93E7270035
:107DA0002307F7026FF0EFE6378700408347E702CB
:107DB00093F73707F5B7378700408347A70293F754
:107DC000C70B93E727002305F7026FF08FE437878F
:107DD00000408347A70293F73707F5B7378700407E
:107DE0008347670293F73707ADB71795010013056F
:107DF000252997700100E78020D297E7FF1F238F86
:107E000007AAD5B3179501001305852897700100BF
:107E1000E78080D097E7FF1F239207AA97E7FF1F0D
:107E2000938787CE03C40700894763F3870009441B
:107E30001374F40F6FF00FDE13070002E392E7EC08
:107E4000631B0B0A638FF500930720026383F50819
:107E5000179501001305452797700100E780E0B3EF
:107E600045B5179501001305652397700100E7805C
:107E7000A0CA0144179D0100130D8D23A14CB387A7
:107E8000840083C507006A85050497700100E780B8
:107E9000C0B0E31694FF1785010013052572977093
:107EA0000100E78060C717E4FF1F034464A101E8F5
:107EB00097E7FF1F2386079E014B6FF0AFD58947D9
:107EC000E310F4E4854717E7FF1F230BF79C6FF0DF
:107ED0004FD417E6FF1F0346969E97E5FF1F83C505
:107EE000059E179501001305251D97700100E78079
:107EF000C0AA6FF00FD26380F50693071002E399D2
:107F0000F5F497E5FF1F83C5A59B179501001305A1
:107F1000A51C97700100E78040A897E7FF1F23A5E5
:107F200097D097E7FF1F9387E7BE944383D7470017
:107F300017E7FF1F034767BE17E6FF1F2320D698EA
:107F40001D4497E6FF1F239DF69697E7FF1F238AA0
:107F5000E7966FF02FCC97E5FF1F83C565961795C1
:107F600001001305E51897700100E78000A397E76B
:107F7000FF1F2387079297E7FF1F239107946FF056
:107F80002FF92547638FE7C89946378700406394E8
:107F9000D70223008702B7E700E0B706400023A01E
:107FA000D71801000100130600FC2301C70223A01B
:107FB000D7106FF08FB99306100A639FD700230084
:107FC0008702B7E700E0B706400023A0D7180100FA
:107FD0000100130680FCD1BF9306A009E381D7FE00
:107FE0009306400AE38DD7FC93062002639DD700D9
:107FF000B7E700E0B706400023A0D7180100010052
:1080000023008702F9B78546E384D7FE930700086B
:10801000E300FBFEB7E700E0B706400023A0D71857
:1080200001000100130620FC23008702BDBF17E7F3
:10803000FF1F034777AD6302F71E63E7E70295472B
:108040006300F7109947630AF704B786004023805E
:108050000602B7E700E03707400023A0E718010059
:1080600001001306A0FC75B99307F005630AF70039
:10807000930750096306F70093071002E317F7FC14
:10808000B7E700E03707400023A0E7180100010030
:10809000B7860040130620FC69B117EBFF1F034BA6
:1080A000ABA6930700045A8D63F46701130D000417
:1080B00097E7FF1F938747B783AC07001374FD0F43
:1080C0002286E685268597700100E780A081B307A8
:1080D0008B40669417E7FF1F2308F7A297E7FF1F5F
:1080E00023A487B4B7870040630C0B022380A70347
:1080F000B7E600E03706400023A0C61801000100E3
:1081000003C72702134707042381E70203C7270297
:108110001377C70F2381E70223A0C6106FF0EFA2E9
:108120002380070237E700E0B70640002320D71876
:1081300001000100130620FC2381C7026FF0AFB9D4
:10814000378700408347370097E6FF1F83C6569D59
:1081500093F70708D58FA301F700B7064000B7E7EC
:1081600000E023A0D718010001001306A0FC35BDD4
:1081700097E7FF1F938787ACCA9783C7070093F7DA
:10818000F70FC1CF97E7FF1F83C767ADD9E717E7A1
:10819000FF1F03477797930700026310F70883AD2B
:1081A000040017DDFF1F034DAD7197DCFF1F83CC6B
:1081B0003C7117DBFF1F034BCB70E6876A87DA86BB
:1081C0006E8697D5FF1F83C5A56D17950100130512
:1081D000A5F397600100E780407C97E7FF1F23AB82
:1081E000B79397E7FF1F2389A79397E7FF1FA385FF
:1081F000979397E7FF1F2382679397D7FF1FA3806B
:10820000876AB7E700E03707400023A0E7180100BE
:108210000100B78600406FF04FA2B7E700E03707D4
:10822000400023A0E71801000100B786004015BDFB
:1082300097E6FF1F83C6A6A20547639CE60429476D
:108240002381E70209472383E7022385E70297E7B3
:10825000FF1FA385078C97E7FF1FA38207A0B7879F
:108260000040A381070017E7FF1FA30B078A0547FC
:108270002383E700B640264496440649F259625AE1
:10828000D25A425BB25B225C925C025DF24D61614C
:10829000828029472381E70209472383E702238558
:1082A000E7022387E7022389E70255B717D7FF1FA5
:1082B000A307F75E6FE01FFF854717D7FF1F230F48
:1082C000F76A17D7FF1F230DF77617E7FF1F230B5A
:1082D000F78217E7FF1F2308F7826FE0BFFE85478D
:1082E00017D7FF1F230CF76817D7FF1F230AF77450
:1082F00017E7FF1F2308F78017E7FF1F2305F78005
:1083000017D7FF1FA30C076617D7FF1FA30A077213
:1083100017D7FF1FA308077E97D7FF1FA385077EE8
:108320008280411106C697000000E78080FBB78776
:10833000004023800700130740FC2386E700130753
:10834000C004A386E70017D7FF1F130727572398FA
:10835000E70017D7FF1F1307675A239AE70017D7BD
:10836000FF1F1307E765239CE70017D7FF1F1307BD
:108370006771239EE70029472381E702094723838A
:10838000E7022385E7022387E7022389E702A38127
:108390000700930600F8A380D7009306900223807D
:1083A000D700FD562383D7002381E70093060005FD
:1083B00037E700E0230BD740B70640002320D71053
:1083C00003C7170013671700A380E700B24097D7D1
:1083D000FF1F2397077441018280411106C6970051
:1083E0000000E78000F0B7870040238007001307F4
:1083F00000FC2386E7003147A386E70017D7FF1F5D
:108400001307C74B2398E70017D7FF1F1307074F22
:10841000239AE70017D7FF1F1307875A239CE7000B
:1084200029472381E70209472383E7022385E702DF
:10843000A3810700930600F8A380D700930690025B
:108440002380D700FD562383D7002381E7009306BE
:10845000000537E700E0230BD740B7064000232094
:10846000D71003C7170013671700A380E700B240B7
:1084700097D7FF1F2396076A41018280F167938790
:10848000072017D7FF1F2327F768854717D7FF1F38
:108490002314F768A14717D7FF1F2300F76897D762
:1084A000FF1FA38C076697D7FF1F2389076697D7FF
:1084B000FF1F2387073E97D7FF1FA382073E8147F1
:1084C00017D5FF1F1305053EFD5517D6FF1F1306D1
:1084D000263E2947B306F5002380B600B306F60012
:1084E000238006008507E397E7FE97D7FF1FA38E3B
:1084F000076097D7FF1FA38C076097D7FF1F2387BD
:10850000076097D7FF1F2382076097D7FF1F23813C
:10851000076097D7FF1FA38B075E97D7FF1F23889E
:10852000075E814717D6FF1F130646704147B30603
:10853000F600238006008507E39BE7FE828017D7BD
:10854000FF1F0347C77185476316F7001703000035
:108550006700E3E8170300006700E3DC411122C471
:1085600006C617D7FF1F0347876F85472E8613F46C
:10857000F50FAA856317F70417D5FF1F13054548A4
:1085800097600100E780003697D7FF1F238A074ACC
:10859000B787004023848702B7E600E03706400033
:1085A00023A0C6180100010003C7A7021377C70F55
:1085B0002385E702B240224423A0C61001454101B1
:1085C000828017D5FF1F1305653797600100E7808C
:1085D000603197D7FF1F2383073AB7870040238274
:1085E0008702B7E600E03706400023A0C618010066
:1085F000010003C767021377C70F2383E7025DBF3C
:10860000411106C697000000E78080E7B2404101B3
:10861000170300006700E3F2411106C697F0FFFF61
:10862000E78080BF97D7FF1F83C75735A1CB97D56A
:10863000FF1F83C5C53489C917D5FF1F13054534EE
:1086400097E0FFFFE780805497D7FF1FA38807328A
:1086500097D7FF1F2384074C37E700E0B706400099
:108660002320D718010001003786004083476602A7
:1086700093F7370F2303F6022320D710B2404101AE
:10868000828041C9D9C597D7FF1F83C76749D1C326
:10869000011122CC4AC84EC656C25AC006CE26CABE
:1086A00052C42E89AA890144930A0004371B03008F
:1086B00063772403B3078940C207C183BE8463F490
:1086C000FA0093040004C204C180130A1BD497D794
:1086D000FF1F83C7A72A9DE37D1A631C0A00F2408F
:1086E0006244D2444249B249224A924A024B05614D
:1086F000828097F0FFFFE78020B2D1BF33858900E9
:108700002694A685420497000000E78060E541803A
:1087100045B78280411106C622C429C12E8495C95D
:1087200097D7FF1F83C7C73F95CB97D7FF1F83C737
:10873000E7248DC713070004AE876374B70093075F
:108740000004139407014180A28597000000E78090
:1087500020E12285B2402244410182800144D5BFFC
:1087600097D7FF1F9387475318429C4383D64500F2
:108770000345070083C5C700035646006396A5005E
:1087800083D5E700638DD502011106CE2386A700AD
:108790002397D700B705CF00DC4B9385757D050780
:1087A0007D162EC2230001003AC42316C1002317F0
:1087B000D10099C30A858297F24005618280828048
:1087C000DC4DDC4B81CFB7E70400904503A3870560
:1087D000914517D5FF1F0345654C028382806D715B
:1087E0003C083EC6B707E500232291103EC8AA8484
:1087F0003C083285232611103ECA232481102320F1
:1088000021112E8997300000E78080632A84979594
:1088100001009385E5921775010013056577976050
:108820000100E7808017A285179501001305C5A1F7
:1088300097600100E7806016294597600100E78096
:10884000A01AB705CB009385757D680097100000CE
:10885000E7800069A285680097300000E780A0509B
:10886000014781467000CA85268597200000E78071
:10887000808C05CD2A84979501009385658C1775AA
:1088800001001305E57097600100E7800011A285E3
:10889000179501001305059C97600100E780E00F24
:1088A000294597600100E78020148320C11003242C
:1088B000811083244110032901105161828097D7D0
:1088C000FF1F9387673D18429C43797122D406D6D7
:1088D0000348070083C807012A8483D6450003554F
:1088E00046006396080183D82701638DD802238848
:1088F000070105072399D7003708CC00DC4B130884
:10890000787D3ACC1307F5FF42CA23080100231EE5
:10891000E100231FD10099C7080832C62EC48297F0
:108920003246A245228597000000E78080EBB250D6
:108930002254456182806D713C083EC0B707E50056
:108940003EC23C083EC4232611102324811023225A
:108950009110231701002318010023190100231A85
:108960000100231B010097B7FF1F83D767A999E375
:10897000C167FD172316F10097B7FF1F83D767A8BC
:1089800091EB97D7FF1F938727319C439C43DC478C
:1089900083D7070017B4FF1F130484A6584C23176E
:1089A000F10083574400484B2318F10031E19785CB
:1089B00001009385E57F177501001305655D9760DC
:1089C0000100E78080FD178501001305A57F9760F2
:1089D0000100E78080FC294597600100E780C00026
:1089E0008320C110032481108324411051618280AF
:1089F00097B7FF1F83C737A189EBB7E70400BC57C0
:108A000082975C4C23AA0700E1BFFD1797B6FF1FB2
:108A1000A38BF69E03560701834704014C470A8542
:108A2000230BF10097300000E780003197D7FF1F3C
:108A3000938787269C430147814688430A866C00BA
:108A400097100000E780206FAA8429C19785010054
:108A5000938505761775010013058553976001000E
:108A6000E780A0F3A685178501001305657697605A
:108A70000100E78080F2294597600100E780C0F699
:108A8000584CB7E70400BC57484B9DBF97B7FF1F32
:108A900083C77797F5D7B7E70400BC4F10448545E7
:108AA00017D5FF1F0345851F82971DBF5C4EDC4B0A
:108AB000B9CFB1CD411122C4177501001305454D41
:108AC0002E84978501009385E56C06C697600100AA
:108AD000E780A0ECA2851785010013052572976039
:108AE0000100E78080EB294597600100E780C0EF37
:108AF000B7E704002244B24003A3870517D5FF1F40
:108B00000345C51913064006914541010283828041
:108B1000411122C417B4FF1F1304448C1C4C06C619
:108B200089C7DC4399C34C488297584CB7E7040087
:108B3000BC57484B82975C4CB240224423AA0700A2
:108B40004101828017B7FF1F1307478B8347070038
:108B50009306F00B850793F7F70F63E9F60097B6D6
:108B6000FF1F238DF688034507008280930700F8D6
:108B7000FDB7835745006386071001114AC817B92E
:108B8000FF1F1309E98752C4032AC90106CE22CC6C
:108B900003274A0126CA4EC656C2F15735E31307CA
:108BA000D00DFD57636EC704B7E9040083A709071A
:108BB0002A841305860042054181B284AE8A8297D9
:108BC000232AAA000325C9015C49A9E7978501006A
:108BD0009385455A177501001305853B9760010081
:108BE000E780A0DB17850100130585699760010008
:108BF000E780A0DA294597600100E780E0DEDD57D5
:108C0000F2406244D2444249B249224A924A3E85E5
:108C10000561828093874400B705CF002319F500D2
:108C20009385757D310597100000E780602B032543
:108C3000C90183456400310597300000E780A01228
:108C40000325C9012686D685310597300000E780C7
:108C5000A00E7146A2854A8597600100E78080C812
:108C6000504419CA83A78905854517D5FF1F0345B9
:108C7000E5028297814769B797000000E780E0CB63
:108C8000D5BFFD573E858280411126C297A4FF1FA4
:108C900093840477D84C22C437E404003C54484BF6
:108CA00006C68297DC4C0323C4052244B24092449A
:108CB00023AA070017D5FF1F034545FE854541013F
:108CC0000283411126C297D4FF1F9384E4FC9C4089
:108CD00006C622C44AC0D5C3DC43C5C35CC1230059
:108CE000B5002A8497850100938505441775010016
:108CF0001305052A97600100E78020CA294597607F
:108D00000100E78060CE9C4023A4070023A2070057
:108D100097A7FF1F9387876CDC4FDC4B91C72955C2
:108D200097000000E78000DF97A7FF1F9387476D3C
:108D3000DC4FDC4B89C797000000E78020F537E95E
:108D400004008327C905894517D5FF1F034505F58D
:108D500082978327C905914517D5FF1F034505F461
:108D600082979C4003A347016309030022852244A4
:108D7000B2409244024941010283B24022449244EB
:108D80000249410182800111328506CE22CC26CAD9
:108D90002E8497300000E780A00AAA8497850100FE
:108DA0009385C53B177501001305851E976001006B
:108DB000E780A0BE03078400035664008355440087
:108DC000A686178501001305654597600100E780B9
:108DD000C0BC294597600100E78000C197A7FF1F2D
:108DE00083C72760639D9700014597000000E780D7
:108DF00060D281450A8597000000E780C0ECF24010
:108E00006244D244056182806D712324811023263F
:108E100011102322911093F745002E8463870714C5
:108E20003C083EC0B707E5003EC23C083EC42317DD
:108E300001002318010023190100231A0100231B3C
:108E4000010097A7FF1F83D7675999E3C167FD17F3
:108E50002316F10097A7FF1F83D7675891EB97D789
:108E6000FF1F938767E39C439C43DC4783D707003E
:108E700017A7FF1F130787562317F100544F835777
:108E800047002318F100DC4AA1E79785010093858C
:108E90002531177501001305A50F97600100E780C4
:108EA000C0AF178501001305E53197600100E78029
:108EB000C0AE294597600100E78000B31345440028
:108EC0008320C110032481108324411051618280CA
:108ED00097A7FF1F83C7F7502555D9C3FD1717A6BE
:108EE000FF1FA300F65003D6060183470701CC46B7
:108EF0000A85230BF10097300000E780E0E397D765
:108F0000FF1F938767D99C4317A7FF1F1307074DC0
:108F1000978601009386062E88430A866C00971078
:108F20000000E7804021AA8451D9978501009385EC
:108F30002527177501001305A50597600100E78037
:108F4000C0A5A68517850100130585289760010037
:108F5000E780A0A4294597600100E780E0A8268566
:108F600097000000E78000BB91BF93F725009DC7E5
:108F7000B7E70400BC47414681452808829725553C
:108F800097000000E78000B928089305F00F9700CC
:108F90000000E78040D3134524001DB793F7150068
:108FA000014599DF97000000E780209913451400E0
:108FB00001BF5C4D411106C688C317D7FF1F232D83
:108FC000F7CCB7E7040083A70708170500001305CF
:108FD000E5E38297B24097D7FF1F2381A7CC0145D5
:108FE0004101828001113335A000A307A100B7E73A
:108FF000040083A7471706CE1306F1008545130525
:1090000050308297F240056182808280411122C4F3
:1090100006C697D7FF1F83C7E7C9014489EF97B7F3
:10902000FF1F83C77720054499E717B4FF1F034448
:10903000A41F13441400228597000000E780C0FAA3
:10904000178501001305C52E09E4178501001305D6
:10905000252F2244B2404101176301006700E393CA
:10906000797122D4A30F010037E404008327841709
:1090700026D24AD006D6AA842E89130550309305ED
:10908000F10132C6829732468347F10193150601FA
:10909000C18185CB01452EC697000000E780C0F452
:1090A00083274417B2454A8626858297054597004F
:1090B0000000E78060F3B250225492540259456197
:1090C0008280832744174A8626858297EDB741110F
:1090D0009397050122C406C626C2C1872E8463D495
:1090E0000702B7E40400FC5417A5FF1F03454534ED
:1090F000829719C1BC5482972165218DB2402244C8
:1091000092444101828093F715008DC7B7E70400B0
:1091100083A7471A17A6FF1F1306863097D5FF1F90
:10912000938585B817A5FF1F0345853082971345A2
:109130001400E9B793F7250099CFB7E70400BC4FB7
:1091400013060064894517A5FF1F0345652E829706
:109150001345240065B793F7850085CF97D7FF1F88
:1091600083C707B685E7B7E7040003A8871A130784
:10917000401F97A7FF1F83C7A72B814613064006F2
:10918000994517D5FF1F035525B302981345840051
:10919000B5B793F745000145B5D3B7E4040083A7FD
:1091A000041817D5FF1F035525B18297BC4C130631
:1091B0000064914517A5FF1F034585278297134536
:1091C00044002DBF97D7FF1F83D707AF6398A7022F
:1091D00017D7FF1F2313B7AE17D7FF1F2310C7AE34
:1091E00017D7FF1F231DD7AC2E8617850100130547
:1091F000A51BBE85175301006700237A1785010060
:109200001305051C17630100670003910357450010
:1092100097D7FF1F83D747AA631EF704C167411181
:10922000F91722C417D7FF1F2328F7A837E4040033
:1092300097D7FF1F23A407A897D7FF1FA38C07A6C4
:1092400097D7FF1F238E07A67C4C06C6894517A516
:10925000FF1F0345E51D82977C4C914517A5FF1F15
:109260000345051D82972244B240410117030000C7
:10927000670003DA178501001305851417630100E1
:10928000670083897D15954763E2A71C1787010056
:10929000130787080A053A951C41011122CC06CE16
:1092A000BA972E848287178501001305E511976010
:1092B0000100E7806086A1A203C7250099476311DA
:1092C000F7022E8597000000E78080F48345640054
:1092D000178501001305451097500100E780E06BEA
:1092E00097B7FF1F238207F4178501001305851028
:1092F0007DBF03C7250095476319F702C16717D7DC
:10930000FF1F0357679BF91703D5A5006309F702F1
:10931000B7E7040083A7C7178297178501001305D5
:10932000650E97500100E780207F854717B7FF1F24
:10933000230CF7EE178501001305450F8DBF97D756
:10934000FF1F239BA79683D7E50097D6FF1F239681
:10935000F69683D7050197D6FF1F2391F69683D7FC
:10936000250197D6FF1F239CF69497D7FF1FA38351
:109370000794631BE502B7E70400BC4F09661306B8
:109380000690A14517A5FF1F0345850A829703563E
:10939000E4008355A400178501001305E5079750E5
:1093A0000100E780805F51B79307700F2316F1002B
:1093B000B7E7040083A7870D17A6FF1F03464607DC
:1093C0006C0082974DF9854717D7FF1FA304F78ECE
:1093D0005DB71785010013052506D1BD83C525009E
:1093E00091476392F50217850100130565069750B2
:1093F0000100E780607297000000E78060C1F240E2
:1094000062440561828099476392F5022285970044
:109410000000E780E0DF8345640017850100130545
:10942000A5FB97500100E7804057D1BF9547639A4D
:10943000F50083471400E1F3178501001305850348
:10944000BDB51785010013056503E1BF828037575D
:10945000315F97A7FF1F9387E7FE130777D598C360
:109460009356C500178701001307C7F0BA9683C546
:10947000060093568500BD8ABA9603C60600935629
:109480004500BD8A3D89BA962A9783C606000347E0
:109490000700238407002383D700A383E7002382E8
:1094A000B700A382C70097A7FF1F9387A7FA23835C
:1094B000B700A383C7002384D700A384E70082807A
:1094C000411106C697000000E780A0F8B7E7040046
:1094D00083A7871417A6FF1F1306C6F6D5450145B7
:1094E0008297B2404D4697A5FF1F9385A5F61305B9
:1094F00070304101170300006700C3B66171232477
:10950000811A37E40400832704082326111A232232
:10951000911A2320211B232E311917050000130552
:1095200045BB829717A9FF1F130989F09947854406
:109530002300A900231CF10097850100938585E293
:109540009307400617750100130585A4231CF10835
:109550002308910097C9FF1F9389C92097500100E4
:10956000E780A04383D5090017850100130585DE38
:1095700097500100E7806042294597500100E7803D
:10958000A04603D50900896997000000E78060ECD8
:109590008327441710088545130550308297832789
:1095A000441717A6FF1F1306E6EACD4513057030D2
:1095B00082978327441717A6FF1F1306A6E7B54512
:1095C00013056030829783274417300889451305B7
:1095D00010318297832744173009894513052031BC
:1095E000829783274415938509900D458297832799
:1095F00044159385099011458297A3059100230690
:10960000910002CD23080100230C0100832784165A
:1096100030099145130570408297832784161306FD
:10962000B10085451305004082978327841670009A
:109630008545130510408297832784163008854599
:10964000130520408297832784161008854513054B
:1096500050408297832704157D55829783274413B2
:109660007D5582977D5597A0FFFFE7806000832797
:10967000440C829797A0FFFFE780C0DB8327841408
:1096800017A6FF1F130606DCD545014582978947BB
:109690001306700F814528092306F1009790FFFFFC
:1096A000E780E0A68D471306000881452808230CB3
:1096B000F1089790FFFFE78080A59147230CF10008
:1096C000976701009387477E984383C747003AC84E
:1096D000230AF10097D0FFFFE78020B7700085458F
:1096E000054597A0FFFFE780C0FF30099305700F85
:1096F000094597A0FFFFE780C0FE300893050008EA
:109700000D4597A0FFFFE780C0FD10089545114566
:1097100097A0FFFFE780E0FCC16717C7FF1F130793
:10972000A759F9171CC32322070017A5FF1F13050C
:10973000E5CF97A0FFFFE780A0F98327C41D17C5D9
:10974000FF1F1305E55582973C48034509008545F1
:1097500082978320C11A0324811A8324411A032982
:10976000011A8329C1195D618280C16717C8FF1F73
:1097700003588854F9176301F8083DCDB5CD0111A0
:1097800026CAB7E4040083A7841222CC2E862315B0
:10979000B10006CE2A8401478146ED454285829775
:1097A0002AC611ED17850100130505BE975001006B
:1097B000E7808036F2406244D24405618280FC44F6
:1097C0000356A100A28582972C0017C5FF1F0355E1
:1097D000A54E97A0FFFFE78060FC69DD17850100BB
:1097E0001305C5BB97500100E780003383A7C4125F
:1097F000ED45280082977DBF82800DC5854717A75C
:10980000FF1FA30EF7C297A7FF1F238B07C2354682
:1098100097A5FF1F938505C213056030170300004D
:109820006700438497A7FF1FA38B07C0E9BF97C7B3
:10983000FF1F83C7E748A9EFC16717C7FF1F03577B
:10984000A747F9176306F7044111854722C417C7D4
:10985000FF1F2307F74637E404007C4C06C6A145EA
:1098600017A5FF1F0345C5BC82970323841A224412
:10987000B24097A7FF1F83C7A7BB17C5FF1F03559C
:10988000A5431307401F8146314699454101028394
:1098900082806D71232481102326111023229110C0
:1098A000328401CD8947630AF5028320C110032465
:1098B00081108324411051618280178501001305B6
:1098C000A5BCAE8497500100E7800025A2852685BF
:1098D00097C0FFFFE780A0B7C9BFB7E70400FC4708
:1098E00028008297178501001305C5BA975001001B
:1098F000E78080228347810039C41307000B63800F
:10990000E7021387A7051377F70F8D4663EDE6028D
:10991000A285280097C0FFFFE780602779B78547B9
:10992000E3F587F8834591001775010013058597C6
:10993000B335B00097A7FF1F2388B7769750010073
:10994000E780A0059DB703479100A207D98F35672F
:109950001307D7556385E7086368F7022D67130778
:10996000B7556387E70631671307C755638AE7046E
:1099700029671307A7556394E702A285280097C0BB
:10998000FFFFE780205F15B739679306E7656381BE
:10999000D70863E9F6001307E7556384E706A28555
:1099A00028003DB73D679306F755638AD70613072E
:1099B000F766E396E7FE97C0FFFFE780A077F5B56F
:1099C0000146A285280097C0FFFFE780E047F1BD70
:1099D000A285280097C0FFFFE7800058F9B58947A6
:1099E000E3F587EC97000000E780A0E49305E4FF2F
:1099F000C205C1811305A1009790FFFFE780A07CFD
:109A00006DB5A285280097C0FFFFE780A05771BD04
:109A1000A285280097C0FFFFE780606279B597C0F4
:109A2000FFFFE780E06A51B5C16717C5FF1F035507
:109A3000A528F9176307F500B7E7040003A3C717C4
:109A400002838280854717C7FF1F2305F72601453C
:109A500017F3FFFF670043591783FFFFE702836691
:109A60002A8408452E89B28919C900C197150000BA
:109A70009385A586610597300100E7802005814424
:109A80007D5A97100000E780E03963C7A404814441
:109A900097100000E780003A63C8A40497C7FF1F2F
:109AA000938747229C43DC47B307F9409187230201
:109AB000F400638309048327C900B307F440958742
:109AC000A302F4001C4C89C79C4799C32285829746
:109AD0001783FFFF670043625C44139714008504FB
:109AE000BA972390470171BF1C481397140085044F
:109AF000BA972390070069BF832789000547B307FA
:109B0000F4409587A302F40083570400638EE702B4
:109B10008DC309476384E7040D47E395E7FA978708
:109B200001009387E7E91CCC97870100938747EAF8
:109B300011A897870100938727B01CCC9787010055
:109B4000938787B05CC8BDBF978701009387C79B89
:109B50001CCC978701009387279CEDB7978701005E
:109B60009387C7EA1CCC97870100938727EBD9BF5F
:109B700095E51783FFFFE7028356004618448347A5
:109B8000940075839D8B6317F70097100000E780A2
:109B900060B448C41783FFFF6700A3568280178311
:109BA000FFFFE702235213893500C16442094111C6
:109BB000AA890144F11413590901054A2EC69710C8
:109BC0000000E7802026B2456348A400014541011A
:109BD0001783FFFF6700435283A709001317140080
:109BE000BA9783D707006388B700639497006374BC
:109BF0002A010504E1B70545D9BF1783FFFFE70236
:109C0000834BAA892E89328BB6843A8ABE8A97A062
:109C10000000E780C0FE71C9268597200000E7801C
:109C2000C00C8D4763E7A7007D551783FFFF6700D2
:109C3000034C83DB440097100000E780A0242A84B3
:109C400097100000E78040259307740031443305E6
:109C5000850263CDA70297100000E780A02297102D
:109C60000000E78020222A8497100000E780C022AD
:109C70009307740031443305850263C3A70497102A
:109C80000000E78020209307450029A897100000D6
:109C9000E7808020330585021307F0179307C0176C
:109CA000E35FA7FA2D55E3C277F963040B02D6866A
:109CB0005286A6854A8597200100E780C0BDB5B7CA
:109CC00097100000E780401D330585029307C5FF0C
:109CD000D1BF832749001385C90083D5270097008A
:109CE0000000E78000EC61F581B769553DBF97C77B
:109CF000FF1F239BA7FC97C7FF1F9387A7FC9043D9
:109D000081470C463307F500420741836393B70050
:109D100082805446139847008507C2962390E60038
:109D2000D5B797C7FF1F9387E7F99C4303C5870003
:109D3000828017C5FF1F035525F982801783FFFF17
:109D4000E702E339C1671387D7FF630BE502636A54
:109D5000A700F1176300F50201451783FFFF6700B5
:109D6000433A1387E7FF6302E502FD171D8D1335A4
:109D70001500E5B797500000E780602A7D15C5BF44
:109D800097500000E780E0FED5BF97500000E780C5
:109D900000FDEDB71783FFFFE70263344111AA848A
:109DA00001442EC697100000E780C008B245634802
:109DB000A400014541011783FFFF670083349C48DD
:109DC000131514003E9583570500E385B7FE05047F
:109DD000C9BF03485500814693F7F60F63E50701B5
:109DE00081473E858280584593975600BA9703D79E
:109DF00027006316B70003D70700E304C7FE8506F4
:109E0000E1BF8346450001479377F70F63E4D7002E
:109E1000814711A81C45131657000507B29703D6B2
:109E20000700E313B6FE3E8582801783FFFFE7023B
:109E3000632993170501C18797CAFF1F938A8AE890
:109E4000635BF00883A70A00C0479C4703570400E0
:109E5000198D420541816368F5000144228517830D
:109E6000FFFF6700632912052A94CDBFDC471394D6
:109E70004900014A3E94834744006341FA02014A83
:109E8000834754006349FA028509C20993D909013D
:109E900083A70A009847E3EBE9FCC1B71C441319F8
:109EA0005A00A6853E994A8597000000E780C0EEDB
:109EB00005E1050AC9B75C4413195A00A6853E9905
:109EC0004A8597000000E78020ED19E1050A4DBFA3
:109ED000E30C09FA61B7AA8481495DBF1783FFFFCC
:109EE000E702E31F1C452A8481E79307C5001CC5D0
:109EF0001C44231204001CC09307F00F63EDB7004D
:109F000093F5F50F228597200000E780C0E51783C1
:109F1000FFFF6700031F93940501C167C18063F9C8
:109F2000F500A685228597200000E780E0E8C5B708
:109F3000C18193F5F50F228597200000E780A0E20C
:109F4000A685228597200000E780E0E3C9B797C780
:109F5000FF1F938727D7884382801C4599C797C7DF
:109F6000FF1F23A1A7D6014582807D55828097C718
:109F7000FF1F938727D5984383474500484792079B
:109F80003E9582801783FFFFE702631561710045EC
:109F90001C183EC6B70780013EC81C183ECA83572E
:109FA000440002CE02D002CC231EF100834784007D
:109FB0002A8902D22301F1023C083ED402D697003E
:109FC0000000E78000FB835705002316F10297503D
:109FD0000000E78000C82307A1025C40035564002D
:109FE000F18313F717008347F10252055181F99B62
:109FF000D98FA307F10297100100E780207939CDAE
:10A00000AA840355050097A00000E78020C083D7ED
:10A0100004002AD26800231CF10083D72400231DEA
:10A02000F1001C4803D647008C4397200000E780CE
:10A03000A0D08347B400CA861776010013064646AF
:10A040008117A305F4006C00481097200100E780F9
:10A0500080845D611783FFFF6700A30A2155D5BF88
:10A060001C45B1CF03C5A700894613576500630B94
:10A07000D7028D46630ED70285466300D7021307C9
:10A0800040063305E50203C7B700418B15CB83C7F4
:10A09000B700BD8B3355F54082801375F503130768
:10A0A000803EC5B709671375F50313070771D1BF64
:10A0B000372709001375F5031307077CD9B7014546
:10A0C00082801783FFFFE702830103A98500630CE9
:10A0D00009048347B900AE8493F7070E85C303458F
:10A0E0009900930520030D810505B305B502884449
:10A0F000610597300100E78080AD35A02E8597007F
:10A100000000E78020F62A8419CD97000000E78040
:10A11000605C8325C900B307B54063FA87002E94BD
:10A12000B305A440E9F51783FFFF670083FD85456C
:10A130007DBF1783FFFFE70283FA2A8403D505005A
:10A14000011132C636C43AC22EC002CA02CC02CEB7
:10A1500097A00000E78080AB82452ACA22852ECCDA
:10A1600097000000E780E0E003570500231EE100B0
:10A1700097500000E780E0ADA24632469247230F99
:10A18000A10036874C08B286228501469700000060
:10A19000E780E0A605611783FFFF670083F617835A
:10A1A000FFFFE702C3F361711C183EC6B7078001C9
:10A1B0003EC81C183ECA3C0800453ED4AA8402CCC6
:10A1C00002CE02D002D202D697000000E78060DA09
:10A1D0008357050035592316F10297500000E78098
:10A1E00040A72307A10209C48357440081EB2159EA
:10A1F0004A855D611783FFFF6700A3F00355640084
:10A200005205518197100100E78040582A8965D195
:10A210008347B40093F7070E99C71305840197305D
:10A220000100E780009D83574400231EF10083470F
:10A2300084002301F1025C4003550900D98313F720
:10A24000070883471102231CA10093F7F707D98F52
:10A25000A300F10283572900231DF1005C40F18324
:10A2600013F717008347F102F99BD98FA307F10277
:10A2700097A00000E78080992AD235D983479400BF
:10A280006800139757008347B400FD8BD98FA3054F
:10A29000F4001C4803D647008C4397200000E78059
:10A2A000A0A9A687177701001307871F740005462A
:10A2B0004C10268597000000E78060942A890DD90C
:10A2C0008347B400A685FD8BA305F400970000002A
:10A2D000E78060DF31BF1783FFFFE70243E083249D
:10A2E00085FE2A844111268597000000E78080D7EB
:10A2F000834734FF93F7070E8DCB2AC62685970038
:10A300000000E78060C809CD834734FFB245FD8B6C
:10A31000A309F4FE91C5228597300100E780208BC8
:10A3200041011783FFFF6700C3DD7DD98327C4FF89
:10A330002685829775F5834734FF93F7070E91C7FB
:10A34000228597300100E780C08A032584FE9700AC
:10A350000000E78000E5E9B71783FFFFE70223D598
:10A360009C4141112A8903C7070089472E849356CF
:10A3700067006380F6040D466388C6049307F00700
:10A380006304F7022E8597200000E78060ABAA8463
:10A390008149C16B130C490097C7FF1F93878792B0
:10A3A0009C43984763E4E90441011783FFFF67007A
:10A3B000C3D303D745008547E3F8E7FE2E859720F2
:10A3C0000000E78040ADE1B703D74500E3FEE7FCBE
:10A3D0002E8597200000E780A0A6AA8422859720DA
:10A3E0000000E78000A8C204C98C5DB7DC470355B4
:10A3F000A900139A49003E9A93170501C187635D2E
:10A40000F00083570A006397A70263E7740383276A
:10A41000CA00034D5A002DA0A1672167A98F130719
:10A42000F7EFE374F7FE6397090097000000E780F9
:10A43000209161FD85098DB783278A00034D4A006D
:10A44000835DA90003576900216A138BC7003AC6D0
:10A45000814A33CA4D01631E5D0197C7FF1F938771
:10A46000E7869C43E1DBA28662868145268582974A
:10A47000D1B7A1679387F7EF930C4BFF63F24703C4
:10A48000B2455A8597F0FFFFE780A0710DC1032701
:10A490008B00104709CE10436382C4023107D5BF39
:10A4A000EE85668597000000E780008F71F993863E
:10A4B0001A0093FAF60F130B0B0271BF8356440078
:10A4C0005C43E3E9F6F622853AC697200000E78070
:10A4D0002081A1679387D7042A8A035D440032470D
:10A4E00063E897008347D90093E707F8A306F900CC
:10A4F0001C4766852286E2858297C1670844FD175E
:10A50000337AFA00529508C02312A40125B797B7F1
:10A51000FF1F9387277B9843814715C314478147C3
:10A5200063FFD500939745004C47BE9519C903C7F3
:10A53000550081476375E600DC451606B2973E85F7
:10A54000828003C745008147E37BE6FE16069C45F3
:10A55000F5B71783FFFFE702E3B6AA892E8A814485
:10A5600097BAFF1F938A0A7683A70A00984763E683
:10A57000E4001783FFFF670023B8DC47139444000F
:10A5800001493E9413BB140083474400634BF90018
:10A59000014913BB140083475400634FF90085043D
:10A5A000E1B70844931759005287DA860146A2851D
:10A5B0003E9582990509C9BF4844931759005287AF
:10A5C000DA860546A2853E9582990509E9B7178383
:10A5D000FFFFE702C3B0814517F5FFFF13050548EC
:10A5E00097B7FF1F2392076E97000000E780A0F641
:10A5F0001783FFFF6700E3B097B7FF1F9387876C50
:10A600009C4395C31783FFFFE70263AD814517F5B0
:10A61000FFFF1305A54497000000E780C0F31783F0
:10A62000FFFF670003AE82801783FFFFE70283A965
:10A6300037E404008327841241112315E100AE8919
:10A640003289368A3A8681460147ED45AA84829747
:10A650002AC621C90356A100D28597400100E78090
:10A6600060288327C413CE8526858297058905C96E
:10A670008327440D2314210101462C00268582974F
:10A680002A8401C9B7E7040083A7C712ED45280053
:10A690008297228541011783FFFF6700E3A54944A4
:10A6A000D5B76554FDB75C41FD175CC18280178347
:10A6B000FFFFE702C3A2B7E70400FC5F829795475C
:10A6C0003305F50281450D811783FFFF670063A302
:10A6D0001783FFFFE702A3A0B7E70400FC5F8297A0
:10A6E00095473305F5020D811783FFFF670063A1CE
:10A6F0001783FFFFE702A39EB7E7040083A7870B3A
:10A700000355050082971783FFFF6700839F178318
:10A71000FFFFE702C39C035505003287AE861796FC
:10A72000FF1F035646D997B5FF1F9385655A9700BB
:10A730000000E780A0EF1783FFFF6700839C17836B
:10A74000FFFFE702C399B7E7040083A7C717829703
:10A750001783FFFF6700E39A1783FFFFE702239841
:10A76000B7E7040083A7871397B5FF1F9385455666
:10A77000829701451783FFFF6700A3981783FFFFA8
:10A78000E702E395B7E7040083A7C71F8145179544
:10A79000FF1F035545CE82971783FFFF670063961F
:10A7A0001783FFFFE702A393B7E7040083A787138C
:10A7B00097B5FF1F9385C552829701451783FFFF09
:10A7C000670023941783FFFFE7026391B7E7040054
:10A7D00083A7C71F81451795FF1F0355C5CF8297D4
:10A7E0001783FFFF6700E3911783FFFFE702238FC3
:10A7F0002E8597800000E78080B397800000E78077
:10A8000080F01783FFFF6700C38F1783FFFFE70206
:10A81000038D97800000E78080FA1783FFFF6700B1
:10A82000438E5C49E1175CC95CC583572501A107CC
:10A830002319F50083570501A1072318F50082802D
:10A84000F1473305F50297B7FF1F9387674B9C438A
:10A850003E9582808D476315F60803D746008547ED
:10A8600063F0E7081783FFFFE702638736853684C6
:10A870002E8997100000E780A05C29C98357440007
:10A8800093140501C18063E39704228597100000AB
:10A89000E780005BFD14231294009307A00263007D
:10A8A000F5029307B0026307F50293079002631F56
:10A8B000F500228597000100E780608901A8014624
:10A8C000CA85228597A00000E78000B41783FFFFA8
:10A8D00067002383228597100000E7806007FDB79B
:10A8E000828097B6FF1F9386E6419C42014599CF2F
:10A8F0009843D44217B6FF1F2326E6406396D7003D
:10A9000097B6FF1F23A2E6401385C7FE8280177308
:10A91000FFFFE702C37C97000000E780A04B714473
:10A9200033058502914597900000E780C0EC11E562
:10A9300065551773FFFF6700C37C97B7FF1F23AFF1
:10A94000A73A97000000E780E0483305850291456B
:10A9500097900000E78020EA61DD97B7FF1F23A1F1
:10A96000A73A97000000E780E04697B7FF1F2391C2
:10A97000A73897000000E780E04597B7FF1F239AAC
:10A98000A736977701009387E7B617B7FF1F2325F0
:10A99000F73697070000938707E917B7FF1F232BA8
:10A9A000F734014579B71773FFFFE7024373AA85B0
:10A9B00017B5FF1F1305C53397100000E780605FD0
:10A9C0001773FFFF6700E3731773FFFFE70223713D
:10A9D00097000000E78060FD97100000E780E05ED0
:10A9E00097B7FF1F938707329C4391CF1387C7FE0A
:10A9F00019CB83D5C7FF17B5FF1F13052531972046
:10AA00000100E780C01C1773FFFF6700836F177397
:10AA1000FFFFE702C36C97000000E780C0EC09CDA0
:10AA2000834785002A8493F7070499EB0355E500D3
:10AA300097000000E78080F91773FFFF6700636CE1
:10AA40008347C5009304450117B9FF1F1309892BDC
:10AA500085E3832709005CC997B7FF1F23A4972AC2
:10AA600083274900F1FB97B7FF1F23AF9728E9B76A
:10AA7000FD172306F500610597800000E78060DA86
:10AA80008307840063CB07048347840093E707F8B8
:10AA90002304F400B7E704009C5F82974205A947AE
:10AAA00041813375F5028347840093F707FCC98F12
:10AAB0002304F4008347D4003E951C402318A400CF
:10AAC00089CF984319CB8347C400504081458507FF
:10AAD0003305F502420541810297832709005CC8CE
:10AAE00097B7FF1F23A097228327490089E797B7CD
:10AAF000FF1F23AB97208347C4009DDF83550401CC
:10AB000017B5FF1F1305852097200100E780200C53
:10AB100025B71773FFFFE702835C97B7FF1F938783
:10AB200027449C4701448583858B85E3AE84B285A9
:10AB30003A8697100000E780204F2A8419C59710A5
:10AB40000000E7806045829408CC22851773FFFFE0
:10AB50006700235B1773FFFFE702C35641112E897D
:10AB600032C6AA8997000000E780C0313247130639
:10AB70000502CA86970500009385C5CC17B5FF1F4F
:10AB80001305051797000000E780E0F82A8425C91F
:10AB90009304C50097000000E780E0411946AA85AC
:10ABA000268597100000E780201985452685971097
:10ABB0000000E780001517750100130565914E959B
:10ABC00083450500268597100000E780C0195C4882
:10ABD00031468145A1075CC85CC483572401E11755
:10ABE0002319F40083570401E1172318F4001C4CC7
:10ABF0003E859770FFFFE7808051A30425012285E1
:10AC000041011773FFFF6700234F1773FFFFE70230
:10AC1000034D4111AA842EC632C497100000E7806C
:10AC2000003A004DB2452246834784000CC050C014
:10AC300093F7F70393E707042304F40023180400B1
:10AC4000268597100000E780203583479400A946A9
:10AC50002317A40013D7370005073307D7029D8BAE
:10AC600085072306F400A306E40083C70401D8483F
:10AC70008507230FF7FE17B7FF1F1307A7085843D1
:10AC8000232A04009307440129E317B7FF1F232D4C
:10AC9000F70617B7FF1F2327F70617B4FF1F130484
:10ACA000E406228597200100E780A0E41C44858B00
:10ACB0005D8D19E58145228597200100E78020F10F
:10ACC00041011773FFFF6700C3431CC317B7FF1F82
:10ACD000232CF702D9B71773FFFFE702434097050C
:10ACE0000000938565B7014597000000E78000B03C
:10ACF00001451773FFFF6700C3401773FFFFE702AB
:10AD0000033E97000000E78080B01773FFFF6700E5
:10AD1000433F8347C500A5E31773FFFFE702233CCA
:10AD20002A840355E50097000000E78000C821C190
:10AD30008347840093F7F7FB2304F4001C4091C77A
:10AD4000DC4381C74C400145829797000000E780B3
:10AD500080B917B5FF1F130565FB97200100E78039
:10AD600040E90355E40097000000E78020C6177310
:10AD7000FFFF6700033982801773FFFFE702233666
:10AD800097B7FF1F938707F897050000938565C85D
:10AD900017B5FF1F130585F723A0070023A207009F
:10ADA00097200100E78080D21773FFFF67006335AB
:10ADB0001C4D91CFDC4381CF1773FFFFE702233295
:10ADC0008345070082971773FFFF670083338280F4
:10ADD00097B7FF1F9387C7F59C4303C50700828081
:10ADE00097B7FF1F9387C7F49C4303C51700828062
:10ADF00097B7FF1F9387C7F39C4303C52700828043
:10AE000097B7FF1F9387C7F29C4303C54700828013
:10AE100097B7FF1F9387C7F19C4303C53700828014
:10AE200097B7FF1F9387C7F09C4303C557008280E5
:10AE300097B7FF1F9387C7EF9C4303C567008280C6
:10AE400097B7FF1F9387C7EE9C4303C577008280A7
:10AE500097B7FF1F9387C7ED9C4303C58700828088
:10AE600097B7FF1F9387C7EC9C4303C59700828069
:10AE700097B7FF1F9387C7EB9C4303C5A70082804A
:10AE800097B7FF1F9387C7EA9C4303C5B70011E13B
:10AE90001D45828097B7FF1F938787E99C4303C5B1
:10AEA000C700828097B7FF1F938787E89C4303C53D
:10AEB000D700828097B7FF1F938787E79C4303C51E
:10AEC000E700828097B7FF1F938787E69C4303D5EF
:10AED0000701828097B7FF1F938787E59C4303C5CF
:10AEE0002701828097B7FF1F938787E49C4303D590
:10AEF0004701828097B7FF1F938787E39C4303D561
:10AF00006701828097B7FF1F938787E29C4303D531
:10AF10008701828097B7FF1F938787E19C4303C512
:10AF2000A701828097B7FF1F938787E09C4303C5E3
:10AF3000B701828097B7FF1F938787DF9C4303C5C4
:10AF4000C701828097B7FF1F938787DE9C4303C5A5
:10AF5000D701828097B7FF1F938787DD9C4388576F
:10AF6000828097B7FF1F9387A7DC9C4303D5C70256
:10AF7000828097B7FF1F9387A7DB9C4303D5E70227
:10AF800019E11305800C828097B7FF1F938747DA7A
:10AF90009C4303C50703828097B7FF1F938747D958
:10AFA0009C43C85B828097B7FF1F9387E7D788438E
:10AFB000828097B7FF1F938767D78843828019E104
:10AFC0007D558280F5DE984265DFFDD917B7FF1FFA
:10AFD000130707F91847AA877155058B631D0724C6
:10AFE00003C507001547E37DA7FC03C7370013051A
:10AFF000F0057D171377F70FE364E5FC03C35700F3
:10B00000E30003FC83C86700E38C08FA03C77700FA
:10B01000494579171377F70FE364E5FA03C7A700EB
:10B0200011481305F7FF1375F50FE36BA8F803CE6E
:10B0300097000D481305FEFF1375F50FE362A8F89E
:10B0400003C8B7006309080065181378F80F1305E3
:10B05000600DE36705F703C5C700794879151375D7
:10B06000F50FE36FA8F403C8D7000D457D181378DA
:10B07000F80FE36705F503D80701930E4017511841
:10B08000420813580801E3ED0EF303C8E7007D18EA
:10B090001378F80FE36605F303C827017D181378CA
:10B0A000F80FE36F05F103C88700C54E75181378D4
:10B0B000F80FE3E70EF103D86701856E938EBEE0CB
:10B0C0006D18420813580801E3EC0EEF03D847014E
:10B0D0006D18420813580801E3E40EEF03D8870106
:10B0E0007918420813580801E36C05ED03C8A7015D
:10B0F0007D181378F80FE36505ED03C5B7011D480A
:10B100007D151375F50FE36DA8EA03C5D7017148E6
:10B1100079151375F50FE365A8EA03D5E701130860
:10B12000E00F7D1542054181E36CA8E803C50702E5
:10B13000494879151375F50FE364A8E8C85301C9A8
:10B1400037C834005915130858BFE36BA8E603A8A5
:10B15000870237C53400130555BF5918E36205E768
:10B1600017B5FF1F2324C5BC03C6050117B5FF1F74
:10B170002320F5BC0545E375C5E403D82501D04976
:10B1800033760603E31E06E203C61501E30A06E270
:10B1900017B6FF1F232AB6B883C527000146638769
:10B1A000A50003C61700F1453306B60283C707039F
:10B1B0009305C00272971A071307C70516031A975B
:10B1C00096084697B387B70241553E973297420794
:10B1D00041836362E8061773FFFFE70243F0368599
:10B1E00097800000E780406C97000100E780C04B2B
:10B1F0002A8497A00000E780205E2A9497F0000040
:10B20000E780002A2A9497900000E78040852A94DE
:10B2100097F0FFFFE780E06F2A9497400000E780F7
:10B2200000972A9497700000E78040A0229517733A
:10B23000FFFF670003ED82801773FFFFE70223EA39
:10B240004111A307A10097A00000E78040C9930522
:10B25000F100170500001305E5B597F0FFFFE78043
:10B26000802F014541011773FFFF670083E91773C2
:10B27000FFFFE70243E417B4FF1F130464CE032863
:10B28000840079599368180097B4FF1F23AE14CD3A
:10B290001378180063100802BA84BE89368B328A8C
:10B2A0002E89AA8A97F0FFFFE780E0A77D152695F3
:10B2B00019E531594A851773FFFF670043E397F09B
:10B2C000FFFFE78040A67D152695A167E353F5FEB5
:10B2D00097B7FF1F938787FF98433E8C814B01CB25
:10B2E000014597F00000E780C047933B15004A8571
:10B2F000DA865686D28597900000E78060512A89C9
:10B3000011CD1C44F99B17B7FF1F232FF7C48327C8
:10B310000C00CDD3E3800BFA829769BF268597B7DF
:10B32000FF1F23A107C497F0FFFFE780809C4146E1
:10B33000CE8517B5FF1F130525CC97300100E78098
:10B34000605A97D00000E780E09C0325040B97D05B
:10B350000000E780A0A0054597D00000E780A0A7E7
:10B36000054597000000E78060EDA9B797B7FF1F7C
:10B37000938707BF9C47858BEDC71773FFFFE702D5
:10B3800003D617B5FF1F130565C597B7FF1F23A980
:10B3900007BC97B7FF1F23A707BC97B7FF1F23A5BD
:10B3A00007BC97200100E780C08497500000E78029
:10B3B00080F997100100E780405097100100E78066
:10B3C000405697B7FF1F938727B89C4391C7054501
:10B3D00097800000E780E02397B7FF1F938787A03F
:10B3E0009C4399C741657D1597700000E780E0A5F3
:10B3F00097F00000E780804197D00000E78020931D
:10B4000097B7FF1F938787CA9C431397170163560B
:10B41000070097F00000E780A0B097B7FF1F23ADAB
:10B4200007BC97B7FF1F23AB07BC97B7FF1F23A924
:10B4300007BC97B7FF1F23A707BC97000000E78052
:10B44000008C97000000E780A07597F0FFFFE78071
:10B45000401897F00000E780E0D91773FFFF6700FE
:10B4600043CA828097B7FF1F938787AF8843828044
:10B4700097B7FF1F9387C7AEC8438280B7E7B00076
:10B480009387075063E1A70297B7FF1F938747ADE4
:10B49000D843FD576367E50097B7FF1F23A4A7AC08
:10B4A00081473E858280B957EDBF1773FFFFE702E2
:10B4B00003C397800000E780607597800000E780F5
:10B4C000C0771773FFFF6700C3C31773FFFFE7025F
:10B4D00063BF2A849304140201112E85B289A685C4
:10B4E000214636C63A8997300100E780403D0DE994
:10B4F000B24638082686CE8513059404975000007E
:10B50000E780604121462C084A8597300100E7809A
:10B51000003B1335150005611773FFFF6700C3BDBE
:10B520000145D5BF1773FFFFE70263BB93054506CF
:10B5300017B5FF1F1305058097100100E7802069EC
:10B540001773FFFF6700E3BB1773FFFFE70223B921
:10B5500041112EC697F0FFFFE780C017B24588C1A2
:10B5600041011773FFFF6700C3B91773FFFFE702BD
:10B5700063B5AA842E8497800000E780006CAA89B6
:10B580008545228597000000E780E07D83C7E401C0
:10B590001389940899E313890403CE8522859700C3
:10B5A0000000E780407C2146930519022285970020
:10B5B0000000E780607897B7FF1F9387679A8C43F6
:10B5C000228597100000E780C0822146938584027F
:10B5D000228597000000E78020761773FFFF670041
:10B5E000A3B11773FFFFE70203AD397197F00000B5
:10B5F000E780E0B49305400661E997800000E780AA
:10B6000000606302051497A7FF1F83C7677413B711
:10B61000170097A6FF1F238DE672014499CFC164DE
:10B6200017B9FF1F1309C9939309400EFD14970022
:10B630000000E78020836342A40A97F0FFFFE780C1
:10B6400060094169B7290900096AFD7A2A8B81449A
:10B650007D199389F97B130A0A71938A8AC7970027
:10B660000000E780208063D7A4041304400EB38752
:10B67000840217B7FF1F1307A78E0324070B3E94FE
:10B680008357C4016382270B18403307EB4063EAFA
:10B69000E900834744008507B3874703D69763656E
:10B6A000F70801468145094597F0FFFFE780C04A4A
:10B6B000AA8B29E597400000E780808385476317C0
:10B6C000F50689659385057117A5FF1F1305856626
:10B6D00097100100E780A04F95A0B307340303271C
:10B6E000090BBA9703D7C7016308970003C7570030
:10B6F000A38207002382E700050415BF9305C50058
:10B70000228597000000E78080E65E8522869765A7
:10B710000100938525DD97F0FFFFE780404F5E85B0
:10B7200097100000E780608A850415BF97B7FF1F58
:10B73000938707839C478D83858BC1F7216117739E
:10B74000FFFF6700C39A01468545094502D002D232
:10B7500002D402D697F0FFFFE7800040AA8479DD8B
:10B7600097F00000E780E09C1389C4002A8481459B
:10B770004A8597000000E780005F0C4041464A85FB
:10B7800097000000E780405B832944006385090C33
:10B790004E8502D802DA02DC02DE97300100E78033
:10B7A000E0382ACE141005462C0808184ECC9750C5
:10B7B0000000E780E00A1375F50F51ED8355840012
:10B7C00093E525004A8597000000E780E05E11467A
:10B7D0000C104A8597000000E780005601469765E7
:10B7E00001009385A5D0268597F0FFFFE7802042D2
:10B7F000268597000000E780407D5C40A1D301468C
:10B8000085450D4597F0FFFFE7800035AA841DD5DB
:10B8100048401389C40097300100E78020312AC6D0
:10B820004A8597000000E780404C3246636FC500B0
:10B830004C404A8597000000E78000500146814552
:10B84000268597F0FFFFE780803C26859700000063
:10B85000E780A077E5B583558400ADB71773FFFF88
:10B86000E702E38797A7FF1F9387876F9C471DC158
:10B8700093E7870017A5FF1F1305C54B17A7FF1FE9
:10B880002324F76E97100100E78040321773FFFF03
:10B8900067002387DD9B17A7FF1F2327F76C9730CF
:10B8A0000000E780E0647DF117A5FF1F13058548C0
:10B8B00097100100E780E033D1BF1763FFFFE70275
:10B8C000837F4169AA892E8AB28A368BBA8B8144DA
:10B8D00017ACFF1F130CCC68930C400E7D1997F02A
:10B8E000FFFFE780205863C4A40001443DA03384D7
:10B8F000940383270C0B3E948357C401638627056A
:10B900005A87D6865286CE85130504039700000019
:10B91000E780E0BB01C923800B0022851763FFFF8E
:10B920006700E37C8347F40185C35A87D686528635
:10B93000CE851305940897000000E78040B909C53B
:10B9400085472380FB00D1BF850451BF8357450045
:10B950006380071E1763FFFFE702C37601112A8485
:10B9600097000000E780C04D09C985476309F506C7
:10B9700005611763FFFF6700237897E00000E78009
:10B98000007C7DF5835744004947ED9BE392E7FE39
:10B99000C145228597000000E7804033AA842285B4
:10B9A00097000000E780204F0357440002CE9147E4
:10B9B0002A89631AF700228597000000E780A051CA
:10B9C0003C082ACC3ECE97E00000E78080765C55AC
:10B9D000C5D374084A86A6850545829751BF03578B
:10B9E0004400D147E3F6E7F8032A0400C16901499E
:10B9F00097AAFF1F938ACA56130B400EFD1997F0A2
:10BA0000FFFFE7802046634FA90E2285032A04002A
:10BA100097000000E780C042A1452A89228597004F
:10BA20000000E780A02AAA84228597000000E78012
:10BA3000804A14402A86AA8978082685CA859700F4
:10BA40000000E780C0E7AA8405D503C7F401894751
:10BA50006315F7008347C10181DF5546D285138501
:10BA6000640097300100E780E0E70145978000001F
:10BA7000E780C01901C583D7C401A5E797A7FF1FB9
:10BA80009387074E9C4793551900858913D7370034
:10BA9000058B01CF8983858B6399B70001452EC63D
:10BAA00097000000E780C0DBB2454E85978000001C
:10BAB000E780601F0346C1012A849375190026851B
:10BAC00097900000E780E03935C126859780000017
:10BAD000E780E018268511C0014597800000E780C7
:10BAE000004C97300000E780A0408547E312F5E85E
:10BAF00083C754001307F00FE38CE7E68507A382A2
:10BB0000F400BDB5B304690383A70A0BBE9483D7C1
:10BB1000C401638B37015546D28513856400973085
:10BB20000100E780C0D955DD0509D1BD5DD86DB7ED
:10BB300082801763FFFFE702E35897800000E780E9
:10BB4000000C05C1C164014417A9FF1F1309494135
:10BB50009309400EFD1497F0FFFFE780A030634E7D
:10BB6000A40017A5FF1F1305E51C97100100E7802F
:10BB7000E0031763FFFF670023583305340383276F
:10BB8000090B3E958357C501638897002312050072
:10BB900097800000E780A00C050475BF97A7FF1FE2
:10BBA0009387073C9C478D83858B8DE31763FFFF4D
:10BBB000E702E35217A5FF1F1305C51797100100F1
:10BBC000E78020031763FFFF6700A353828017639A
:10BBD000FFFFE702C350970500009385C5A017A596
:10BBE000FF1F1305251597100100E78020EE17634E
:10BBF000FFFF670003511763FFFFE702434E8841D1
:10BC0000B7E70400BC5B050542054181829709C581
:10BC100085472300F50005051763FFFF6700634EA6
:10BC200083C7F5FF2E858507A38FF5FE828083C726
:10BC3000F5FFFD1793F7F70FA38FF5FE99EF176345
:10BC4000FFFFE702C349B7E70400BC571385F5FFC0
:10BC500082971763FFFF6700C34A82801C41035726
:10BC600045008D8FBA951CC12312B5003E85828098
:10BC700093D78500A2051441DD8D835745001387B6
:10BC8000E6FF18C189072312F50013D6850041117C
:10BC9000238FB6FEA38FC6FE410182801841930711
:10BCA000F7FF1CC18357450085072312F500A30F3A
:10BCB000B7FE8280835745008D8F2312F5001C410B
:10BCC000BE950CC12E858280AA8703D74700084104
:10BCD0000D8FAA952392E7008CC3828018410845F6
:10BCE0003305A740828083574500035765001D8FA9
:10BCF0001C4108453385A7403305A7408280176360
:10BD0000FFFFE702C33D41112EC62A8497000000C1
:10BD1000E780A0FDB2456373B50001A083574400DE
:10BD20000840BE952312B4003E9541011763FFFF02
:10BD30006700233D1763FFFFE702633A41112E843A
:10BD4000B28532C697000000E780A0FB3246A2858C
:10BD500097300100E78000B941011763FFFF6700DA
:10BD6000433A1763FFFFE70283372E848545970028
:10BD70000000E78000F9230085001763FFFF6700DC
:10BD800043381763FFFFE702833541112317B100E2
:10BD9000894597000000E780C0F68347E100230053
:10BDA000F5008347F100A300F50041011763FFFF91
:10BDB000670023351763FFFFE702633293D78500DF
:10BDC000A2054111DD8D2317B100894597000000C0
:10BDD000E78020F38347E1002300F5008347F1006B
:10BDE000A300F50041011763FFFF6700833117636C
:10BDF000FFFFE702C32E1397850193D78501C16624
:10BE0000938606F0D98F13D78500758FD98FA20539
:10BE10003707FF00F98D4111DD8D2EC69145970042
:10BE20000000E78000EE6C00114697300100E780CB
:10BE300060AB41011763FFFF6700A32C1763FFFF8F
:10BE4000E702E3291C41854503C407009700000071
:10BE5000E78080E622851763FFFF6700832A176368
:10BE6000FFFFE702C3271C414111894503C70700B3
:10BE700083C717002307E100A307F1009700000024
:10BE8000E78080E30355E10041011763FFFF67008E
:10BE900043271763FFFFE70283241C4141118945B3
:10BEA00003C7070083C717002307E100A307F100BA
:10BEB00097000000E78040E08357E100410113D57F
:10BEC0008700A2075D8D420541811763FFFF670070
:10BED00043231763FFFFE70283200C4141112A84AB
:10BEE0001146680097300100E780C09F9145228588
:10BEF00097000000E78040DCB247C166938606F0F9
:10BF00001397870113D58701598D13D78700758F34
:10BF1000598DA2073707FF00F98F5D8D4101176327
:10BF2000FFFF6700031E1C45BE950CC18280AE87D3
:10BF3000944391E6584101EF0CC15CC1828003C774
:10BF4000570013671700A382E700B687D5B70CC365
:10BF5000EDB7AA87084119CD1841D44398C363139C
:10BF6000D500D8C32A87034657009376160081E68A
:10BF7000232007008280944381CA8C4203A8470093
:10BF80008CC363930601CCC3799A14C3A302C70080
:10BF90003687D1BF1C45DC471D8DB777DBB693874D
:10BFA00077DB09853305F502420541818280F1473F
:10BFB000B385F50248452E95828083474500850765
:10BFC0002302F50082801763FFFFE70243112A84F2
:10BFD00009E41763FFFF6700C31283474400F5DBE2
:10BFE000FD1793F7F70F2302F400E5F71C4403D77E
:10BFF000270005072391E700DC4399C32285829738
:10C000004C4889CD83475400898B99E71C4422858D
:10C010009C479C439C478297232A0400004023208E
:10C0200004007DB71763FFFFE702630B835725000A
:10C0300041112EC681EB0144228541011763FFFFA8
:10C040006700230C035705008147F146E305F7FE1F
:10C05000B385D702404585072E948345440008C424
:10C06000F5F5B247AA8481E7232A040009A81C45F4
:10C070006C0022859C439C43829748C84DDD8547D0
:10C080002312F400B24723200400231804002319CC
:10C09000F4005C485CC483D72400FD172391F400AE
:10C0A00061BF1763FFFFE702830397A7FF1F938713
:10C0B00067CA8843232605002324050041059710FD
:10C0C0000100E78000B31763FFFF67008303176376
:10C0D000FFFFE702C30017A4FF1F1304A4C71C40FF
:10C0E000411199CF9C472300B5002AC65CC1970037
:10C0F0000000E78040FB1C40DC4399C33245829737
:10C1000041011763FFFF6700C3FF0347450029E3B1
:10C11000584DAA877D551DCF1763FFFFE70223FC0B
:10C120001CC3DC4797A6FF1F23A6E6C2F1561305E2
:10C1300007012390D700970500009385050297100B
:10C140000100E780A09801451763FFFF670063FBCC
:10C150007D55828082801763FFFFE70243F801115B
:10C160006146814528009760FFFFE78040FA97A766
:10C17000FF1F938727BE9C4328009305F00FDC47E1
:10C180003EC697000000E780C0F405611763FFFF1B
:10C19000670023F797A7FF1F9387C7BB9C43D84728
:10C1A000A1679387C702631EF70A397106DE22DC96
:10C1B00026DA80004AD84ED652D456D23285B2847E
:10C1C00097000000E780C0C7AA8926859700000075
:10C1D000E78020C92318A4FC268597000000E7808B
:10C1E00040C82319A4FC268597000000E78060C79B
:10C1F00083D744000A8A231AA4FC858393F7F70F98
:10C20000230EF4FC8607BD0793F7073F3301F14087
:10C210008A8A01498347C4FD6367F902CE85130505
:10C2200084FC232C54FD97000000E78080EA5281B3
:10C23000130104FCF2506254D2544259B259225AAA
:10C24000925A21618280268597000000E78060C1B4
:10C2500093171900D69705092390A7001379F90FB2
:10C2600055BF828097A7FF1F9387C7AE9C43D847CF
:10C27000A1679387A702631AF70A397106DE22DCE9
:10C2800026DA80004AD84ED652D456D23285B284AD
:10C2900097000000E780C0BAAA89268597000000B1
:10C2A000E78020BCFD572318A4FC26852319F4FC45
:10C2B00097000000E780E0BA83D744000A8A231A77
:10C2C000A4FC858393F7F70F230EF4FC8607BD07C4
:10C2D00093F7073F3301F1408A8A01498347C4FD40
:10C2E0006367F902CE85130584FC232C54FD970067
:10C2F0000000E78000DE5281130104FCF25062541A
:10C30000D2544259B259225A925A216182802685CA
:10C3100097000000E780E0B493171900D69705094D
:10C320002390A7001379F90F55BF828097A7FF1FAD
:10C33000938747A29C43D847A16789076310F70AF0
:10C34000397106DE22DC26DA80004AD84ED652D475
:10C3500056D23285328997000000E78060AEAA8904
:10C360004A8597000000E780C0AF835749000A8ADA
:10C370002318A4FC858393F7F70F230CF4FC86079E
:10C38000BD0793F7073F3301F1408A8A8144834711
:10C3900084FD63E7F402CE85130584FC232A54FD53
:10C3A00097000000E780E0D25281130104FCF250B4
:10C3B0006254D2544259B259225A925A216182800F
:10C3C0004A8597000000E780C0A993971400D6978C
:10C3D00085042390A70093F4F40F55BF828097A79C
:10C3E000FF1F938727979C43D847A1679387E7044C
:10C3F000631EF70A397106DE22DC26DA80004AD88D
:10C400004ED652D456D23285B28497000000E780CF
:10C4100020A3AA89268597000000E78080A423181E
:10C42000A4FC268597000000E780A0A3231AA4FCA3
:10C43000268597000000E780C0A283D744000A8ABF
:10C440002319A4FC858393F7F70F230EF4FC8607CA
:10C45000BD0793F7073F3301F1408A8A01498347BB
:10C46000C4FD6367F902CE85130584FC232C54FDBB
:10C4700097000000E780E0C55281130104FCF250F0
:10C480006254D2544259B259225A925A216182803E
:10C49000268597000000E780C09C93171900D69767
:10C4A00005092390A7001379F90F55BF828097A73C
:10C4B000FF1F9387278A9C43D847A1679387C704A8
:10C4C000631AF70A397106DE22DC26DA80004AD8C0
:10C4D0004ED652D456D23285B28497000000E780FF
:10C4E0002096AA89268597000000E7808097FD574F
:10C4F0002318A4FC2685231AF4FC97000000E7808B
:10C50000409683D744000A8A2319A4FC858393F7B5
:10C51000F70F230EF4FC8607BD0793F7073F33019F
:10C52000F1408A8A01498347C4FD6367F902CE85D9
:10C53000130584FC232C54FD97000000E78060B9AC
:10C540005281130104FCF2506254D2544259B25940
:10C55000225A925A21618280268597000000E78046
:10C56000409093171900D69705092390A7001379D7
:10C57000F90F55BF82809797FF1F9387A77D9C4334
:10C58000D847A167DD076317F7041763FFFFE702CA
:10C5900003B579713285328497000000E780408AC4
:10C5A0002AC6228597000000E780A08B2311A102F4
:10C5B000228597000000E780A088B2452300A102F1
:10C5C000280897000000E780C0B045611763FFFFAF
:10C5D000670023B382809797FF1F9387A7779C43B9
:10C5E000D847A167938787046317F7041763FFFF92
:10C5F000E702E3AE79713285328497000000E7806C
:10C6000020842AC6228597000000E78080852311B8
:10C61000A102228597000000E7808082B2452300B6
:10C62000A102280897000000E780A0AA45611763CF
:10C63000FFFF670003AD82809797FF1F9387877185
:10C640009C43D847A1679387A7046312F702176337
:10C65000FFFFE702C3A801112800814597000000F1
:10C66000E78020A705611763FFFF670083A9828029
:10C670009797FF1F9387076E9C43D847A1679387BF
:10C6800057026319F7021763FFFFE70243A5011181
:10C69000328597F0FFFFE780A07A2308A10081454B
:10C6A000280097000000E780C0A205611763FFFF24
:10C6B000670023A582809797FF1F9387A7699C43F4
:10C6C000D847A1679387E702631BF7041763FFFF4F
:10C6D000E702E3A001113285328497F0FFFFE78083
:10C6E0004078AA84228597F0FFFFE780807785470E
:10C6F00009E9228597F0FFFFE78080744205B33790
:10C70000A00028008145231891003ECA9700000030
:10C71000E780209C05611763FFFF6700839E82808E
:10C720009797FF1F938707639C43D84799476313E5
:10C73000F7081763FFFFE702839A79713285328425
:10C7400097F0FFFFE780C06F2AC6228597F0FFFFB2
:10C75000E78020712310A102228597F0FFFFE78078
:10C76000206E2301A102228597F0FFFFE780406D34
:10C77000A301A102228597F0FFFFE780606C2302EE
:10C78000A102228597F0FFFFE780806B2313A102AF
:10C79000228597F0FFFFE780A06AB2452314A1022B
:10C7A000280897000000E780C09245611763FFFFEB
:10C7B0006700239582809797FF1F9387A7599C4313
:10C7C000D847A1679387C7036313F7081763FFFF71
:10C7D000E702E39079713285328497F0FFFFE780BA
:10C7E00020662AC6228597F0FFFFE7808067231026
:10C7F000A102228597F0FFFFE780A0662311A10226
:10C80000228597F0FFFFE780A0632302A102228523
:10C8100097F0FFFFE780C062A302A102228597F094
:10C82000FFFFE780E0612303A102228597F0FFFF6D
:10C83000E7800061B245A303A10228089700000029
:10C84000E780208945611763FFFF6700838B828043
:10C850001763FFFFE702A38801112A8497F0FFFF07
:10C86000E780005EAA84228597F0FFFFE780605F83
:10C87000228597F0FFFFE780C05E035744008D4795
:10C8800063F7E700228597F0FFFFE780805D228550
:10C8900097F0FFFFE780E05C2800A6859700000086
:10C8A000E780208305611763FFFF67008385979703
:10C8B000FF1F9387274A9C43D847A167FD07631F43
:10C8C000F7001763FFFFE7028381328597000000BE
:10C8D000E78040F81763FFFF6700A3828280979785
:10C8E000FF1F938727479C43D847A167E507631538
:10C8F000F7081753FFFFE702837E79713285328490
:10C9000097F0FFFFE780C0532AC6228597F0FFFF0C
:10C91000E7802055228597F0FFFFE78080542310A1
:10C92000A102228597F0FFFFE780A05352055181B5
:10C930002311A10222852302010297F0FFFFE78065
:10C940002050A302A102228597F0FFFFE780404F0D
:10C950002303A102228597F0FFFFE780604EB245D6
:10C96000A303A102280897F0FFFFE78080764561C6
:10C970001753FFFF6700E37882809797FF1F938725
:10C98000673D9C43D847A1679387E703631FF70080
:10C990001753FFFFE702A374328597000000E7807A
:10C9A00060EB1753FFFF6700C37582809797FF1FE7
:10C9B0009387473A9C43D847A16793874704631EF0
:10C9C000F7021753FFFFE7028371797132853284D2
:10C9D00097F0FFFFE780C0462AC6228597F0FFFF49
:10C9E000E7802048B245280897F0FFFFE780606E97
:10C9F00045611753FFFF6700C37082809797FF1F41
:10CA0000938747359C43D847A16793878702631074
:10CA1000F7041753FFFFE702836C79713285328484
:10CA200097F0FFFFE780C0412AC6228597F0FFFFFD
:10CA3000E7800041B2452300A102280897F0FFFFDC
:10CA4000E780206945611753FFFF6700836B828091
:10CA50001753FFFFE702A368011197F0FFFFE7807C
:10CA6000203EAA85280097F0FFFFE78080660561D9
:10CA70001753FFFF6700E3689797FF1F9387872D82
:10CA80009C43D847A167D107631FF7001753FFFFE7
:10CA9000E702E364328597000000E780A0FB1753AC
:10CAA000FFFF6700036682809797FF1F9387872A9F
:10CAB0009C43D847A167C507631FF7001753FFFFC3
:10CAC000E702E361328597000000E780A0F8175382
:10CAD000FFFF6700036382809797FF1F9387872775
:10CAE0009C43D847A167B907631FF7001753FFFF9F
:10CAF000E702E35E328597000000E780A0F5175358
:10CB0000FFFF6700036082809797FF1F938787244A
:10CB10009C43D847A167AD07631FF7001753FFFF7A
:10CB2000E702E35B328597000000E780A0F217532D
:10CB3000FFFF6700035D82809797FF1F9387872120
:10CB40009C43D84789476318F7021753FFFFE70252
:10CB500003590111328532C897F0FFFFE780402E5C
:10CB6000AA85280097F0FFFFE780A05605611753BC
:10CB7000FFFF6700035982809797FF1F9387871DE8
:10CB80009C43D847A1678D076311F7041753FFFF34
:10CB9000E702E35401113285328497F0FFFFE7800A
:10CBA000202A13066100AA844C00228597300000D9
:10CBB000E780C0232800A68597F0FFFFE78060513B
:10CBC00005611753FFFF6700C35382809797FF1FCC
:10CBD000938787189C4381CFDC4391CB1753FFFF8A
:10CBE000E702E34F82971753FFFF6700835182806C
:10CBF0001753FFFFE702A34E79713C08AE843ED283
:10CC0000A165B7070A002A843ED448103C08DD0518
:10CC10003ED636C432C63AC297D0FFFFE780402CDA
:10CC200012474810BA8597F0FFFFE780C0133246DD
:10CC30004810B28597F0FFFFE780E014A246481045
:10CC4000B68597F0FFFFE78000125010014781463C
:10CC5000A685228597D0FFFFE780E04D45611753F9
:10CC6000FFFF6700034A1753FFFFE7024347011125
:10CC70007C000329C501AE843ECAA165B707070041
:10CC80002A843ECC48087C00C5053ECE97D0FFFFE5
:10CC9000E78000258345D900480897F0FFFFE7802B
:10CCA000800C500801478146A685228597D0FFFF5A
:10CCB000E780604805611753FFFF670083441753FF
:10CCC000FFFFE702C34183C7950093F7F707A384EB
:10CCD000F50097000000E78040F91753FFFF670059
:10CCE00043421753FFFFE702833F79713C08AE844C
:10CCF0003ED2A165B70709002A843ED448103C08FB
:10CD0000938545043ED632C636C497D0FFFFE780F0
:10CD1000201DA2464810B68597F0FFFFE780A004CB
:10CD200032464810B28597F0FFFFE780C0055010EB
:10CD300001478146A685228597D0FFFFE780A03F67
:10CD400045611753FFFF6700C33B1753FFFFE7021F
:10CD5000033983C7950041112A8493F7F707A38409
:10CD6000F50032852EC697F0FFFFE780800F8567BC
:10CD70002AC46370F50297700000E78020E922461C
:10CD8000B24509ED11478146228597000000E780F2
:10CD900060E641011753FFFF6700A3360147834652
:10CDA000F501DDB71753FFFFE702C33101113C0066
:10CDB0003ECAB7070A003ECC3C003ECE83C7950072
:10CDC000AA89328593F7F707A384F5002E8497F09C
:10CDD000FFFFE78000098567637DF504A165AA84EC
:10CDE00093858504480897D0FFFFE780600F26856C
:10CDF00097700000E78080E12A8929E19145480881
:10CE000097F0FFFFE78020F6A685480897F0FFFF20
:10CE1000E78060F7CA85480897F0FFFFE780A0F435
:10CE2000014781465008A2854E8597D0FFFFE780D5
:10CE3000803005611753FFFF6700032C81454808C8
:10CE400097F0FFFFE78020F20349090275BF1753EF
:10CE5000FFFFE702232779711C103ECAB7070F00B6
:10CE60003ECC404D1C10AA84AE894808994532C674
:10CE700036893ECE97D0FFFFE780800632464808CD
:10CE8000B28597F0FFFFE78000EE630C0902A5452D
:10CE9000480897F0FFFFE780C0E62546CA8597203F
:10CEA0000100E78020A4500801478146CE852685F1
:10CEB00097D0FFFFE780202845611753FFFF6700E9
:10CEC000A3238355C402480897F0FFFFE780A0EB37
:10CED0000355E402814505C5854785456301F50293
:10CEE000C167FD179305F00F630BF5007D15977073
:10CEF0000000E780208E9305150093F5F50F480894
:10CF000097F0FFFFE78020E683450403480897F089
:10CF1000FFFFE78040E583451403480897F0FFFFD3
:10CF2000E78060E483552403480897F0FFFFE7801B
:10CF300080E583554403480897F0FFFFE780A0E4AD
:10CF40009DB71753FFFFE702831983C795008146FA
:10CF5000014693F7F707A384F50097000000E780E8
:10CF600040EF1753FFFF6700C3191753FFFFE70296
:10CF7000031779713E841C103ECA2E89B7070F0033
:10CF8000A1653ECCFD051C10AA84480842C03AC2E7
:10CF90003ECE36C432C697D0FFFFE78060F43246FB
:10CFA0004808B28597F0FFFFE780E0DBA24648081B
:10CFB000B68597F0FFFFE78000DD12474808BA8585
:10CFC00097F0FFFFE78020DC0248630C08029145E0
:10CFD000480897F0FFFFE780C0D21146A28597204E
:10CFE0000100E7802090500801478146CA852685C8
:10CFF00097D0FFFFE780201445611753FFFF6700BC
:10D0000043108945480897F0FFFFE78080CF8347AA
:10D0100004002300F50083471400A300F500E1B7E6
:10D020001753FFFFE702030A83C7950001112A8AFD
:10D0300093F7F707A384F5003285AE8432C697F0E4
:10D04000FFFFE78000E232462A89328597F0FFFF32
:10D05000E78000DF85676373F902AA894A859770C4
:10D060000000E780A0BA2A8419ED114781464A865C
:10D07000A685528597000000E780C0B70561175369
:10D08000FFFF670063079387E9FF93F7F70F0547F3
:10D09000E366F7FE8347F50195EB8947E380F9FEE8
:10D0A0008346F401528501474A86A6859700000011
:10D0B000E78040B4A167D90748083ECC230A0100A5
:10D0C00002CE97000000E780A0B04DBF639EE7004E
:10D0D0008947639EF90093071020231FF50097707E
:10D0E0000000E780C0B76DBF0947E39BE7FA8D47B3
:10D0F000E398F9FA228597700000E78080DF979720
:10D10000FF1F938767E49C4399E79797FF1F9387D7
:10D1100067CD9C4399C703D5040097800000E78042
:10D12000A0CE231F040022855DBF1753FFFFE70237
:10D1300003FB01113C003ECAB7070B003ECC3C008C
:10D140003ECE83C795002A89328593F7F707A384DB
:10D15000F500AE8497F0FFFFE780A0D0931705019C
:10D16000C187635AF006A1652A849385E5024808C1
:10D1700097D0FFFFE780C0D6A285480897F0FFFF51
:10D18000E78060C09797FF1F9387C7C59C43A9EBB3
:10D1900001449375F40F480897F0FFFFE780A0BCA7
:10D1A0009355844093F5F50F480897F0FFFFE7800B
:10D1B00080BB9355044193F5F50F480897F0FFFFA6
:10D1C000E78060BA014781465008A6854A8597D016
:10D1D000FFFFE78040F605611753FFFF670063F22A
:10D1E000416585460546A2857D1597500000E7807C
:10D1F00060BD59DD510597000100E780808F130461
:10D2000040063344850271B71753FFFFE70223ED51
:10D210000111B70706003EC683C7950021642A891D
:10D2200093F7F707A384F500AE8428009305A404C0
:10D230000AC40AC897D0FFFFE78080CA30000147C0
:10D240008146A6854A8597D0FFFFE780C0EE97E02C
:10D25000FFFFE780E01113049404480822CC230A5E
:10D26000010002CE97000000E78080960561175309
:10D27000FFFF670003E91753FFFFE702A3E4C16460
:10D280002A8901449799FF1F938989CD130A800247
:10D29000FD1497E0FFFFE780E0BD6347A400014570
:10D2A0001753FFFF670043E5B307440303A7C90A09
:10D2B000BA9703D707006306970083D727006384D4
:10D2C00027010504F9B70545E1BF1753FFFFE70242
:10D2D00063DF2A8A2E8999C123A0050081498144F0
:10D2E000979AFF1F938A8AA7614B97E0FFFFE78019
:10D2F000A0BE63C7A4004E851753FFFF6700C3DFBE
:10D300003384640383A70A003E948357040099E79B
:10D3100063040900232089008504C1BF4146D285EA
:10D320001305440097100100E780605975F5A28944
:10D33000E5B71753FFFFE702E3D839717C083ED405
:10D34000B7070A003ED67C083ED883C795002A8AD4
:10D35000328593F7F707A384F5002E8932C697F03C
:10D36000FFFFE78000B085676373F5083246AA8443
:10D37000328597F0FFFFE780A0AC8547AA8963E874
:10D38000A706A16593858504281097D0FFFFE78045
:10D3900020B5268597700000E78040872A8429ED14
:10D3A0009145281097F0FFFFE780E09BA6852810A5
:10D3B00097F0FFFFE780209DCE85281097F0FFFFB4
:10D3C000E780609A014781463010CA85528597D020
:10D3D000FFFFE78040D6A1679387770448183EDCBB
:10D3E000230A010202DE97F0FFFFE780607E2161E1
:10D3F0001753FFFF670043D08145281097F0FFFFC8
:10D40000E7806096A685281097F0FFFFE780A09739
:10D410009797FF1F938747EB9C4381CB22856389B6
:10D42000090097D00000E78040248345040271B7CB
:10D4300097D00000E780C022CDBF1753FFFFE7025F
:10D4400063C883C795004111AA8993F7F707A3849E
:10D45000F5003285AE84328A97F0FFFFE78060A046
:10D460008567637FF5022A8997600000E780007A6C
:10D470002A84914631C58347F50105476387E70252
:10D4800091C70D476366F704AD461DA893050503D4
:10D4900003250A00414697100100E78040420DE94C
:10D4A00041011753FFFF670023C593059508032526
:10D4B0000A00414697100100E7806040814669F507
:10D4C0004A86A6854E8597000000E780C081C9BFC7
:10D4D00083250A001305940897700000E780A029AF
:10D4E00019C1C146F1BF9797FF1F9387E7A59C43DA
:10D4F00099E79797FF1F9387E78E9C4399C72285EB
:10D5000097800000E780208A69FD8547A30FF4001B
:10D51000228597B00000E780608422859760000034
:10D52000E780E0734E8581464A86A68597F0FFFF27
:10D53000E780607BA1679387570448003EC42302BD
:10D54000010002C697F0FFFFE780806891BF175384
:10D55000FFFFE70243B683C795004111AA8993F7FD
:10D56000F707A384F50032852E89B28A97F0FFFF72
:10D57000E780208F85676374F50EAA8497600000AA
:10D58000E780C0682A840DED416B014A979BFF1F1D
:10D59000938B0B9D130C400E7D1B19A833048A033B
:10D5A00083A70B0B3E948357C40163836705050A69
:10D5B00097E0FFFFE780008BE342AAFE95460DA0AF
:10D5C0008357C501639697029305050303A50A00D7
:10D5D000414697100100E780802E994611E181466F
:10D5E0002686CA854E8597F0FFFFE780C06F85A825
:10D5F00083A50A001305040397700000E780A017B5
:10D60000C14679FD2285231E940097A00000E78083
:10D61000E074228597600000E78060649797FF1FA1
:10D62000938787CA9C43A9C323000402228597D00D
:10D630000000E78040F04E8581462686CA8597F037
:10D64000FFFFE780406AA1679387070448003EC454
:10D650002302010002C697F0FFFFE78060574101F7
:10D660001753FFFF6700A3A889472300F402E1B71F
:10D67000397106DE22DC4AD8800052D456D25AD004
:10D6800026DA4ED65ECE2E8A32892A8B97D0FFFFBD
:10D69000E780407A0605710541998A8A3301A140E5
:10D6A000232224FC231404FC97D0FFFFE78080781A
:10D6B00083479A000605350593F7F7072315A4FC61
:10D6C000A304FA004A85232624FC97E0FFFFE780A5
:10D6D000407993170501C1876340F0025681130119
:10D6E00004FCF2506254D2544259B259225A925A0E
:10D6F000025BF24B21618280AA844A8597E0FFFF9A
:10D70000E7802076AA894A8597E0FFFFE780607569
:10D71000A1659385C5022A89130544FC97C0FFFFC4
:10D72000E780007C268597C0FFFFE7804070854535
:10D7300011C94A86CE8597C0FFFFE780C069AA8BD2
:10D7400021E98945130544FC97E0FFFFE780A061CC
:10D75000A685130544FC97E0FFFFE780C062CE85F5
:10D76000130544FC97E0FFFFE780E061CA851305DD
:10D7700044FC97E0FFFFE780006101478146130604
:10D7800044FCD2855A8597D0FFFFE780C09AB9B78D
:10D790008145130544FC97E0FFFFE780C05CA68548
:10D7A000130544FC97E0FFFFE780E05DCE8513059D
:10D7B00044FC97E0FFFFE780005DCA85130544FC49
:10D7C00097E0FFFFE780205C814497D0FFFFE78070
:10D7D0006066E3D4A4FA83A70B0113971400BA97E9
:10D7E00083D5070099C5130544FC97E0FFFFE78048
:10D7F00080598504D9BF797106D622D44AD0001841
:10D800004ECE52CC56CA26D25AC8AE893289AA8A7E
:10D8100097D0FFFFE78000620605690541990A8AF3
:10D820003301A140232A24FC231C04FC97D0FFFFD2
:10D83000E780406083C7990006052D0593F7F70739
:10D84000231DA4FCA384F9004A85232E24FC97E021
:10D85000FFFFE780006193170501C187634FF00068
:10D860005281130104FDB250225492540259F249DC
:10D87000624AD24A424B45618280AA844A8597E037
:10D88000FFFFE780005EA1659385A5022A89130545
:10D8900044FD97C0FFFFE780A064268597C0FFFF87
:10D8A000E780E058854509C9CA8597C0FFFFE78032
:10D8B00080552A8B29E18945130544FD97E0FFFF38
:10D8C000E780604AA685130544FD97E0FFFFE780E7
:10D8D000804BCA85130544FD97E0FFFFE780A04A0F
:10D8E00001478146130644FDCE85568597D0FFFF3C
:10D8F000E7806084B5B78145130544FD97E0FFFFDD
:10D90000E7806046A685130544FD97E0FFFFE780AA
:10D910008047CA85130544FD97E0FFFFE780A046D6
:10D92000814497D0FFFFE780E050E3DBA4FA832730
:10D930000B0113971400BA9783D5070099C51305F7
:10D9400044FD97E0FFFFE78000448504D9BF1743FB
:10D95000FFFFE702C37883474500404DD5EFFD57F1
:10D960005DC48346940009476363D70A0346B40045
:10D97000854663EEC6088306E40063CA06085C4574
:10D98000F9562390D7009787FF1F83C7673D99E318
:10D99000A304E4009787FF1F9387C7449C4381E754
:10D9A0008947A306F4009797FF1F9387E7919C434D
:10D9B00081E789472306F400970500009385450613
:10D9C000AA841305040197F00000E7802010FD579A
:10D9D000231AF40281471CDC01489787FF1F23ADFF
:10D9E00087369787FF1F93876737232E040304C06A
:10D9F000804397D0FFFFE780204E61463306C50283
:10DA0000814522859740FFFFE780607081473E8512
:10DA10001743FFFF6700E36EFD57D5BF1743FFFFB6
:10DA2000E702E36B2A840355450297600000E78014
:10DA3000E01D19E5231E04001743FFFF6700636C18
:10DA40008357E401F5DB930504FF17450100130537
:10DA5000A5E397E00000E780E014F9BF1743FFFF5C
:10DA6000E702E3672E89A16541119385E5032A84C6
:10DA700036C432C6BE843AC297C0FFFFE780404634
:10DA800012472285BA8597E0FFFFE780C02D324616
:10DA90002285B28597E0FFFFE780E02EA24622852F
:10DAA000B68597E0FFFFE780002E630309029145EA
:10DAB000228597E0FFFFE780C0241146A6859710D6
:10DAC0000100E78020E241011743FFFF6700636325
:10DAD0008945228597E0FFFFE780A02283C70400E5
:10DAE0002300F50083C71400A300F500E9BF174326
:10DAF000FFFFE702C35E83C79500444D054793F7D8
:10DB0000F707A384F5001C42411183C70700636730
:10DB1000F7062E842A89B1C003C7D400630FF70229
:10DB20001787FF1F1307072C184305C3A386F400AC
:10DB300097A00000E780404A83C7D40099E7416579
:10DB40007D1597400000E780403083D72403918BF8
:10DB500089C797E00000E780C0134A85A28597F047
:10DB6000FFFFE7808010A167C10748003EC4230281
:10DB7000010002C697F0FFFFE780800541011743CF
:10DB8000FFFF670003581743FFFFE702435503D722
:10DB900045008D47AA8441112E8432892E8563E386
:10DBA000E70297E0FFFFE780C02BAA85230009006A
:10DBB000268597C0FFFFE780002541011743FFFF3F
:10DBC0006700235497E0FFFFE780A0292AC622853B
:10DBD00097E0FFFFE780E028B24585472A862300CB
:10DBE000F900268597C0FFFFE780E01EF9B739717D
:10DBF00006DE22DC26DA80004ED652D456D24AD82F
:10DC00005AD05ECEAE89B284AA8A97D0FFFFE78051
:10DC1000602106051305250241990A8A3301A140B6
:10DC2000232224FC231404FC97D0FFFFE780801FED
:10DC300083C7990006054D0593F7F7072315A4FC44
:10DC4000A384F9002685232624FC97E0FFFFE780C4
:10DC5000402193170501C1876340F00252811301EF
:10DC600004FCF2506254D2544259B259225A925A88
:10DC7000025BF24B21618280AA8B03AB040097C048
:10DC8000FFFFE780C01A51E583D74400014985446E
:10DC9000F11793B71700A301F4FC834734FCA16587
:10DCA000C9C79385E504130544FC97C0FFFFE780CF
:10DCB0002023A685130544FC97E0FFFFE780A00A18
:10DCC000DE85130544FC97E0FFFFE780C00B834728
:10DCD00034FC114691E30946DA85130544FC97E0CC
:10DCE000FFFFE78060058144630A0900416B7D1BEB
:10DCF00097D0FFFFE780001363CCA4020147814661
:10DD0000130644FCCE85568597C0FFFFE780A042EE
:10DD1000B1B7A685130634FC97000000E780E0E663
:10DD2000933415002A8986048DBF9385C504A5BF49
:10DD30008327C90013971400BA9783D50700638817
:10DD40006501130544FC97E0FFFFE780C0038504ED
:10DD500045B71743FFFFE702033679711C103EC435
:10DD6000B7070F003EC61C103EC883C79500AA8A9D
:10DD7000328593F7F707A384F500AE89328497E0E4
:10DD8000FFFFE780000E93170501C187635AF00675
:10DD90002A8A228597E0FFFFE780A00C2A89528516
:10DDA000032B040097C0FFFFE780600839ED83571D
:10DDB000440081440544F11793B71700A303F10011
:10DDC00083457100DA872287CA8652862800970029
:10DDD0000000E780E0C8014781463000CE855685C7
:10DDE00097C0FFFFE7802035A1679387D7034808D6
:10DDF0003ECC230A810026CE97F0FFFFE78040DD6E
:10DE000045611743FFFF6700832EA285130671004B
:10DE100097000000E78060D7AA84094455D13544B3
:10DE2000E30055FB4A8597F0FFFFE78000450D446E
:10DE300041D9014497D0FFFFE780C0FE634DA400A5
:10DE4000C16B0144FD1B97D0FFFFE780A0FD634E2F
:10DE5000A4001544B5B7DC4413171400BA9783D750
:10DE60000700638327030504F1B7D8449317140010
:10DE7000BA9703D70700631B7701239027012685F4
:10DE800097A00000E78080DB01441DBF050465BF4B
:10DE90001743FFFFE702032383C7950041112A8A36
:10DEA00093F7F707A384F50032852E89328497E033
:10DEB000FFFFE78000FB93170501C1876353F0065E
:10DEC000AA89228597E0FFFFE780A0F92311A1002E
:10DED0004E85832A040097C0FFFFE78040F539E5AF
:10DEE0008357440085440144F11793B71700A300FA
:10DEF000F1000348110003572100D6875285CE86D2
:10DF00002686CA8597F0FFFFE7806006A167F107C4
:10DF100048003EC42302910022C697F0FFFFE7802D
:10DF200020CB41011743FFFF6700031DA2851306A5
:10DF3000110097000000E78040C52A84894455D924
:10DF40008357210011678544BA97C2071167C183BF
:10DF50001307F7EFE36FF7F89787FF1F9387C7FE65
:10DF60009C4381CB85451305210097500000E78035
:10DF70002075835521002285814497C0FFFFE780EB
:10DF8000A0E125D923100500228597A00000E78095
:10DF900040CD85B71743FFFFE702E31183C7950024
:10DFA00041112A8B93F7F707A384F50032852E8A57
:10DFB000328497E0FFFFE780C0EA93170501C1872D
:10DFC0006351F006AA8A228597E0FFFFE78060E9A7
:10DFD0002A895685832B040097C0FFFFE78020E540
:10DFE00031E58357440081440544F11793B7170086
:10DFF000A301F10003483100DE875A854A87D6869F
:10E000002286D28597F0FFFFE78060F6A167ED07D3
:10E0100048003EC42302810026C697F0FFFFE78038
:10E0200020BB41011743FFFF6700630CA285130665
:10E03000310097000000E78040B5AA8409445DD90B
:10E040009167CA97C2071167C1831307F7EF0544A9
:10E05000E362F7FACA8597C0FFFFE780E0D3014487
:10E0600051F9814997D0FFFFE780C0DC63DBA9004D
:10E07000984893971900BA9703D7070005EF2390A4
:10E08000270197D0FFFFE780E0DA1544E384A9F683
:10E09000268597A00000E780C0BC9787FF1F938765
:10E0A000A7EA9C430144B9D74A8597500000E7800E
:10E0B000C05889B785097DB71743FFFFE702830082
:10E0C00079713E847C083EC82E8AB7071400A1658A
:10E0D0003ECAE5057C08AA89080836C4428932C6CA
:10E0E000BA8AC6843ECC97C0FFFFE78060DFCA854E
:10E0F000080897E0FFFFE78000C732460808B285AE
:10E1000097E0FFFFE78020C8A246630A09049D4507
:10E11000080897E0FFFFE780C0BE1D468145974095
:10E12000FFFFE780C0FE63890A089145080897E071
:10E13000FFFFE78000BD1146A68597000100E7803C
:10E14000607A100801478146D2854E8597C0FFFF4F
:10E15000E78060FE45611743FFFF6700E3F9B6857E
:10E16000080897E0FFFFE78000C21C400808D8437A
:10E170009355C701858912075183B205D98D97E060
:10E18000FFFFE78040C01C40080883C5870097E078
:10E19000FFFFE78040BD1C40080883C5A70097E04B
:10E1A000FFFFE78040BC1C40080883C5970097E04C
:10E1B000FFFFE78040BB85BF8945080897E0FFFF68
:10E1C000E78020B483C704002300F50083C7140050
:10E1D000A300F500BDB71743FFFFE702A3EE83C717
:10E1E00095004111AA8993F7F707A384F5003285BA
:10E1F000AE84328497E0FFFFE780A0C69317050145
:10E20000C187635DF0042A89032A040097C0FFFFD9
:10E21000E780E0C119E9835744000548F11793B737
:10E220001700A307F100814631A81306F100A2856B
:10E2300097000000E78060951DC51C459DC783D6EB
:10E24000470001480347F10093078500D2884A86BA
:10E25000A6854E8597000000E78040E64101174300
:10E26000FFFF670063E909487DBF1D486DBF174385
:10E27000FFFFE70223E565715C083EC4B7077B0139
:10E280003EC65C083EC883C795002A8A328593F74C
:10E29000F707A384F500AE8997E0FFFFE78040BA57
:10E2A0008357E100E1C78945280097C0FFFFE78059
:10E2B00020C38145280097E0FFFFE780C0AA97C0F0
:10E2C000FFFFE78000C99787FF1F9387E7FF9C4305
:10E2D0001784FF1F0344C4A8AA843334800099C361
:10E2E000136424009787FF1F9387C7AF9C4399C38C
:10E2F000136444009787FF1F938707C59C4399C306
:10E300001364840083D504002800014997E0FFFFCF
:10E31000E78060A783D52400280097E0FFFFE7800F
:10E3200080A683D54400280097E0FFFFE780A0A5E2
:10E3300097D0FFFFE78000AB93150501C18128004E
:10E3400097E0FFFFE78020A4A285280097E0FFFF69
:10E35000E78060A39C446360F90201478146300076
:10E36000CE85528597C0FFFFE780E0DC59611743F7
:10E37000FFFF670063D8DC441314490028003E9473
:10E3800097E0FFFFE780609683474400034754000F
:10E3900089070607BA978607E36AF5FC83552400C8
:10E3A0002800814A97E0FFFFE780E09D8345440015
:10E3B000280097E0FFFFE780009B8345540028007A
:10E3C00097E0FFFFE780209A8347440063C9FA0083
:10E3D000814A8347540063C1FA020509A5BF1C4462
:10E3E00013975A002800BA9783D50700850A97E04B
:10E3F000FFFFE7804099C9BF032BC40093975A00E1
:10E4000028003E9B83552B00850A97E0FFFFE7809D
:10E41000809783550B00280097E0FFFFE780A096C8
:10E420004DBF1743FFFFE70283CB5C4993E717001B
:10E430005CC997A00000E78020B61743FFFF670084
:10E4400043CC1743FFFFE70283C92E84814597F031
:10E45000FFFFE780C0E705C583570500FD172310C0
:10E46000F50009C4835725002310F400970000002D
:10E47000E78060FB01451743FFFF670083C8314514
:10E480007DD823100400C5BF1743FFFFE70283C3F5
:10E4900083C7950041112A8A93F7F707A384F500F3
:10E4A00032852E89328497E0FFFFE780809B9317A7
:10E4B0000501C1876356F006AA89C145228597E008
:10E4C000FFFFE780A0802A8B4E85832A040097C037
:10E4D000FFFFE780C09531E9835744002311010015
:10E4E0000544F11793B71700A300F10081440348D6
:10E4F000110003572100D6875285CE862286CA8511
:10E5000097F0FFFFE780A0A6A16793871702480056
:10E510003EC42302810026C697E0FFFFE780406BE0
:10E5200041011743FFFF670023BD13061100A285B9
:10E5300097F0FFFFE7806065AA8409E523110100D9
:10E54000094475B7930521005A8597000000E780BC
:10E5500080EF835721002A84D9DB9787FF1F938799
:10E56000A79E9C4381CB8545130521009750000051
:10E57000E7800015835521002685314497C0FFFFB1
:10E58000E78080812DD52310050026859790000017
:10E59000E780206D0144A1BF1743FFFFE70223B4CA
:10E5A00041112E896C00AA8402C697F0FFFFE78014
:10E5B00000D20DC10357050005072310E5009700A1
:10E5C0000000E78040E681473E8541011743FFFF99
:10E5D000670023B33247954765DBCA8526859730A8
:10E5E0000000E780400DC147E34005FE3244854707
:10E5F00041462310F40083570900A6851305440003
:10E600002311F40097000100E780C02D228545BF4B
:10E610001743FFFFE70203AB83C795004111AA8AA6
:10E6200093F7F707A384F5003285AE89328497E02B
:10E63000FFFFE780008393170501C1876356F0064B
:10E640002A8AC145228597D0FFFFE7802068AA84E7
:10E650005285032B040097B0FFFFE780407D31E92E
:10E6600083574400231101008544F11793B7170025
:10E67000A300F10001440348110003572100DA8789
:10E680005685D2862686CE8597F0FFFFE780208EBE
:10E69000A1679387070248003EC42302910022C667
:10E6A00097E0FFFFE780C05241011743FFFF67007B
:10E6B000A3A4A2851306110097F0FFFFE780E04CAA
:10E6C0002A8409E523110100894475B7268593053D
:10E6D000210097000000E78060ECAA8449FD835583
:10E6E0002100228597B0FFFFE780006B49F50149C3
:10E6F00097C0FFFFE7800074635DA9001848931777
:10E700001900BA9703D707000DEF03572100239094
:10E71000E70097C0FFFFE780E07163062503978756
:10E72000FF1F938767829C4399C703552100975029
:10E730000000E78080F0228597900000E78060521B
:10E740001DBF050975B795443DB705C19307F00F87
:10E75000630FF500C547630CF5009307F5FF05450A
:10E760003315F50042054181828001458280416573
:10E770007D158280B9E91743FFFFE7024396034501
:10E780000603328497000000E78060FC9305803E1A
:10E79000B305B502C205C18181CD0357E4028547A7
:10E7A00063F8E7001305040197E00000E7802042CA
:10E7B0008357E40241677D176385E700FD17231740
:10E7C000F4021743FFFF6700C39382801743FFFFE4
:10E7D000E702638E004283C79500444D034914004D
:10E7E00093F7F707A384F500834704002209116714
:10E7F0003369F900A167B347F90041112A8BAE8A4A
:10E8000063ECE70E834724001307C00EB91793F794
:10E81000F70F6373F71003473400C14763EEE70E49
:10E82000834744001307E00793C707086371F70C99
:10E830008349840083477400A209B3E9F90085671E
:10E8400063F7F90A034A6400834754004E85220A9D
:10E85000336AFA0097500000E780403B61C123967D
:10E860002403834B3400137AFA00239A3403238859
:10E8700074032399440393890401631C090023A6AC
:10E880000402239804024E8597E00000E78060367A
:10E890003DA0034924004A8597000000E78020EB53
:10E8A0002397A402834744004E85A388F402E38D96
:10E8B0000BFCE30B09FC97E00000E780202F97900A
:10E8C0000000E780007381460146D6855A8597E0AF
:10E8D000FFFFE7800058A167938797033EC4230298
:10E8E0000100480002C697E0FFFFE780602E41016B
:10E8F0001733FFFF6700A37F8544A2862686D6854F
:10E900005A8597E0FFFFE780C054A167938797037C
:10E910003EC423029100F1B7BD44C5B79144F1BF95
:10E920001733FFFFE702037A01111C08404D3EC276
:10E93000B7070F003EC41C083EC62A89AE8997C09F
:10E94000FFFFE78000D7585C1C5C6346B70E6394FA
:10E95000E50063E2A70E3385A740B3B7A700B30570
:10E96000B7401306803E81469D8D97000100E780E9
:10E9700080B793140501C180A1659385C503480044
:10E9800097B0FFFFE780C0558145480097D0FFFF53
:10E99000E780603D83550404480097D0FFFFE7807F
:10E9A000803E83552404480097D0FFFFE780A03DB8
:10E9B000814589CCC167FD179305F00F6388F4008A
:10E9C000268597500000E780E0E0AA85480097D0B0
:10E9D000FFFFE780403903554404814501CDC167FD
:10E9E000FD179305F00F6307F50097500000E780CF
:10E9F00060DEAA85480097D0FFFFE780C0368345D8
:10EA00006404480097D0FFFFE780E0358345740435
:10EA1000480097D0FFFFE78000355000014781464E
:10EA2000CE854A8597B0FFFFE780E0700561173318
:10EA3000FFFF6700636C814481B71733FFFFE70274
:10EA4000036A83C7950093F7F707A384F50097003F
:10EA50000000E78020ED1733FFFF6700836A17335C
:10EA6000FFFFE702236683C795004111404D93F7EE
:10EA7000F707A384F5002A8A3285B284AE8997D03D
:10EA8000FFFFE780003E2A8B268597D0FFFFE780B7
:10EA9000403D2A89268597D0FFFFE780603A93178B
:10EAA0000B0163CA0702E177CA97C207C1831167E6
:10EAB00063E3E70293070910C207C1831307B00F8E
:10EAC000637BF70093170901C187AA8A634AF000A4
:10EAD000C54763FE570141011733FFFF6700C3615C
:10EAE00097B0FFFFE7802025E31725FFD5B7630820
:10EAF0000B0263060902814463890A02B7077F009B
:10EB000023106405231124057CC05685970000005E
:10EB1000E780E0C39304803EB304950239A0B707B1
:10EB20007F00232004047CC081440355240497E023
:10EB30000000E780A0A3A1C497C0FFFFE78060B7F3
:10EB4000269593D7F44133379500AE97BA9708DCF2
:10EB50005CDCCE85528597000000E780A0DC99E060
:10EB600023220404A1679387B70348003EC423020D
:10EB7000010002C697E0FFFFE7808005A9BF81473B
:10EB800001481CDC232E0403E9B71733FFFFE7021B
:10EB9000035597C0FFFFE7802034E1473305F502B6
:10EBA000914597500000E78000C5E55711C597775C
:10EBB000FF1F23A5A71A81473E851733FFFF670074
:10EBC000435485471777FF1F230CF71882801733AC
:10EBD000FFFFE702C3509777FF1F9387E717804334
:10EBE0003DC0835704046390A70683572404639CA5
:10EBF000B7043689B28497C0FFFFE78080AB5C5CC6
:10EC000063C3B7046395B7001C5C63EEA702834738
:10EC1000640463F3F400A6872303F40483477404B5
:10EC200063F39700A687A303F40483574404416762
:10EC30007D176385E70085072312F4043C4481C7F0
:10EC4000CA85268582971733FFFF6700834B977726
:10EC5000FF1F938767109C43014599C303C5870035
:10EC600082801733FFFFE70283470111B7070700D0
:10EC70003EC683C79500584D0AC493F7F7070AC8E4
:10EC8000A384F5002A89AE8411CB1C4283C70700F8
:10EC90002304F70097900000E78000342164930577
:10ECA0005402280097B0FFFFE78080239700000000
:10ECB000E78020FAAA85280097D0FFFFE780A00A06
:10ECC000300001478146A6854A8597B0FFFFE7805F
:10ECD000804613044402480822CC230A010002CED5
:10ECE00097E0FFFFE780C0EE05611733FFFF670085
:10ECF00043411733FFFFE702833E01117C003ECA08
:10ED0000B70707003ECC7C003ECE83C795002E841B
:10ED1000AA8493F7F707A384F500A16593855502AC
:10ED2000480897B0FFFFE780A01B97000000E7802E
:10ED300040F2AA85480897D0FFFFE780C00250083C
:10ED400001478146A285268597B0FFFFE780A03E58
:10ED500005611733FFFF6700C33A9777FF1F93875B
:10ED6000A7FF9C43094599C303C597008280977705
:10ED7000FF1F938767FE9C43094599C303C5D700CE
:10ED800082809777FF1F938727FD9C43014599C396
:10ED900003C5A70082801733FFFFE702A3320111EA
:10EDA000B70708003EC683C79500404D0AC493F7D5
:10EDB000F7070AC8A384F5002A89AE8429C414423F
:10EDC000854703C7060063E0E70A834794000946C6
:10EDD00081496380C702B307F740A304E400B33955
:10EDE000F00083C716002305F40097900000E78029
:10EDF000A01E03572403058B19C76386090097D00B
:10EE00000000E78000E9216493058402280097B0A0
:10EE1000FFFFE780E00C97000000E78040F4AA8540
:10EE2000280097D0FFFFE78000F497000000E780FC
:10EE300080F5AA85280097D0FFFFE780C0F2014740
:10EE400081463000A6854A8597B0FFFFE780A02E57
:10EE500013047402480822CC230A010002CE97E072
:10EE6000FFFFE780E0D605611733FFFF6700C32887
:10EE70001733FFFFE702A32601117C003ECAB70744
:10EE800008003ECC7C003ECE83C795002E84AA8429
:10EE900093F7F707A384F500A165938585024808D9
:10EEA00097B0FFFFE780C00397000000E78020EBEA
:10EEB000AA85480897D0FFFFE780E0EA97000000A6
:10EEC000E78060ECAA85480897D0FFFFE780A0E9BB
:10EED000500801478146A285268597B0FFFFE7804D
:10EEE000802505611733FFFF6700A3219777FF1F78
:10EEF000938787E69C43014599C303C5B700828089
:10EF00001733FFFFE702A31D0111B70707003EC635
:10EF100083C79500404D0AC493F7F7070AC8A38436
:10EF2000F5002A89AE8405C81C42054783C707003F
:10EF30006368F7060347B400630FF700A305F40006
:10EF400097900000E78040098347B400B9CF97D07D
:10EF5000FFFFE78040BE21649305B400280097B00E
:10EF6000FFFFE780E0F797000000E78060F8AA85E0
:10EF7000280097D0FFFFE78000DF0147814630007F
:10EF8000A6854A8597B0FFFFE780E01A2904480864
:10EF900022CC230A010002CE97E0FFFFE78040C3A6
:10EFA00005611733FFFF6700C31597D0FFFFE780A8
:10EFB00020BF55B71733FFFFE702631201117C0032
:10EFC0003ECAB70707003ECC7C003ECE83C7950003
:10EFD0002E84AA8493F7F707A384F500A165AD05F5
:10EFE000480897B0FFFFE780A0EF97000000E78098
:10EFF00020F0AA85480897D0FFFFE780C0D65008C8
:10F0000001478146A285268597B0FFFFE780A012C1
:10F0100005611733FFFF6700C30E9777FF1F9387C4
:10F02000A7D39C43094599C303C5C7008280173302
:10F03000FFFFE702C30A01117C00AE843ECAA1654E
:10F04000B70707002A843ECCD1057C0048083ECE95
:10F0500097B0FFFFE780C0E897000000E78020FC42
:10F06000AA85480897D0FFFFE780E0CF5008014706
:10F070008146A685228597B0FFFFE780C00B05611A
:10F080001733FFFF6700E3071733FFFFE70223058E
:10F0900083C7950093F7F707A384F5009700000056
:10F0A000E78020F91733FFFF6700A3051733FFFF41
:10F0B000E702430183C795000329C501411193F776
:10F0C000F707A384F5001C4283C90700854763E660
:10F0D00037079777FF1F9387271F9C432E84AA84A7
:10F0E00085CF97000000E78080F389476306F5022B
:10F0F000630409028347C90063803703230639018B
:10F1000097900000E78040ED83572903898B89C7DA
:10F1100097D00000E780E0B72685A2859700000021
:10F12000E78020F1A167CD0748003EC4230201001B
:10F1300002C697E0FFFFE780A0A941011733FFFF58
:10F14000670083FB9777FF1F938707C19C431D458B
:10F1500099C303C5E70082801733FFFFE70223F856
:10F160000111B70707003EC683C79500584D0AC472
:10F1700093F7F7070AC8A384F5002A89AE8415C758
:10F180001C4283C7070093968701E18663C4060685
:10F1900085466381D7068346E7006388F600230728
:10F1A000F70097900000E78020E321649305E400D6
:10F1B000280097B0FFFFE780A0D297000000E7800B
:10F1C000A0F8AA85280097D0FFFFE780C0B90147C3
:10F1D00081463000A6854A8597B0FFFFE780A0F5FD
:10F1E0003504480822CC230A010002CE97E0FFFF35
:10F1F000E780009E05611733FFFF670083F0173338
:10F20000FFFFE702C3ED01117C003ECAB70707000C
:10F210003ECC7C003ECE83C795002E84AA8493F713
:10F22000F707A384F500A165B905480897B0FFFF6B
:10F23000E78000CB97000000E78000F1AA8548082E
:10F2400097D0FFFFE78020B2500801478146A28592
:10F25000268597B0FFFFE78000EE05611733FFFFBB
:10F26000670023EA1733FFFFE702C3E5AA840144DE
:10F270001779FF1F130989AEE14997C0FFFFE780A7
:10F28000A0C56344A400014519A8330534038327AE
:10F2900009003E95835725006397970011051733A2
:10F2A000FFFF670063E50504C9BF032E8500630AFD
:10F2B0000E121773FF1F130323C9032303006315E3
:10F2C000030029436390061203234E0163150300D4
:10F2D0001D43639907101733FFFFE702C3DDC6899B
:10F2E000428A3E89BA8AB684328BAE8B2A84B5E1D3
:10F2F00003554E0019E501431A851733FFFF6700D8
:10F3000003DFA167A98F116763FBE7009700000087
:10F31000E78080F5814597F0FFFFE780C012084441
:10F32000B70700E05841F98F18455CC1B707001FC7
:10F33000F98F1CC55C4991C7610597E00000E78023
:10F34000408BE38A09FA228597900000E78060C627
:10F350005DB7328597C00000E78040430D4349DD2B
:10F360001C44116703D54700A167A98F63FBE70021
:10F3700097000000E78040EF814597F0FFFFE780AE
:10F38000800C0323840093164B01D1828347B30082
:10F39000035663008588FD8BA305F300FD777D8E02
:10F3A000558EFD76FD16B204F18E83274301C58E7E
:10F3B000231273012313D3002304530123052301D4
:10F3C000A3044301BDDF228597B0FFFFE78080C91A
:10F3D000AA850844B5D1610597D00000E780207F59
:10F3E0008DB71D431A8582801733FFFFE70283CD57
:10F3F0000569AA84AE89328A0144FD5A7D1997C0F5
:10F40000FFFFE78020A26347A40001451733FFFFF9
:10F41000670083CED84493171400BA9703D7070028
:10F42000631F37032390570163070A0026859790CF
:10F430000000E780A0809C449DC383D76700B3F79A
:10F440002701639E3701D2880148814701478146E1
:10F4500001468145268597000000E78040E50504C8
:10F4600079BF1733FFFFE702E3C579711C103EC473
:10F47000B7070F003EC61C103EC883C79500AA8A76
:10F48000328593F7F707A384F5002E89328497D04D
:10F49000FFFFE780009D93170501C187635AF006BF
:10F4A000AA89228597D0FFFFE780A09B2A8A4E85F4
:10F4B000032B040097B0FFFFE780609739ED835777
:10F4C000440081440544F11793B71700A303F100EA
:10F4D00083457100DA872287D2864E86280097E01E
:10F4E000FFFFE780E057014781463000CA85568517
:10F4F00097B0FFFFE78020C4A1679387F703480810
:10F500003ECC230A810026CE97D0FFFFE780406CD7
:10F5100045611733FFFF670023BEA2851306710004
:10F5200097E0FFFFE7806066AA84094455D15285C1
:10F5300097E0FFFFE78060D40D4459D90546D28596
:10F54000268597000000E78060EA2A8451B71733C8
:10F55000FFFFE702C3B883550700034627004111A8
:10F560002A842E8532C62EC497E0FFFFE780E0D0C4
:10F5700001C93246A245228597000000E78000E7D6
:10F5800041011733FFFF6700C3B71733FFFFE702DF
:10F5900083B283C795004111AA8A93F7F707A38422
:10F5A000F5003285AE89328497D0FFFFE780608B0B
:10F5B00093170501C1876357F00AC1452A8A22853E
:10F5C00097C0FFFFE78080702A8D228597D0FFFFCC
:10F5D000E78020892A89228597D0FFFFE78040862F
:10F5E000930705F893F7F70F1307E007AA8B637BE0
:10F5F000F706228597D0FFFFE78080842A8C22853A
:10F6000097D0FFFFE780C083AA8C5285032B0400AC
:10F6100097B0FFFFE780A08139E9835744002311A9
:10F6200001008144F11793B71700A300F1000544CE
:10F630000347110083562100938784005685DA889A
:10F6400022885286CE8597F0FFFFE78020A7A1672A
:10F65000E90748003EC42302810026C697D0FFFF79
:10F66000E780005741011733FFFF670043A81306E7
:10F670001100A28597E0FFFFE7802051AA8409E5E9
:10F680002311010009446DB7930521006A8597F0A5
:10F69000FFFFE780A0F02A8441FD835521009356A7
:10F6A000C9001316490185486688E2875E87858A06
:10F6B0005182268597000000E78060BF2A848DBFB5
:10F6C0001733FFFFE702239F83C7950041112A8B61
:10F6D00093F7F707A384F5003285AE89328497C08B
:10F6E000FFFFE780007893170501C1876352F00A96
:10F6F0002A8A228597C0FFFFE780A076AA8A228502
:10F7000097C0FFFFE780E0752A89228597C0FFFF39
:10F71000E7800073930705F893F7F70F1307E007E7
:10F720002A8C6377F706228597C0FFFFE780407138
:10F73000AA8C228597C0FFFFE78080702A8D5285B2
:10F74000832B040097A0FFFFE780606E39E58357A5
:10F75000440085440144F11793B71700A301F10059
:10F7600003473100930784005A85DE882688D686B1
:10F770005286CE8597F0FFFFE78040948D47480082
:10F780003EC42302910022C697D0FFFFE780404489
:10F7900041011733FFFF67008395A28513063100EF
:10F7A00097E0FFFFE780603E2A84894455D993564D
:10F7B000C9001316490185486A88E6876287858AE9
:10F7C0005182D68597000000E78060AEAA8449BFC9
:10F7D0001733FFFFE702038F2A8981440144617ACE
:10F7E000916A176BFF1F130B2B7697B0FFFFE78013
:10F7F000606463C7A40022851733FFFF6700C38FCF
:10F800008327090093991400CE9703D50700330787
:10F810004501420741836364570305C103270B0079
:10F8200019C785453E8597400000E78060E983273A
:10F8300009000504CE972390070085047DB7970043
:10F840000000E78060A2832709000504CE9723907B
:10F85000070065D5814597F0FFFFE780C0BEF1BF87
:10F860001733FFFFE702038683C7950041112A8AF9
:10F8700093F7F707A384F50032852E89328497C069
:10F88000FFFFE780005E93170501C187635AF0040C
:10F89000AA89832A040097A0FFFFE780405931E539
:10F8A0008357440085440144F11793B71700A3011F
:10F8B000F10003483100D68752850147CE8626865F
:10F8C000CA8597D0FFFFE780806AA167F5074800E7
:10F8D0003EC42302910022C697D0FFFFE780402F4D
:10F8E00041011733FFFF67002381A2851306310012
:10F8F00097E0FFFFE78060292A8489445DD99767F4
:10F90000FF1F938767649C4381CF044997B0FFFF33
:10F91000E7804052AA85268597400000E78040DABC
:10F920001305040197000000E780C0EA2285978054
:10F930000000E78000338144ADBF1723FFFFE702DB
:10F94000837783C795004111AA8A93F7F707A384A9
:10F95000F5003285AE8932842311010097C0FFFF84
:10F96000E780205093170501C1876354F0062A8A67
:10F97000C145228597C0FFFFE7804035AA8B52859D
:10F98000032B040097A0FFFFE780604A21E983571B
:10F99000440085440144F11793B71700A300F10018
:10F9A0000348110003572100DA875685D286268640
:10F9B000CE8597D0FFFFE780805BA1679387270202
:10F9C00048003EC42302910022C697D0FFFFE78083
:10F9D000202041011723FFFF67006371A2851306F2
:10F9E000110097E0FFFFE780401A2A8489444DD92F
:10F9F0009767FF1F9387475598433E8901CF044976
:10FA000097B0FFFFE7800043AA8526859740000056
:10FA1000E78000CB1305040197000000E78080DB3E
:10FA200097B0FFFFE780004195443DD99305210041
:10FA30005E8597F0FFFFE78060B6AA8435F11C4829
:10FA40000357210022852390E70097800000E7807C
:10FA5000402183270900A9D70355210097400000C2
:10FA6000E780A0BD35BF1723FFFFE702C36483C74C
:10FA700095004111AA8A93F7F707A384F500328510
:10FA8000AE89328497C0FFFFE780A03D9317050140
:10FA9000C1876351F0062A8A228597C0FFFFE7805D
:10FAA000403C2A895285032B040097A0FFFFE78082
:10FAB000003831E58357440085440144F11793B77A
:10FAC0001700A301F10003483100DA8756854A8701
:10FAD000D2862686CE8597D0FFFFE7804049A16772
:10FAE000F90748003EC42302910022C697D0FFFFC9
:10FAF000E780000E41011723FFFF6700435FA285E7
:10FB00001306310097E0FFFFE78020082A8489442C
:10FB10005DD99167CA97C2071167C1831307F7EFD1
:10FB20008544E362F7FA9767FF1F9387E74198439D
:10FB3000BE8B01CF044997B0FFFFE780A02FAA85B5
:10FB4000268597400000E780A0B7130504019700C1
:10FB50000000E78020C897B0FFFFE780A02D954404
:10FB60003DD11C48228581442390270197800000C5
:10FB7000E780200F83A70B00B9D74A859740000084
:10FB8000E780A0AB89B71723FFFFE70243552A841C
:10FB90004105B28497000000E780C0C311C52285EB
:10FBA00097800000E780E00B81460146A68522850C
:10FBB00097800000E780C04E1C4C89C7DC4799C382
:10FBC000228582971723FFFF6700A3539767FF1FC4
:10FBD000938787189C43014599C313850701828049
:10FBE0009767FF1F93874717884382801723FFFF7C
:10FBF000E702E34E9317C600DD8DC2054111C181B6
:10FC00002A8432C697C0FFFFE780E017324622857C
:10FC100011829375F60F97C0FFFFE780C014410172
:10FC20001723FFFF6700E34D1723FFFFE702834918
:10FC300079713C083ED2B7070C003ED43C083ED652
:10FC400083C79500AE842A8993F7F707A384F5004C
:10FC5000A16593853504481097A0FFFFE7804028F1
:10FC6000C165FD150144176AFF1F130A6A2F930A25
:10FC7000400EAE892E8B2EC697B0FFFFE780801E08
:10FC80004205931704014181C183B24563E9A7028C
:10FC9000C167FD176387F500481097C0FFFFE78035
:10FCA000800E501001478146A6854A8597A0FFFF28
:10FCB000E780604845611723FFFF6700E343330790
:10FCC000540383270A0BBA9703D6C701630A360188
:10FCD000638A3501481097000000E78060F1DA85FB
:10FCE000050451BFB285EDBF1723FFFFE702A33C18
:10FCF00079717C083EC8B70711003ECA7C083ECC2B
:10FD000083C79500AA89328593F7F707A384F50086
:10FD10002E8997C0FFFFE780C01485676378F504DC
:10FD2000A165AA848905080897A0FFFFE780401B0A
:10FD3000268597400000E78060ED133415000A0423
:10FD4000A285080897C0FFFFE780E001A6850808A4
:10FD500097C0FFFFE780200325CC014781461008AC
:10FD6000CA854E8597A0FFFFE780E03C45611723D9
:10FD7000FFFF6700C337B30754030327CA0ABA97C4
:10FD800003D70700631C970003D62700638065052F
:10FD9000080897000000E780A0E5DE8505042EC670
:10FDA00097B0FFFFE780000D4205931704014181E2
:10FDB000C183B245E3E1A7FCC167FD17E38FF5F806
:10FDC000080897C0FFFFE78000FC41BFB285F9B784
:10FDD000C165FD150144176AFF1F130A6A18930ACB
:10FDE00080022E8BAE8B65BF1723FFFFE702232F08
:10FDF00018418347170083460700A207D58FD20713
:10FE0000D1832390F50083472700034717008D45D2
:10FE1000A207D98F91832310F60097C0FFFFE780D8
:10FE2000A0E91723FFFF6700C32D1723FFFFE70299
:10FE30006329C16401441769FF1F130969129309FB
:10FE40008002FD1497B0FFFFE780C0026347A40063
:10FE500001451723FFFF6700232A33053403832757
:10FE6000C90A3E9583570500E38597FE0504D9BF6F
:10FE70001723FFFFE70203252A8AAE89B284B68AD8
:10FE800097400000E78080D819E591473E85172309
:10FE9000FFFF670063262A894E8597C00000E78030
:10FEA000E08E2A84638E0A048D476DD103570500C6
:10FEB000C547E31D47FD0347F9018546AD47E317F5
:10FEC000D7FC8347450081CF4146A6855D0597F065
:10FED0000000E780C09E814755D9AD4745BF130953
:10FEE00065012302E500CA85268597100000E7809A
:10FEF000606231C1A547E38B0AF82302040079B799
:10FF000005C183570500E39247F94146A6851905C7
:10FF100097F00000E780A09A81472DD99947BDB797
:10FF20004E8597000000E78080F02A84954739DDF0
:10FF3000130955004DBF4146A685231044012311E6
:10FF400034011305190097F00000E780A09922857D
:10FF500097800000E780A0EA81470DBF1723FFFFCD
:10FF6000E702E31779717C003ECCB7070A003ECE6A
:10FF70007C003ED083C79500B2842E8493F7F707A8
:10FF8000A384F5001306A1002A892C00268597007A
:10FF90000000E780A0E5A16528088D0597A0FFFF78
:10FFA000E78000F490408355A10003558100854609
:10FFB00097000000E78000ECAA84AA85280897C073
:10FFC000FFFFE78040DA0356A1008355810028082F
:10FFD00097000000E780C0C1300801478146A28534
:10FFE0004A8597A0FFFFE7800015854748103ED45B
:10FFF0002302910202D697D0FFFFE78060BD4561E2
:020000040001F9
:100000001723FFFF6700E30F1723FFFFE702230D0E
:1000100079717C003ECCB7070A003ECE7C003ED012
:1000200083C79500B2842E8493F7F707A384F50065
:100030001306A1002A892C00268597000000E7807E
:10004000E0DAA16528088D0597A0FFFFE78040E969
:1000500090408355A1000355810081469700000020
:10006000E78040E1AA84AA85280897C0FFFFE780BF
:1000700080CF0356A1008355810028089700000017
:10008000E78000B7300801478146A2854A8597A0DE
:10009000FFFFE780400A48102302910202D402D6F3
:1000A00097D0FFFFE780C0B245611723FFFF6700CD
:1000B00043051723FFFFE702830297000000E78054
:1000C00060DB1723FFFF6700C3039767FF1F93875A
:1000D000E7C8884382801723FFFFE7024300835766
:1000E00025004111AE842A842307B10017F5FFFFD4
:1000F000130525466C002316F10097A0FFFFE7804B
:10010000804591C4228597800000E780E0D6FD57A6
:100110002310F40013062002814513055400972094
:10012000FFFFE780C0FE41011723FFFF670063FD6B
:100130001723FFFFE70203F979717C003ECCB70774
:100140000A003ECE7C003ED083C79500AA89AE84CB
:1001500093F7F7073285A384F5001306A1002C005E
:1001600097000000E78080C8035581001144974044
:100170000000E780A0A915C50355A100014497B070
:100180000000E780A06011CD035705008357810070
:1001900045446318F700854597000000E780E0F3C9
:1001A0000144216993053900280897A0FFFFE780E3
:1001B00020D3A285280897C0FFFFE780C0BA035666
:1001C000A10083558100280897000000E78040A225
:1001D000300801478146A6854E8597A0FFFFE7803E
:1001E00080F548104AD42302810202D697D0FFFF3F
:1001F000E780009E45611723FFFF6700E3EF1723A9
:10020000FFFFE70223EC9767FF1F9387E7B42A8479
:1002100088432E8915C5035745038357C4016311CD
:10022000F7022326050223180502410597D0000096
:10023000E780209C6306090097800000E78060DB70
:1002400081449769FF1F9389A9D1130A800297B04F
:10025000FFFFE78020C263C4A4049767FF1F938752
:1002600067B89C4399C70355C40197200000E780F5
:10027000C0BD63070900228597800000E780C0A009
:100280001306400E814522859720FFFFE78020E876
:10029000FD57231EF4001723FFFF6700E3E53385B6
:1002A000440383A7C90A3E95035705008357C40139
:1002B0006317F700CA8597000000E78000E2850415
:1002C00079B71723FFFFE702E3DF83C795004111EA
:1002D000AA8993F7F707A384F5003285AE8497C007
:1002E000FFFFE78000B885676378F5042A899740A7
:1002F0000000E780A091014401CD83D70400314480
:1003000063882701854597000000E78080EF01445E
:100310004E85A2864A86A68597D0FFFFE780A09CDF
:10032000A1679387170448003EC42302810002C6D8
:1003300097D0FFFFE780C08941011723FFFF6700C7
:10034000A3DB1723FFFFE702E3D79767FF1F93871E
:10035000A7A0804329C4014597C00000E780002181
:1003600081470148C1641CDC232E040323200404BC
:100370001769FF1F1309C9BE01449309400EFD14FC
:1003800097B0FFFFE78000AE634FA400814517F5EB
:10039000FFFF1305857F97A0FFFFE780C01B172392
:1003A000FFFF670063D5330534038327090B3E95B0
:1003B0008357C50163879700854597000000E78054
:1003C00040E4050475BF9357050113D78700A38048
:1003D000F50093170501C183A1832380E5002381E4
:1003E000F500A381A50082801723FFFFE70223CF3A
:1003F0002300050083C71500A300F50083C725006F
:100400002301F50083C73500A301F50083C745002C
:100410002302F50083C75500A302F50083C76500DA
:1004200093059500A30305002303F50023040500AD
:10043000328597000000E78040F91723FFFF67002F
:1004400043CC1723FFFFE702E3C74111E9540DCD69
:1004500085CD93F9C5FF2E842A89AA84338AA90001
:10046000B7EA040063189A020D88854411CCB7E7F7
:1004700004009C5F82972AC622866C0033053901EE
:1004800097E00000E7800046268541011723FFFF23
:10049000670083C683A78A03910482979317050197
:1004A000C183A183A38EF4FE93570501238FF4FE2D
:1004B000A183238EA4FEA38FF4FE6DB763E6D5025D
:1004C0001723FFFFE702A3C1B28741113686BE851D
:1004D00036C697E00000E780E040B246410136852D
:1004E0001723FFFF6700E3C181463685828083873B
:1004F00005001387F5003D05FD8793F777088346D0
:1005000007007D158606B58FA300F5006307B700C9
:100510007D17834717009D83DDB782801723FFFF78
:10052000E702E3BBB7E7040083A7070932872A86FF
:100530003A858297133515001723FFFF670063BCC8
:1005400015C181478DC11723FFFFE70243B941461B
:1005500097E00000E780003985473E851723FFFFBD
:10056000670023BA81473E8582801DCD1723FFFF98
:10057000E702E3B6414681452A849720FFFFE780E2
:1005800000B941468145130504039720FFFFE7802A
:1005900000B80147C1672322040438C87CC8054558
:1005A0001723FFFF6700E3B50145828081473DCDFA
:1005B000B5CD1723FFFFE70283B2B2842E8913065D
:1005C000800581452A849720FFFFE78040B4CA85D3
:1005D00024C4268597000000E780C0F64146814587
:1005E00022859720FFFFE78080B23044A2852285D4
:1005F00097000000E780C0F293040401A2852685DD
:1006000097000000E780E0EEA6851305040297003E
:100610000000E78000EE228597000000E78020F5CB
:1006200085473E851723FFFF6700A3AD3E85828087
:100630001723FFFFE70203A94111E9540DCD85CD32
:1006400093F9C5FF2E842A89AA84338AA900B7EAC0
:100650000400639844030D88814411CCB7E704007B
:100660009C5F82972AC622866C003305390197E089
:100670000000E7802027268541011723FFFF670040
:10068000A3A783A78A039104829793170501C183C7
:10069000A183A38EF4FE93570501238FF4FEA1835B
:1006A000238EA4FEA38FF4FE6DB765CD1723FFFF45
:1006B000E70243A1B28411E605451723FFFF670057
:1006C000A3A32A842E890145EDD93C487848B3E696
:1006D000E700E5D69386F7FFB3B7F6007D17032A48
:1006E0004404BA9734C87CC863050A06C149130597
:1006F0000A03B38949412295637D3601B2862E866D
:10070000A68597000000E780A0DB7C40BE9464C013
:1007100065B7CE862E86CE8597000000E78040DA4A
:10072000C114D2944E9923220404A2879306040193
:1007300003C7070003C607038507318FA38FE7FEB2
:10074000E398F6FE3044A285228597000000E780FA
:1007500020DD2699C1493306994063EC9900A9DC54
:10076000A686A6851305040397000000E78040D500
:1007700079BF8147B306F4003307F600034707004B
:1007800083C5060085072D8F2380E600E39437FF9D
:100790003044A285228597000000E78060D8C1140C
:1007A0005DBF014582800DC11723FFFFE702239340
:1007B0001306800581459720FFFFE780409505459A
:1007C0001723FFFF6700E39301458280814749C5F6
:1007D000C1C51723FFFFE7028390FC4141462E84E9
:1007E000AA846399C70413860501A2878146C1457F
:1007F00003C7070003C507038507298F3305D60004
:10080000034505008506298FA38FE7FEE392B6FE18
:100810003044A285268597000000E78060D02285BD
:1008200097000000E78060F885473E851723FFFFAB
:100830006700238D138507031D8E81452295972020
:10084000FFFFE780C08C7C40130700F8130604020A
:10085000A2972388E70251BF3E8582801723FFFFBE
:10086000E702E3876D712E84B284AA859010280078
:10087000368997000000E780A0D309EDD55725A061
:1008800050400C40280097000000E78040E27DD5F2
:10089000FD142104F5F42C004A8597000000E78040
:1008A00020F3814761DD3E8551611723FFFF67001B
:1008B00043851723FFFFE702838241112EC432C60E
:1008C0002C00054697000000E78080F941011723BE
:1008D000FFFF670003831723FFFFE7024380011137
:1008E0002A842EC602C802CA02CC02CE97E00000BB
:1008F000E780C023B2462A86A28508089700000038
:10090000E78060FB1375F50F05611713FFFF6700A4
:10091000437F1713FFFFE702837C7971B2872A8434
:1009200021462308B10013051101BE853AC436C61D
:1009300097E00000E78000FBB24693059101368501
:1009400097000000E78060A82285141035460C0847
:1009500097000000E78020F62A84224701E921461B
:100960000C103A8597E00000E780C0F722854561CA
:100970001713FFFF6700E3781713FFFFE7022376E3
:100980007171AE84AA850A85328497000000E780E1
:1009900060BB11C90A86A685228597000000E78002
:1009A00020B8814711E1C5473E854D611713FFFF10
:1009B000670023751713FFFFE702636F1D712A8A13
:1009C000B289BE8435468547130511012E8CB68A3F
:1009D0003A8BC28C468D2308F10097E00000E78037
:1009E00060F010100C085285231F010097000000D2
:1009F000E780C0F82A843DEDA1476313FD08930703
:100A0000900591E0E5473546E285130511011399FC
:100A10000A012308F1001359090197E00000E7805B
:100A200060EC1357890093978A00D98F90080C08BF
:100A30005285231FF10097000000E78020F42A84EC
:100A400015E9A1E49387FA0091831379F9003EC672
:100A5000631309004149668B8144C14B854DB24700
:100A6000639F970C6A868C0033855C0197E00000D9
:100A7000E78040E7228525611713FFFF6700E366E3
:100A800093079004C9F0A547BDBF834701050947F7
:100A9000C14B2308F10083471105A58FA308F1007E
:100AA00093872400814463E1FB04014714083386E3
:100AB000E6008C08B386E400BA95DA9683C6060091
:100AC00083C505000507AD8E2300D600E390E7FE41
:100AD0004147639CE70490080C085285970000008A
:100AE000E780C0E925D181A0B3069B00BA87100832
:100AF000B305F60090083E9603C5060003460600BF
:100B000085078506298E2380C500E39277FF998F9C
:100B100090080C085285BE9497000000E78000E61C
:100B20008947014749D12A84B1B790083E960346C8
:100B300006001408BE962380C600850759BFB24739
:100B400085046387971481471808B306F70098084F
:100B50003E973386F90003470700034606008507E2
:100B6000318F2380E600E39177FF90080C085285CF
:100B700097000000E78080E05DF53546E2851305CB
:100B800011012308B10197E00000E780A0D5139779
:100B900004014183939784002183D98F10180C0896
:100BA0005285231FF10097000000E78020DD25FD1E
:100BB000814710183387F9003E9603470700034624
:100BC0000600B306FB008507318F2380E600E39221
:100BD00077FF65A81808B306F70098083E97338694
:100BE000F90003470700034606008507318F23807D
:100BF000E600E3E127FFCA87639E770990080C08A7
:100C0000528597000000E78060D711FD814798006A
:100C1000B306F700900818103E973E96034707006A
:100C2000034606008507318F2380E600E39177FFB6
:100C30003546E285130511012308B10197E0000054
:100C4000E78040CA1397040141839397840021836E
:100C5000D98F10180C085285231FF100970000004F
:100C6000E780C0D1E31105EC814710183387F90004
:100C70003E960347070003460600B306FB008507C0
:100C8000318F2380E600E3E227FFC109410BC1BB9E
:100C9000814785B79408BE9683C6060018083E971C
:100CA0002300D700850789BF638006321713FFFF33
:100CB000E702E33F59712A84BE89B28B85473546E6
:100CC000130511022E8B468C4289BA8A368A23007C
:100CD000F10297E00000E780E0C010180C102285B8
:100CE0002317010297000000E78040C9631805122E
:100CF000A147631FFC069307900563930900E5472E
:100D00003546DA851305110293140A012300F10216
:100D1000C18097E00000E780E0BC93178A0013D7FA
:100D20008400D98F90080C1022852317F1029700B8
:100D30000000E780A0C47DE1639209049307FA00F4
:100D4000BD88918391E0C144C207C183DE8C814A92
:100D50003EC6414DB24763E2FA0E6286B3854B014F
:100D6000881097E00000E78080B54DC93D557DA013
:100D700093079004E39609F8A54759B783470105FF
:100D80000947C14C2300F10283471105B3C7F9009D
:100D9000A300F10293872900814963E1FC048146A5
:100DA00018103306D7008C083387D900B6955697AC
:100DB0000347070083C5050085062D8F2300E60045
:100DC000E390D7FE41476390E70690080C10228518
:100DD00097000000E78080BA35D189A0B3863A0138
:100DE000BA871010B305F60090083E9603C50600BA
:100DF0000346060085078506298E2380C500E392F9
:100E000097FF3387EC4090080C102285BA99970021
:100E10000000E780A0B68947014741D165611713FB
:100E2000FFFF6700832C90083E96034606001410CF
:100E3000BE962380C600850779B7B247850A939985
:100E40000A01939D8A0093D909016391570F854741
:100E50003546DA85130511022300F10293D9890082
:100E600097E00000E78000A8B3ED3D0190000C1072
:100E700022852317B10397000000E78020B059FDB9
:100E80008147A68963EA970626860C084A8597E07B
:100E90000000E78020A581471810B306F70010086E
:100EA00098083E973E9603470700034606008507CD
:100EB000318F2380E600E3E197FE639FA905900848
:100EC0000C10228597000000E78040AB21F9814794
:100ED0009810B306F700900818183E973E960347FF
:100EE0000700034606008507318F2380E600E39163
:100EF000A7FF4109C10CB9BD18089000B306F7005F
:100F00003E963387FC00034707000346060085072B
:100F1000318F2380E600B5B798084E970347070046
:100F20001C10CE972380E700850941BF85473546D1
:100F3000DA85130511022300F10293D9890097E0A5
:100F40000000E780209AB3ED3D0190000C1022854F
:100F50002317B10397000000E78040A2E31005ECDF
:100F6000814718089000B306F7003E963387FC00CF
:100F700003470700034606008507318F2380E600FC
:100F8000E391A7FF41460C084A8597E00000E780FF
:100F9000609581471810B306F700100898083E972F
:100FA0003E9603470700034606008507318F2380DE
:100FB000E600E391A7FF90080C102285970000003F
:100FC000E780C09B1DD599BD7D5582801713FFFF1B
:100FD000E702E31001112A842E859305510032891E
:100FE00002C002C202C402C69304740097F0FFFF5D
:100FF000E780A03D1D46A6851305910097E00000FF
:10100000E780408E10088A854A8597000000E780B7
:10101000E09619ED93071400180883C607000346ED
:10102000070085070507B18EA38FD7FEE397F4FE6F
:1010300005611713FFFF6700C30C1713FFFFE702DB
:1010400063082E848C414111AA8983871500328957
:10105000914463D30700A1449757FF1F9387C72686
:101060009C43A1C7C1CA8D472310F10083C7250047
:101070004A852301F10083C73500A301F10083C72E
:1010800045002302F10083C75500A302F10083C786
:10109000650093059100A30301002303F1002304DD
:1010A000010097F0FFFFE78040320C404A860A8536
:1010B00097F0FFFFE7808033032804008356440045
:1010C000A6881D0881470147E51642868A854E8518
:1010D00097000000E780408E2A8919E5A6852285C1
:1010E00097B0FFFFE780E0C14A8541011713FFFF7A
:1010F000670083004A860A8597F0FFFFE780002F8C
:101100006DB71713FFFFE702E3FB2E848C414111FB
:10111000AA89838715003289914463D30700A144CB
:101120009757FF1F9387471A9C43A1C7C1C68D4796
:101130002310F10083C725004A852301F10083C7EE
:101140003500A301F10083C745002302F10083C7E6
:101150005500A302F10083C7650093059100A30326
:1011600001002303F1002304010097F0FFFFE78053
:10117000C0250C404A860A8597F0FFFFE7800027CC
:1011800083564400032804008A85858EC2061D0804
:10119000C1822312D400A68881470147E516428602
:1011A0004E8597000000E78060B041011713FFFFF4
:1011B000670083F44A860A8597F0FFFFE7800023E3
:1011C0004DBF1713FFFFE70283F1B335B0000111E4
:1011D00085052A891315F601336515012308B10029
:1011E0009305110136843AC632C03EC442C297F01C
:1011F000FFFFE780801DA2471248425593D6870023
:10120000230BF1009305910193578800A30AD100A5
:10121000A30BF100230C010197F0FFFFE780E01A18
:101220003247024603280400B337E00083564400E7
:101230009207914411C2A1444A85A68842860C08AF
:1012400097F0FFFFE78040772A8919E5A685228578
:1012500097B0FFFFE780E0AA4A8505611713FFFFFB
:10126000670023EA1713FFFFE702C3E501113EC63B
:101270008647B335B0008505AA891315F6015D8D43
:101280002308B1009305110136843A89B28442C41F
:1012900046C297F0FFFFE780401322489248164568
:1012A00093578800A30AF1009305910193D7880012
:1012B000230B0101A30BF100230C110197F0FFFF99
:1012C000E780A0103247104083564400B337E00057
:1012D000920703280900914891C0A1480C084E8547
:1012E00097000000E780809CAA8401E983554400B0
:1012F0004A8597B0FFFFE780C0A0268505611713D8
:10130000FFFF670063DFAA959307F00F170701003F
:101310001307075B6317B50013C5F7FF1375F50FC8
:10132000828005058346F5FFB58FBA9783C707000E
:10133000D5B70357450014419307F00F1706010076
:1013400013060658369742074183139506014181DB
:10135000631BE500AD8FB29703C50700130515F3B6
:10136000133515008280850603C5F6FFA98FB29755
:1013700083C70700D9BF1713FFFFE70243D6B28721
:1013800036842E86BA86AA853E85BA8497F0FFFFFA
:10139000E7806052634F0500228597D00000E78008
:1013A000E0782A86A686A285268597F0FFFFE7804B
:1013B00080501713FFFF6700C3D41713FFFFE70226
:1013C00063D05D712A8BAE8A170501001305C54CE9
:1013D0002C00B284368ABA893E8997F0FFFFE780F5
:1013E000C04F2A845DE134104146DA85280097F029
:1013F000FFFFE780404C2A8449E98547A303F100B9
:10140000A6C2930771002408BEC4A68685470D4670
:101410002C18281002DC02DED6C0BEC697F0FFFFF3
:10142000E78000442A8435E183477102A6860D4691
:1014300093F7F7072300FA00C1473EDE2C188947CF
:10144000281026DCA303F10097F0FFFFE78040415E
:101450002A8405ED4146A6854E8597D00000E78099
:1014600060488D47A6860D462C182810A303F1006E
:1014700097F0FFFFE780C03E2A8401E94146A68538
:101480004A8597D00000E780E04522856161171307
:10149000FFFF670063C61713FFFFE70243C497F718
:1014A00000009387E7A0984383C7470079712A8992
:1014B000AE84170501001305A53E0C083AC42306A7
:1014C000F10097F0FFFFE78040412A8405ED1410FA
:1014D0004146CA85080897F0FFFFE780C03D2A848F
:1014E00015E1140815462C00081097F0FFFFE7805F
:1014F000803C2A8401E921462C08268597D00000EB
:10150000E780403E228545611713FFFF670063BFF8
:101510001713FFFFE702A3BC97F7000093874799D3
:101520009C477971AA842E84170501001305C537DD
:101530000C083EC697F0FFFFE780203A0DE9141033
:101540004146A685080897F0FFFFE780C03605E111
:10155000140811466C00081097F0FFFFE780A035D3
:1015600019E58347F10193F7F7032300F400456180
:101570001713FFFF6700E3B81713FFFFE70223B657
:101580003688A14881470147E54697F0FFFFE7808D
:10159000A0421713FFFF6700C3B61713FFFFE70250
:1015A00003B43688A14881470147E54697F0FFFF1D
:1015B000E780C06F1713FFFF6700A3B41713FFFF87
:1015C000E702E3B101112A842E850C0832C697F098
:1015D000FFFFE780803009ED3247970601009386D0
:1015E000262B1008C145228597000000E780E0D82F
:1015F00005611713FFFF6700C3B01713FFFFE70272
:1016000003AE4111C1472EC032C48A8509463EC28D
:101610003EC697F0FFFFE780A02441011713FFFFAC
:10162000670023AE1713FFFFE70263AB4111AE86DD
:1016300013061009AA850A8502C002C202C402C6A6
:1016400097F0FFFFE780202741011713FFFF670096
:1016500043AB1713FFFFE70283A832879706010009
:10166000938606252E869305000297000000E780EA
:10167000C0D01713FFFF6700C3A81713FFFFE702CF
:1016800003A67971C1472ACC2ED032D42C080D463E
:1016900028003ECE3ED23ED602C402C602C802CACE
:1016A00097F0FFFFE780C01B45611713FFFF67003E
:1016B00043A51713FFFFE70283A20111AA842E841A
:1016C000170501001305451F8A8597F0FFFFE78086
:1016D000C02015E514084146A6850A8597F0FFFF4E
:1016E000E780601D09ED8347E1010347F101A2078F
:1016F000D98FCA07C9836177D98F2310F400056198
:101700001713FFFF6700E39F15CD1713FFFFE702D5
:10171000039D9747FF1F9387E76890439745FF1FF7
:10172000938585681745FF1F1305C56397D0000093
:10173000E78000C51745FF1F1305C5621713FFFF9C
:101740006700239C1745FF1F1305C56182808DCD5F
:101750001713FFFFE702A3989747FF1F938787643C
:10176000944301112E840A869745FF1F9385C56314
:1017700097D00000E78040C60A85029401450561C4
:101780001713FFFF6700E3977D5582801713FFFF54
:10179000E702E39497D00000E78080D19747FF1FCE
:1017A00023A2A76017F5FFFF1305E5C997B0000056
:1017B000E780C0741713FFFF6700A3941747FF1F4C
:1017C000130787609317150008433E95FD572310B4
:1017D000F50082801713FFFFE70263902A84084018
:1017E00009E51713FFFF6700C3911C4158401CC057
:1017F0006313E5005CC08347550023200500F99B77
:10180000A302F50097A0FFFFE780207CC9BF171354
:10181000FFFFE702238B9747FF1F9387E75C9843FF
:101820002A8411CB8347350093F7070289C70355F4
:101830000500894502971305440197B00000E78031
:10184000403B835504000355E40097300000E780D7
:10185000A00C485819C597A0FFFFE7800077232AFE
:1018600004021305840397000000E780E0F681443A
:10187000B1499790FFFFE780206A63CBA4028347BA
:1018800034002320040493F727FCA301F40000484C
:101890009790FFFFE7804069131615008145228568
:1018A0009710FFFFE780A0861713FFFF6700C38430
:1018B000B38734030329040385043E994A859700BE
:1018C0000000E78060F12304090065B78347350015
:1018D00093F7070299E3014582808357E500E39C73
:1018E000B7FEC167FD176316F60005458280054502
:1018F00099A81703FFFFE702837E93170601C187AC
:10190000B2842A8401496359F002835705009DCBB4
:1019100001456367F600034584003E953325A60024
:101920001375F50F0DA01C4813171900BA9783D72C
:101930000700E38E97FA05099790FFFFE780C05EE6
:10194000E343A9FE01451703FFFF6700837B1703ED
:10195000FFFFE7022377AE89AA849790FFFFE78015
:1019600060522A8497D0FFFFE780A02EAA86014705
:101970001306840197050000938585E41745FF1F32
:101980001305C5449790FFFFE780E0182A8925C911
:101990008C441304C50022859E0593F5050897A085
:1019A000FFFFE780403CCC4083877400E18163DD2A
:1019B000070493E50508228597A0FFFFE780A03A7A
:1019C0000D4693854400228597A0FFFFE780C0362F
:1019D00083D50400228597A0FFFFE780E03D83D5F3
:1019E0002400228597A0FFFFE780003D03D6490031
:1019F00083A50900228597A0FFFFE780E0334A8591
:101A00001703FFFF6700436F93F5F5076DB71703E3
:101A1000FFFFE702C36C01112A84328532C697A00A
:101A2000FFFFE780E0279780FFFFE780C030835704
:101A300004001747FF1F1307A7523246231BF1006C
:101A4000930700F8A30DF1001C471843231AA100C7
:101A50008983858BB307F740B28548083ECE231CA7
:101A60000100230D010097000000E78080EE056172
:101A70001703FFFF6700E3681703FFFFE7028364B4
:101A8000004101453DC49304C40026853289AE89D6
:101A900097A0FFFFE780C02495452A8A2685035B2F
:101AA000040197A0FFFFE7802021268597A0FFFF74
:101AB000E780603E8D45AA8A268597A0FFFFE780D4
:101AC000A01F268597A0FFFFE780E03C5C48420A04
:101AD000135A0A01D2975CC42318640181476398A2
:101AE0003A0146054D81330625419337160013F51B
:101AF000F70F1703FFFF670023601703FFFFE702DD
:101B0000835B89692A8BAE8B328AB68A8144014411
:101B1000314CFD199790FFFFE780004063CDA40092
:101B20009790FFFFE7804042018D33B5AA0017036D
:101B3000FFFF6700C35B3389840383270B003E9953
:101B400063170A008347890085043E94E1B7035672
:101B50000A00DE854A8533F6C90097000000E78059
:101B6000E0F16DD10545E1B71703FFFFE702235709
:101B700001112A847C000355E5003ECAB70707001F
:101B80003ECC7C003ECE97200000E78020082A89CA
:101B90008545480897A0FFFFE78020399945480808
:101BA00097A0FFFFE780E015AA844A8597200000F0
:101BB000E780A0082380A4009747FF1F9387473A38
:101BC0009C434166130606F09396870113D787015D
:101BD000558F93D68700F18E558FA207B706FF0069
:101BE000F58FD98F11462C00138514003EC497D071
:101BF0000000E78020CF5008A38204008945228599
:101C000097000000E780E0E019C9AA851305840366
:101C100097A0FFFFE780E0313C4085073CC00561AD
:101C20001703FFFF6700E34D1703FFFFE702234B96
:101C30009790FFFFE78040312A8405049790FFFFCB
:101C4000E780802F3305A402F14791453305F50263
:101C500097200000E78020BA11E565551703FFFFC4
:101C60006700234A9747FF1F23A8A7169790FFFFF7
:101C7000E780802D2A8405049790FFFFE780C02B22
:101C80003305A4028945060597200000E780A0B629
:101C900069D59747FF1F23A9A7129790FFFFE780F9
:101CA000A02A2A8405049790FFFFE780E0283304E8
:101CB000A4029747FF1F239B87109790FFFFE780A1
:101CC000A0282A849790FFFFE7800027930714003D
:101CD0003385A7029747FF1F239BA70E9707010095
:101CE000938747811747FF1F2326F70E0145BDB78E
:101CF0001703FFFFE702033DAA842E890144974999
:101D0000FF1F9389E925130A80069790FFFFE7805C
:101D1000A0226347A40001451703FFFF6700C33DEE
:101D20003305440383A709024A86A6853E9597009A
:101D30000000E780E0B919E10504C1BF0545E9BF2E
:101D40001703FFFFE7022337AA8A2E8BB28B368C4C
:101D50003A8A814401448149974CFF1F938C4C205F
:101D6000130D80069790FFFFE780001D63C9A40054
:101D700011E085494E851703FFFF6700433733891C
:101D8000A40383A70C025E86D6853E994A859700F8
:101D90000000E780E0B31DC19790FFFFE780C01A05
:101DA0000544636D4501D2866286DA851305090311
:101DB00097000000E780A0D411C1854985045DB774
:101DC0001703FFFFE7020330C16441112A89014470
:101DD0009749FF1F9389C918130A8006FD1436C658
:101DE00032C42EC29790FFFFE7800015924522462D
:101DF000B2466348A400014541011703FFFF670095
:101E0000A32F3305440383A709023E9509C68347E0
:101E10003500C18B9DC791C68347350093F70702F4
:101E20008DC3630699008357E500639C2701035720
:101E3000050001CB63E7E50083478500BA97E3CD52
:101E4000F5FA050469BF1703FFFFE702A327C16482
:101E50002A8901449749FF1F93898910130A800634
:101E6000FD149790FFFFE780200D6346A400170341
:101E7000FFFF670063283305440383A709023E95EB
:101E80008357E500638A97006304990063962701EE
:101E900097000000E780E0970504E1B71703FFFF14
:101EA000E702E32089692A8AAE8A328BB68B8144A5
:101EB000174CFF1F130CCC0A930C8006314DFD19F3
:101EC0009790FFFFE780400763C6A4001703FFFF5A
:101ED0006700A3213389940383270C028355CA0129
:101EE0005A863E994A8597000000E780609E31C17E
:101EF000814D15A03384AD038327090303D60B005E
:101F0000D68533F6C9003E94228597000000E7800D
:101F1000E0B609E9850D9790FFFFE780E0FFE3CB8E
:101F2000ADFC01A8228597000000E780E08A230429
:101F30000400850471B71703FFFFE702C317416967
:101F4000AA8A014A174BFF1F130B8B017D19C14B46
:101F5000054C9790FFFFE78020FE6346AA00170319
:101F6000FFFF6700C31893098006B3073A0383296C
:101F70000B02BE9983D7E900638E270163842A018F
:101F8000639A570103A4890301E84E859700000076
:101F9000E780C0BD050A75BF8357040163997709BF
:101FA0009304C400268597A0FFFFE78060D3854592
:101FB0002A8D2685835C040197A0FFFFE780C0CFB0
:101FC000268597A0FFFFE780A0E76205618563593A
:101FD00005048D45268597A0FFFFE780E0CD894564
:101FE000268597A0FFFFE78020CD8945268597A00D
:101FF000FFFFE78060CC8545268597A0FFFFE7803F
:10200000E0CC83470500094793F7F707639AE70099
:102010009945268597A0FFFFE78040CBA302850165
:102020004848337D2D01231894016A9548C4004027
:10203000A1BF1703FFFFE702830A37E404008327E9
:10204000041D82979747FF1F83C787DE1715FF1F61
:102050001305C54DA300F5008327441C82978327F1
:10206000841C81461306F00F8145014582971703B2
:10207000FFFF670003091747FF1F130767CB1843CC
:102080009745FF1F83C5C5DA9747FF1F9387C7D8BA
:1020900083468703034697036397D5009747FF1F3F
:1020A0002388C7D8828083C587010347A7036317A6
:1020B000B6009747FF1F238DE7D6828003C68701AE
:1020C0006317C7009747FF1F2384D7D6828083C634
:1020D0008701130750026319D7009307600217475F
:1020E000FF1F2307F7D4828083C68701130660028F
:1020F0006315D60093077002DDB783C7870155BF0C
:102100009747FF1F938747D1D44B0947638DE60854
:102110001703FFFFE702A3FC1749FF1F130909CDAF
:102120003E8483470900918B9DCFB7E4040083A7C9
:10213000041D829783A7441C1745FF1F130585CBF9
:10214000829783A7841C81461746FF1F034686CCCF
:1021500081450145829721C583470900ED9B1747BB
:10216000FF1F2305F7C88347040093F7F70F85CBBC
:1021700091471747FF1F232BF7CA97000000E780FE
:1021800080EB97000000E78040EFB7E70400BC4F0A
:10219000414691451745FF1F034585C882971703A0
:1021A000FFFF670003F682801703FFFFE70223F3B8
:1021B0008D4741116306F504C5476308F50285475D
:1021C0006310F5029747FF1F2386A7C6B7E70400F1
:1021D000BC4B930500101745FF1F034565C482974C
:1021E00041011703FFFF6700C3F185471747FF1F32
:1021F0002302F7C4B7E70400BC4B93050020E1BFFE
:102200009747FF1F938747C1D44B1147638DE60063
:10221000B7E7040083A7071D8297B7E70400BC4B0C
:10222000930500044DBF05491747FF1F232027C111
:1022300083C7070032C62E8493F7F70FD5D3B7E4D0
:10224000040083A7041D7D141374F40F8297E376B2
:1022500089FCB245994703C61500E3F0C7FCFC446E
:1022600009061745FF1F130525BD8297BC48930536
:1022700000081745FF1F0345A5BA829779BF1703CA
:10228000FFFFE702C3E51747FF1F1307E7B8404703
:10229000184B1C409746FF1F23A6F6B86316E400B0
:1022A0001747FF1F2322F7B8130584FE9790FFFFFF
:1022B000E78060A6035564FF9780FFFFE780E06E2C
:1022C00097A0FFFFE78060D01703FFFF670063E37D
:1022D0001703FFFFE702A3E09747FF1F9387C7B3EA
:1022E000D84BDC4789C797000000E78080F9854715
:1022F0001747FF1F232CF7B29747FF1F938747A36A
:102300009C43930500021745FF1F034565B183C732
:1023100087031747FF1F230DF7B0B7E70400BC4B37
:1023200082971703FFFF6700C3DD9747FF1F23A7AF
:10233000A7AE82801703FFFFE702C3D837E404008B
:102340007C4CA1451745FF1F034585AD82977C480E
:10235000A1451745FF1F0345A5AC9744FF1F938474
:10236000A4AB8297DC4489EB97000000E78080D91A
:102370001703FFFF670043D803D567FF9780FFFF70
:10238000E780A062AA896DD1D84891476310F7020F
:102390007C4C91451745FF1F034585A882977C48D3
:1023A00091451745FF1F0345A5A7829703A949013A
:1023B00003D409018947B7E904001747FF1F232702
:1023C000F7A683A7091D21044204829783C78401CD
:1023D0001715FF1F1305851561191717FF1FA30791
:1023E000F71483A7491C418082979747FF1F2383D7
:1023F00007A483A7C91C814609469375F40F4A8533
:10240000829711E99747FF1F83C707B389C79700D2
:10241000FF1FE780207EB7E70400BC4F2146A1459F
:102420001745FF1F0345C59F829799B71703FFFF05
:10243000E702E3CA93F7052001112E8481CF9700AC
:102440000000E78020E91345042005611703FFFF22
:10245000670023CB93F70510A9CF9744FF1F938400
:10246000A49BDC4897000000E78020C11747FF1FAE
:102470001307078C184383C7840103478703631836
:10248000F700DC4489C797000000E78080DF8547BC
:102490001747FF1F232CF798B7E70400BC4B9305A1
:1024A00000021745FF1F0345A597829713450410A7
:1024B00069BF93F70508BDC79747FF1F83C7D79725
:1024C000E91719469745FF1F938525971305D100F6
:1024D00093F4F70F1749FF1F0349099697C00000AF
:1024E000E780404093970401C1831747FF1F1307FC
:1024F0002795231DF100231CF1009747FF1F9387A9
:10250000A7913ACE3ACAD8432306010009CBDC434F
:102510009315890154080D46E1856800829713459B
:10252000040825B793F72500A5C39747FF1F938796
:10253000A78ED84B89476306F7029747FF1F83C7CB
:10254000E78A13F7270011EF918B99CFB7E70400C3
:10255000BC4F1306000A89451745FF1F0345458CEC
:10256000829713452400D5B59737FF1F9387477C83
:102570009C4383C787031747FF1F230BF78A9700E6
:102580000000E78060DBF1BF93F7050281CB970085
:102590000000E78060DA1345040245BD93F785002B
:1025A00081CB97000000E780E0D21345840071BD25
:1025B00093F7150081CB97000000E780A0B4134586
:1025C000140061B593F7450081CB97000000E780C8
:1025D00060B31345440095BD93F7050495C3974731
:1025E000FF1F83C7678391CB97000000E780A0A4FB
:1025F00091471747FF1F232BF78213450404B1B5FA
:1026000093F705010145E38207E49747FF1F93878E
:10261000A780D84B91476310F7049737FF1F938724
:10262000E77C9C4313D727008583D98F858B91E75F
:10263000B7E7040083A7071D8297B7E70400FC4FA4
:1026400091451735FF1F0345A57D829785471737AD
:10265000FF1F232DF77C13450401C5BB9747FF1FC0
:10266000238CA78C82801703FFFFE70243A79737CD
:10267000FF1F23A9077A9737FF1F23A7077A8547EC
:102680001734FF1F1304C46A1737FF1F2320F77A7C
:102690001C4083C787031737FF1F230BF7789790DA
:1026A000FFFFE780A08F29C59717FF1F23A4A7E886
:1026B0001C40170500001305A5D783C787031737EC
:1026C000FF1F2307F7761717FF1FA301F7E69737BA
:1026D000FF1FA3830774B7E7040083A70708829747
:1026E0009737FF1F238EA7721703FFFF670063A1B1
:1026F000B7C7898E938767ED1717FF1F232CF7E263
:1027000045BF1737FF1F03472771795555E797379F
:10271000FF1F9387677003C7170005079736FF1FD2
:10272000A38CE66E03C717008D463377D702973622
:10273000FF1FA383E66E83C617001737FF1F13071B
:10274000275F184393F6F60FA9EE834787031737E1
:10275000FF1F230FF76C85471737FF1F230EF76AFC
:102760009737FF1F938787689C430145998BA9E79B
:102770001703FFFFE702A39637E404007C48C14536
:102780001735FF1F0345C56982973C4885451735B6
:10279000FF1F0345E568829701451703FFFF6700A8
:1027A000439683C7170085466395F60083479703D2
:1027B00079BF8347A70361BF82809737FF1F83C715
:1027C000A765A1CF1703FFFFE702639137E4040079
:1027D0009737FF1F238207647C4885451735FF1F05
:1027E0000345056482977C4C91451735FF1F0345CF
:1027F000256382977C4891451735FF1F0345456245
:1028000082973C48C1451735FF1F03456561829794
:1028100001451703FFFF6700C38E795582801703B8
:10282000FFFFE702C38B2A84035565FF9780FFFFF4
:10283000E780A0179737FF1F9387075ED847BE84AE
:102840001DEF9790FFFFE78080779C4823200400CE
:102850009DEB9737FF1F23A9875C9737FF1F23A3A3
:10286000875CB7E70400BC4B89451735FF1F03455C
:10287000255B829701451703FFFF67008388630A82
:102880008700184375BF80C39737FF1F23AE875853
:10289000C9BF7955CDB71703FFFFE70243849737C8
:1028A000FF1F9387A769884323260500232405007B
:1028B000510597A00000E780C0331703FFFF6700B2
:1028C00043841703FFFFE70283811734FF1F1304BC
:1028D000E4661C40411199CF9C472302B5002AC6EB
:1028E0001CC197000000E78040FB1C409C4B99C333
:1028F0003245829741011703FFFF6700838017F37A
:10290000FEFFE702C37D4111444D328532842EC65D
:102910009790FFFFE780C0522AC422859790FFFF5F
:10292000E780205403A84400630C0800B245835795
:1029300044001840224683D54500AA862685029881
:10294000410117F3FEFF6700C37B17F3FEFFE702A9
:102950000379404D1DC808C09705000093856503A5
:102960001305440197A00000E78040169737FF1F2A
:102970009387C75C9C43014589E79737FF1F23AFC7
:10298000875A17F3FEFF6700C3777D55DDBF17F346
:10299000FEFFE702C374011168009305F00F02C641
:1029A00002C802CA02CC02CE97000000E780A0F164
:1029B000056117F3FEFF6700C3749737FF1F938706
:1029C000E7579C43D847A1679D076319F70217F3A0
:1029D000FEFFE702C370011132859790FFFFE78089
:1029E0002046230AA1008145680097000000E78087
:1029F00080ED056117F3FEFF6700A37082809737B3
:102A0000FF1F9387A7539C43D847A16793877703FA
:102A10006319F70217F3FEFFE702636C01113285B9
:102A20009790FFFFE780C041230AA100814568001D
:102A300097000000E78020E9056117F3FEFF6700BB
:102A4000436C82809737FF1F9387474F9C43D8473B
:102A500095476316F70417F3FEFFE7024368011179
:102A6000328532849790FFFFE780803D230AA100E2
:102A700022859790FFFFE780C03E83574400231BC9
:102A8000A10081453ECC1C4068003ECE970000006E
:102A9000E78060E3056117F3FEFF670083668280CD
:102AA000930785FF8DC38327C5FF91CFDC4B81CF73
:102AB00017F3FEFFE702A362032585FF829717F352
:102AC000FEFF67000364828017F3FEFFE7022361C5
:102AD0002A8432859790FFFFE7808036BD4763EBFD
:102AE000A70018449377F5000345B70041995D8D21
:102AF000A305A70017F3FEFF6700A36017F3FEFF0F
:102B0000E702E35D01117C003ECAB70707003ECC37
:102B10007C003ECE5C4DA9C72A8413858700AE8415
:102B200097A00000E780E0FCA1652A899D05480880
:102B30009770FFFFE780C03A9305803EB345B90226
:102B4000480893F5F50F9790FFFFE780C0210147F4
:102B500081465008A68522859770FFFFE780A05D1B
:102B6000056117F3FEFF6700C35917F3FEFFE70285
:102B7000035797000000E780A0F817F3FEFF6700F7
:102B8000435817F3FEFFE702835501117C00AE8422
:102B90003ECAA165B70707002A843ECC48087C00DE
:102BA000938575033ECE9770FFFFE78060331C442A
:102BB000480883C5B700BD899790FFFFE780A01A3A
:102BC000500801478146A68522859770FFFFE78060
:102BD0008056056117F3FEFF6700A35217F3FEFF4F
:102BE000E702E34F2A84AE8497000000E78000EEFE
:102BF000A685228597000000E780E0F817F3FEFF26
